:020000040800F2
:1000000000000110C1B30308E55F03081D0D0108DE
:10001000C5B40308C5B40308C5B403080000000054
:10002000000000000000000000000000ED5F030879
:10003000E95F030800000000E15F03082D230108C9
:10004000C5B40308C5B40308C5B40308C5B40308A0
:10005000C5B40308C5B40308699700085998000897
:10006000C5B403081D980008E197000809B400080A
:10007000F9B30008E9B30008D9B30008C9B3000810
:10008000B5B30008A1B30008C5B40308C5B403089C
:10009000C5B40308C5B40308C5B40308A597000890
:1000A000C5B4030845140108E513010855140108F7
:1000B000351401082514010815140108C5B40308F6
:1000C000C5B40308C5B40308C5B40308C5B4030820
:1000D000C5B40308898D0008C5B40308ED8C000879
:1000E0002D970008C5B403087D010308C5B40308B3
:1000F000F5130108C5B40308051401088DB3000801
:10010000C5B40308C5B40308C5B40308C5B40308DF
:10011000518C0008C5B40308C5B40308C5B403086E
:1001200079B3000865B3000851B300083DB3000877
:1001300029B30008C5B40308C5B40308C5B403084F
:10014000C5B40308C5B40308C5B403083DFB0208E1
:1001500015B3000801B30008EDB20008B58B000824
:10016000C5B40308C5B40308C5B40308C5B403087F
:10017000C5B40308C5B40308C5B40308C5B403086F
:08018000C5B40308C5B403086F
:100188001400020020290020782900200000000027
:10019800D40500080B100C005C2500207C290020E9
:1001A80000000000D6050008160008009429002069
:1001B8009C29002000000000E20500082700040038
:1001C800B42A0020AC2B002000000000EA0500083B
:1001D80001010400002D0020D03F00200000000095
:1001E8000000000008020900A43F0020D43F0020BE
:1001F80000000000D7810008FF010100CC3F00206B
:10020800E03F002000000000EE05000802000C009E
:10021800B03F0020E43F0020000000000000000084
:1002280010000300B441002000420020000000003C
:10023800F005000828000C00A84100200442002016
:1002480000000000F405000826000800A041002076
:1002580010420020000000000006000823000E00E5
:1002680090410020184200200000000039F60108E3
:1002780019000500884100202842002000000000E5
:1002880008060008F80101008441002030420020DF
:10029800000000000E060008000104008041002054
:1002A8003442002000000000100600081A00080070
:1002B800C441002038420020000000001406000855
:1002C80029005000D44600204847002000000000C4
:1002D800000000000312320002490020D04800202C
:1002E800000000000000000025005A001C48002003
:1002F800764800200000000000000000F601080019
:10030800144800200C4800200000000000000000F5
:1003180001000A00EC4E00203C4F002000000000C5
:100328001C0600080C002400C05000200C5E0020B1
:1003380000000000B59B02080E00DE00C44F00203C
:10034800305E002000000000F116020813000400CF
:10035800F8500020105F0020000000002806000868
:1003680002010300B34F0020145F002000000000CA
:10037800019701082C00100008610020F860002097
:1003880000000000114E02082B0024003C610020F0
:100398001861002000000000E14D02081B00F40075
:1003A800D06100201C63002000000000B1BF0208DB
:1003B80012001600006300201064002000000000F6
:1003C8002C06000801020500806A0020906A0020BF
:1003D8000000000035820308000205005065002077
:1003E800986A002000000000000000001E000400C1
:1003F8008C680020A06A0020000000004206000867
:1004080022000C0010680020A46A002000000000F0
:1004180046060008FB010100388900205C8A00209C
:1004280000000000E9010108FC0109000088002023
:10043800608A002000000000B5010108F7010600ED
:10044800F88700206C8A002000000000520600088F
:100458000A001200647C0020748A0020000000005A
:10046800580600080D002C00387C0020888A0020DF
:1004780000000000114D0308020203002C7C00203C
:10048800B48A0020000000000000000011000C00E9
:10049800AC700020B88A0020000000000198010814
:1004A8000400C00054B80020F0B90020000000008B
:1004B80000000000F90104008CC0002090C000205A
:1004C80000000000C981000818002C0058C0002056
:1004D80094C00020000000001552020806001A000F
:1004E80084BB0020C0C000200000000011170208D3
:1004F80034001000B0BA0020DCC00020000000006A
:10050800ED1903081500700054C300203CC40020F6
:1005180000000000000000000300010050C300209C
:10052800ACC4002000000000000000002A006000A9
:1005380060C20020B0C4002000000000C5190308F4
:10054800FD011E0008C7002064C70020000000004D
:1005580059810008FE010800F4C6002084C7002065
:1005680000000000F10101080500050018C800207E
:10057800B8C80020000000006A060008F501620003
:10058800B0C70020C0C8002000000000657A02083B
:1005980003010600BCC9002004CA002000000000B6
:1005A800700600081F000E0078CF002040D0002001
:1005B800000000007606000805020100C0CF0020F8
:0C05C80050D00020000000008406000855
:1005D40003002B21231E0101000001000A01C409AC
:1005E4000000190128282003000001000001050073
:1005F4000000000100000000000000000115580286
:10060400D903C5030000280100000400FA0000001B
:100614007E05EA05B40532000A0AE8030000640016
:1006240001000000080104000000000100000000B7
:1006340000000000000000000000000000000000B6
:100644000100C800141E010064002C0128002401CC
:100654000000D80E00300100005A00000000900194
:100664002C01C80064000101020001000401010022
:100674000000000000000000010000000005000070
:010684000075
:10068500010000005001000007000000020000000A
:10069500000000000000000001020304060708092D
:1006A50001010000800C04087443040800000000E8
:1006B50000000000900C0408980C040800000000DD
:1006C500012000009C0C0408A40C04080000000094
:1006D50001400000A80C04082417040800000000CD
:1006E50001200000B40C0408C00C04080000000040
:1006F50004000000C40C04087C4404080000000049
:1007050004000000D00C0408843104080000000037
:1007150001000000020000000000803F0000803F53
:10072500FF00000024E203080508040000000000A3
:100735004C0A0408E809040810E203080000000058
:1007450050E2030805080A00000000004C0A0408EE
:10075500E8090408C4E6030800000000FFFFFFFFE6
:10076500006002401060024000000000000B000025
:1007750000002000000000000000000000600240B2
:100785002860024000000000060C00000000200068
:1007950000000000000000000060024040600240D0
:1007A50000000000100D0000000020000000000007
:1007B5000000000000600240586002400000000098
:1007C500160E0000000020000000000000000000E0
:1007D500006002407060024000000000200F000031
:1007E5000000200000000000000000000060024042
:1007F5008860024000000000261000000000200074
:10080500000000000000000000600240A0600240FF
:100815000000000030110000000020000000000072
:100825000000000000600240B860024000000000C7
:10083500362F00000000200000000000000000002E
:10084500006402401064024000000000003800000F
:1008550000004000000000000000000000640240AD
:100865002864024000000000063900000000400036
:1008750000000000000000000064024040640240E7
:1008850000000000103A00000000400000000000D9
:1008950000000000006402405864024000000000AF
:1008A500163B0000000040000000000000000000B2
:1008B500006402407064024000000000203C00001B
:1008C500000040000000000000000000006402403D
:1008D500886402400000000026440000000040003B
:1008E500000000000000000000640240A064024017
:1008F500000000003045000000004000000000003E
:100905000000000000640240B864024000000000DE
:100915003646000000004000000000000000000016
:10092500602204080F000000000000000000000025
:100935000000000028150020FFFFFFFFAC1A040887
:10094500B41A0408BC1A04080000000000000000E6
:100955000000000000000000C41A040804000000A4
:100965001FB102080000000000000000C81A0408BA
:100975000100000000000000000000000000000071
:10098500000000000E000000000000000000000054
:10099500000000000A2900200100C4090000000031
:1009A500082900200100C4090000000006290020D4
:1009B5000100C40900000000042900200100C40949
:1009C50000000000002900200100C409000000000B
:1009D500022900200100C40900000000FE280020B3
:1009E5000100C40900000000FC2800200100C40922
:1009F50000000000644F00200100C8000100000055
:100A0500624F00203200307532000000614F002037
:100A1500055A05005C4F002000FF0100604F0020D3
:100A250001000000BC0200205E4F00200200000013
:100A3500FC0804085B4F002000FF01005F4F002009
:100A450001000000BC0200205D4F002002000000F4
:100A5500FC080408F41A04080F0000000000000058
:100A65000000000000000000C4020020F8C90020BA
:100A75009CFF2C01000000006C1600200A000000FD
:100A8500C4E603088CC90020E0150C17000000001F
:100A95006D16002008000000E80904086E16002005
:100AA500050000004C0A040837650020020000001C
:100AB500DCE60308FE50002001200100FD50002067
:100AC50002000000E8E60308AA5000200000F40137
:100AD50001000000A85000200000F4010100000002
:100AE500A65000200000F40101000000A4500020E1
:100AF5000000F40101000000A250002000FF0100E9
:100B0500BE500020E803D0070A000000BC500020BA
:100B1500006401000A000000BD50002000640100CF
:100B25000A000000B6500020006401000A00000021
:100B3500BB500020006401000A000000BA500020EC
:100B4500006401000A000000B950002000640100A3
:100B55000A000000B550002000FF01000A00000057
:100B6500B450002000FF01000A000000C04F002023
:100B75000000F40101000000BE4F00200000F40158
:100B850001000000BC4F00200000F401010000003E
:100B9500BA4F00200000F40101000000B150002010
:100BA50000C80100B050002000C80100AF5000206F
:100BB50000C80100AE500020006401000A000000DA
:100BC500AD50002000FF01000A000000ED5000209C
:100BD50000C80100EC50002000C80100EB500020C7
:100BE50000C80100EA50002000C80100E9500020BB
:100BF50000C80100E850002000C80100E7500020AF
:100C050000C80100E650002000C80100E5500020A2
:100C150000C80100FC1A04080000000000000000E4
:100C250000000000000000000C1B04080900000083
:100C3500000000006803002004000000141B0408E5
:100C450009000000000000005C0300200400000013
:100C5500B81F040809000000000000005003002030
:100C6500040000001C1B040809000000000000002F
:100C75004403002004000000201B040809000000B4
:100C8500000000003803002004000000281B0408B1
:100C950009000000000000002C03002004000000F3
:100CA500301B04080900000000000000200300209C
:100CB50004000000381B04080900000000000000C3
:100CC5001403002004000000C81A040801000000F5
:100CD500000000000000000000000000000000000F
:100CE5000E000000000000000000000000000000F1
:100CF500401B040800000000000000000000000088
:100D0500000000000844040807000000000000007F
:100D15008C03002000000000501B040808000000A0
:100D25000000000080030020000000005C1B040898
:100D3500080000000000000074030020000000000F
:100D4500C81A0408010000000000000000000000AF
:100D550000000000000000000E0000000000000080
:100D65000000000000000000641B040800000000F3
:100D7500000000000000000000000000741B0408D3
:100D85000D00000000000000C80300200000000066
:100D95007C1B04080D00000000000000BC030020BF
:100DA50000000000841B040807000000000000008C
:100DB500B4030020000000008C1B04080D00000097
:100DC50000000000A803002000000000941B040898
:100DD5000D000000000000009C0300200000000042
:100DE5009C1B04080700000000000000940300207D
:100DF50000000000C81A04080100000000000000FF
:100E05000000000000000000000000000E000000CF
:100E1500000000000000000000000000A41B040802
:100E250000000000000000000000000000000000BD
:100E3500084404080C00000000000000664F002074
:100E450000000000B81B04080C00000000000000B2
:100E5500684F002000000000C81B04080C000000BB
:100E6500000000009E4F002000000000D81B040871
:100E75000C00000000000000924F00200000000060
:100E8500EC1B04080C000000000000006A4F002065
:100E950000000000D80A04080C0000000000000053
:100EA5006C4F002000000000F81B04080C00000037
:100EB500000000006E4F0020000000000C1C04081C
:100EC5000C00000000000000664F0020000000003C
:100ED500141C04080C00000000000000684F0020EE
:100EE500000000001C1C04080C00000000000000AD
:100EF500744F002000000000281C04080C000000AE
:100F050000000000764F002000000000301C04089F
:100F15000C00000000000000784F002000000000D9
:100F25003C1C04080C000000000000007A4F002063
:100F350000000000481C04080C0000000000000030
:100F45007C4F002000000000541C04080C00000029
:100F5500000000007E4F002000000000601C040817
:100F65000C00000000000000804F00200000000081
:100F75006C1C04080C00000000000000824F0020DB
:100F850000000000781C04080C00000000000000B0
:100F9500964F002000000000801C04080C00000093
:100FA50000000000944F002000000000881C040889
:100FB5000C00000000000000A24F0020000000000F
:100FC500941C04080C00000000000000A44F002041
:100FD50000000000A01C04080C0000000000000038
:100FE500AA4F002000000000204404080C00000067
:100FF50000000000844F002000000000AC1C040825
:101005000C000000000000008C4F002000000000D4
:10101500B41C04080C00000000000000864F0020EE
:1010250000000000C01C04080C00000000000000C7
:10103500884F002000000000CC1C04080C000000B4
:10104500000000008A4F002000000000D41C0408A6
:101055000C000000000000008E4F00200000000082
:10106500801404080C00000000000000984F0020C8
:1010750000000000E01C04080C0000000000000057
:10108500904F002000000000EC1C04080C0000003C
:1010950000000000A04F002000000000F81C04081C
:1010A5000C000000000000009A4F00200000000026
:1010B500001D04080C000000000000009C4F0020EB
:1010C50000000000081D04080C00000000000000DE
:1010D500A64F002000000000101D04080C000000B1
:1010E50000000000A84F002000000000C81A0408F6
:1010F50001000000000000000000000000000000EA
:10110500000000000E0000000000000000000000CC
:1011150000000000181D0408000000000000000089
:101125000000000000000000281D04080500000064
:1011350000000000B94F002000000000C81A040894
:101145000100000000000000000000000000000099
:10115500000000000E00000000000000000000007C
:1011650000000000301D0408000000000000000021
:1011750000000000000000007443040800000000A7
:1011850000000000821D0020040000003C1D040832
:101195000D000000D9B0020828040020000000005E
:1011A500204604080D000000CDB102081C040020F3
:1011B50000000000401C04080D000000B1B1020849
:1011C5001004002000000000401D04080800000075
:1011D500000000000404002004000000AC1C04080A
:1011E5000D00000095B00208F80300200000000083
:1011F500481D04080900000000000000EC03002061
:1012050004000000501D04080300000081C7010808
:10121500D403002000000000C81A040801000000E3
:1012250000000000000000000000000000000000B9
:101235000E0000000000000000000000000000009B
:10124500541D04080000000000000000000000001C
:1012550000000000641D04080D00000000000000EF
:101265003C040020000000006C1D04080A0000007A
:1012750000000000FF50002000000000781D040859
:101285000A000000000000000751002000000000D7
:10129500801D04080A000000000000000F51002016
:1012A50000000000881D0408070000000000000081
:1012B5003404002000000000C81A040801000000E2
:1012C5000000000000000000000000000000000019
:1012D5000E000000000000000000000000000000FB
:1012E500941D04080000000000000000000000003C
:1012F50000000000A81D0408070000000000000011
:101305007804002000000000B41D04080800000057
:10131500000000006C04002000000000C01D04084F
:10132500080000000000000060040020000000002C
:10133500CC1D040808000000000000005404002033
:1013450000000000D81D040808000000000000008F
:101355004804002000000000C81A0408010000002D
:101365000000000000000000000000000000000078
:101375000E0000000000000000000000000000005A
:10138500E41D040800000000000000000B1600200A
:1013950000000000F01D04080B0000000000000024
:1013A500E004002000000000F81D04080B00000008
:1013B50000000000D404002000000000041E040802
:1013C5000B00000000000000C80400200000000021
:1013D500101E04080B00000000000000BC040020E3
:1013E500000000001C1E04080B00000000000000A7
:1013F500B004002000000000281E04080B000000B7
:1014050000000000A404002000000000301E0408B5
:101415000B00000000000000980400200000000000
:101425003C1E04080B000000000000008C04002096
:1014350000000000481E040808000000000000002D
:101445008004002000000000C81A04080100000004
:101455000000000000000000000000000000000087
:101465000E00000000000000000000000000000069
:10147500541E0408000000000000000000000000E9
:1014850000000000681E04080800000000000000BD
:101495001005002000000000741E0408080000006C
:1014A500000000000405002000000000801E040864
:1014B5000800000000000000F80400200000000003
:1014C5008C1E04080800000000000000EC04002049
:1014D50000000000C81A0408010000000000000018
:1014E5000000000000000000000000000E000000E9
:1014F500000000000000000000000000941E040829
:101505000000000000000000081600200000000098
:10151500A41E04080B000000000000004005002088
:1015250000000000B01E04080B00000000000000D1
:101535003405002000000000BC1E04080700000060
:10154500000000002C05002000000000C81E040853
:101555000700000000000000240500200000000036
:10156500D41E040807000000000000001C05002030
:1015750000000000C81A0408010000000000000077
:101585000000000000000000000000000E00000048
:10159500000000000000000000000000E01E04083C
:1015A50000000000000000000816002000000000F8
:1015B500EC1E040807000000000000008C05002058
:1015C50000000000F41E04080700000000000000F1
:1015D5008405002000000000FC1E04080700000030
:1015E500000000007C05002000000000041F040826
:1015F5000700000000000000740500200000000046
:101605000C1F040807000000000000006C05002006
:1016150000000000141F040807000000000000007F
:1016250064050020000000001C1F040807000000DE
:10163500000000005C05002000000000241F0408D5
:101645000700000000000000540500200000000015
:101655002C1F040807000000000000004C050020B6
:1016650000000000C81A0408010000000000000086
:101675000000000000000000000000000E00000057
:10168500000000000000000000000000341F0408F6
:101695000F000000000000004D38020800000000A7
:1016A50094050020B74F00200A320100B64F0020F4
:1016B50001FA0100B24F002000C80100B04F002020
:1016C500E803D00701000000434C524143494E470F
:1016D500463400005A4F002000030100594F0020F6
:1016E500000301003C1F04080F00000089370208B1
:1016F500653702080000000070060020481F040836
:101705000F0000002D370208ED360208000000002A
:10171500E8060020541F04080F000000C537020822
:10172500AD370208000000009C070020601F040878
:101735000F0000006338020800000000A13A02080B
:10174500940A0020681F04080F00000059B1020820
:101755000000000000000000E40A0020701F0408DB
:101765000F000000CD3B0208A13B02089D3A02088C
:10177500C00B0020781F04080F000000193902086B
:10178500E938020800000000600C0020801F0408F2
:101795000F00000095390208D93902080000000041
:1017A500000D0020B2500020010301008C1F040829
:1017B5000F000000B5380208893802080000000053
:1017C500F00D0020941F04080F000000493902089D
:1017D500D13A0208000000007C0E0020A01F04087A
:1017E5000F000000053A02081D3B0208000000003A
:1017F5001C0F0020AC50002001030100A81F0408A5
:1018050000000000000000000000000000000000D3
:10181500B41F040808000000000000003C10002070
:1018250000000000BC1F04080700000000000000C5
:101835003410002000000000CC1F04080700000041
:10184500000000002C10002000000000D81F040834
:101855000700000000000000241000200000000028
:10186500E41F04080300000081C701080C100020D4
:1018750000000000C81A0408010000000000000074
:101885000000000000000000000000000E00000045
:10189500000000000000000000000000EC1F04082C
:1018A5000000000000000000000000000000000033
:1018B500FC1F04080A00000000000000DC0C0408FE
:1018C50000000000042004080A00000000000000D9
:1018D500FC150408000000000C2004080A000000A4
:1018E50000000000EE500020000000001420040855
:1018F5000A00000000000000481000200000000061
:10190500C81A0408010000000000000000000000E3
:1019150000000000000000000E00000000000000B4
:1019250000000000000000001C200408000000006A
:10193500000000000000000000000000282004084E
:101945000300000081C7010894100020000000007A
:101955004C1F04080300000081C701087C1000200B
:1019650000000000401F04080300000081C70108B3
:101975006410002000000000342004080500000069
:1019850000000000584F0020000000003C20040823
:1019950007000000000000005C10002000000000AF
:1019A5004820040807000000000000005410002033
:1019B50000000000C81A0408010000000000000033
:1019C5000000000000000000000000000E00000004
:1019D5000000000000000000000000005420040882
:1019E50000000000000000000000000000000000F2
:1019F500B80B04080300000081C70108DC100020B3
:101A050000000000682004080300000081C70108E9
:101A1500501B002000000000702004080300000097
:101A250081C70108C41000200000000078200408C8
:101A35000300000081C70108AC1000200000000071
:101A4500C81A0408010000000000000000000000A2
:101A550000000000000000000E0000000000000073
:101A650000000000000000008420040800000000C1
:101A750000000000000000000000000090200408A5
:101A850007000000693B02087411002000000000F7
:101A9500D01C04080300000081C701085C11002068
:101AA500000000009C2004080300000081C7010815
:101AB5004411002000000000A420040803000000D9
:101AC50081C701082C11002000000000AC2004088B
:101AD500070000004D3B0208241100200000000013
:101AE5003C4604080300000081C701080C110020D2
:101AF50000000000B82004080300000081C70108A9
:101B0500F410002000000000C81A040801000000BD
:101B150000000000000000000000000000000000C0
:101B25000E000000000000000000000000000000A2
:101B3500C42004080F00000015380208DD3702082C
:101B4500000000007C110020CC2004080F000000DC
:101B5500713A020800000000000000001C1200207D
:101B6500D82004080F000000D1360208B536020857
:101B750000000000A8120020E02004080F0000006B
:101B85000000000000000000000000005C130020C1
:101B9500F02004080F000000493A0208853B0208BE
:101BA50000000000E8130020F820040800000000F1
:101BB50000000000000000000000000004210408EF
:101BC5000300000081C70108101500200000000077
:101BD500E42004080300000081C70108F814002070
:101BE50000000000DC2004080300000081C7010894
:101BF500E0140020000000000C2104080300000090
:101C050081C70108C814002000000000182104083D
:101C15000300000081C70108B01400200000000087
:101C250020210408020000006DC501080000000025
:101C35000000000028210408020000006DC501080D
:101C4500010000000000000034210408020000002B
:101C55006DC5010802000000000000000000000042
:101C65000E00000000000000000000000000000061
:101C750001000000ADFC01080000000000000000AC
:101C8500010000000000803F20700020702D7200D0
:101C9500FA00000001000000010000000101010040
:101CA50009024300020100C03209040000010202DA
:101CB500010005240010010524010001042402028D
:101CC5000524060001070582030800FF0904010039
:101CD500020A000000070501024000000705810215
:101CE50040000000FF0000000000010101010100AB
:101CF50000000000010203040102030406070809AD
:101D0500E00100000000803F08FFFF000001010125
:101D15000100000004030904120100020202004050
:101D2500830440570002010203010000F5B80208D0
:101D3500116D0208F5B3020891670208BD6C02082F
:101D4500A1670208BD67020881670208716702087A
:101D5500000000000000000001000000AC140408B1
:101D6500000000000000000011970108A086010096
:101D7500040000000000000000000000000000005A
:101D8500000000000000000000000000000000004E
:101D9500D01C04081014040800000000B923010831
:101DA5007D000000060000000000000000000000AB
:101DB500000000000000000000000000000000001E
:101DC5000000000098440408000000000000000026
:101DD50031A40308E8030000030000000000000030
:101DE50000000000000000000000000000000000EE
:101DF5000000000000000000A044040800000000EE
:101E0500000000001518020810270000030000005C
:101E150000000000000000000000000000000000BD
:101E2500000000000000000000000000AC440408B1
:101E350000000000854C020891730108204E000047
:101E45000500000000000000000000000000000088
:101E5500000000000000000000000000000000007D
:101E6500442A04080000000000000000ED9E03085D
:101E75001027000001000000000000000000000025
:101E8500000000000000000000000000000000004D
:101E950000000000B044040800000000000000003D
:101EA50081010108E80300000500000000000000B2
:101EB500000000000000000000000000000000001D
:101EC5000000000000000000BC4404080000000001
:101ED50000000000419A0108204E000003000000A8
:101EE50000000000000000000000000000000000ED
:101EF500000000000000000000000000CC440408C1
:101F050000000000000000004B980108204E000072
:101F150003000000000000000000000000000000B9
:101F250000000000000000000000000000000000AC
:101F3500DC44040800000000000000004D9D03087B
:101F4500400D030003000000000000000000000039
:101F5500000000000000000000000000000000007C
:101F650000000000400B0408000000000000000015
:101F7500995B030810270000010000000000000025
:101F8500000000000000000000000000000000004C
:101F950000000000000000001C1404080000000000
:101FA5000000000085D00208102700000300000093
:101FB500000000000000000000000000000000001C
:101FC500000000000000000000000000840B040871
:101FD50000000000000000005D4D0308A00F000098
:101FE50001000000000000000000000000000000EB
:101FF50000000000000000000000000000000000DC
:10200500EC4404080000000000000000297F0208DD
:102015001027000001000000000000000000000083
:1020250000000000000000000000000000000000AB
:1020350000000000881504080000000000000000F2
:102045003D970108A00F00000100000000000000FE
:10205500000000000000000000000000000000007B
:102065000000000000000000DC2004080000000063
:1020750000000000513C03081A4100000100000067
:10208500000000000000000000000000000000004B
:102095000000000000000000000000009827040870
:1020A5000000000000000000419103081027000017
:1020B500010000000000000000000000000000001A
:1020C500000000000000000000000000000000000B
:1020D500684204080000000000000000C13C02083E
:1020E5001A4100000100000000000000000000008F
:1020F50000000000000000000000000000000000DB
:1021050000000000F8440408000000000000000082
:10211500ED4C0308400D0300000000000000000026
:1021250000000000000000000000000000000000AA
:102135000000000000000000004504080000000049
:1021450000000000359C0108A08601000300000086
:10215500000000000000000000000000000000007A
:10216500000000000000000000000000296C0208CB
:10217500E16B0208316B0208000000004D670208A0
:10218500856A0208056B0208ED6902080000000077
:10219500000000004167020839F2020835F2020822
:1021A50031F2020825F2020821F202082DF2020896
:1021B50029F20208ADF20208A1F2020879F202083A
:1021C5008DF2020865F2020851F202083DF202089A
:1021D500C04604080F000000F97103080000000064
:1021E50000000000D01C00209446040800000000F8
:1021F5000000000000000000000000007443040817
:1022050000000000000000003C1D0020040000004C
:10221500204604080D0000002D77030898210020B2
:1022250000000000401C04080D00000003770308AF
:102235008C21002000000000401D0408080000005B
:10224500000000008021002004000000AC1C0408F0
:102255000D000000A1750308742100200000000096
:10226500501D04080300000081C701085C210020FF
:1022750000000000A44604080300000081C701080F
:102285004421002000000000C81A040801000000D5
:102295000000000000000000000000000000000039
:1022A5000E0000000000000000000000000000001B
:1022B5009446040800000000000000000000000033
:1022C5000000000074430408000000000000000046
:1022D5003C1D002004000000D04504080300000058
:1022E500997303082C21002008000000AC1C040889
:1022F5000D000000A17503087421002000000000F6
:10230500501D04080300000081C701085C2100205E
:1023150000000000A44604080300000081C701086E
:102325004421002000000000C81A04080100000034
:102335000000000000000000000000000000000098
:102345000E0000000000000000000000000000007A
:10235500AC4604080000000000000000000000007A
:1023650000000000744304080000000000000000A5
:102375003C1D002004000000D845040803000000AF
:1023850081C70108A421002000000000C81A040824
:102395000100000000000000000000000000000037
:1023A500000000000E00000000000000000000001A
:1023B5000000000000FFFF00000000002D202D2D73
:1023C500202D2D2D2D202D2D2D000000000000008D
:1023D5000000000000000000000000AA55050100F3
:1023E50000AA550B010000AA5507010000AA5509CE
:1023F50002000000AA5503009F0000000100000034
:10240500C0122D202D2D202D2D2D2D202D2D2D2DA6
:1024150000000000000000000000000000000000B7
:10242500000000007AC9002088130C170100000085
:102435007CC9002088130C170000000028450408FB
:102445000000000000000000000000000000000087
:10245500384504080800000000000000B01D0020F9
:1024650004000000444504080800000000000000C6
:10247500A41D002000000000501D040804000000F9
:10248500857703080000000000000000C81A040852
:102495000100000000000000000000000000000036
:1024A500000000000E000000000000000000000019
:1024B5000000000078C9002088130C1701000000F7
:1024C50076C9002088130C17000000008045040819
:1024D5000F00000049720308000000000000000022
:1024E500BC1D002089C90020010000000C0A040859
:1024F50075C9002001000000180A04087EC90020E3
:1025050002000000200A0408EAB9002000000000CB
:1025150000000000E8B900200000000000000000F5
:10252500E6B900200000000000000000E4B900202A
:102535000000000000000000E2B9002000000000DB
:1025450000000000E0B900200000000000000000CD
:10255500801D0020000000000000000074C900205C
:10256500020000002C0A0408884504080000000049
:1025750000000000000000000000000038450408CD
:102585000800000000000000401E002004000000BC
:10259500444504080800000000000000341E002027
:1025A50000000000501D0408040000002972030803
:1025B5000000000000000000C81A04080100000027
:1025C5000000000000000000000000000000000006
:1025D5000E000000000000000000000000000000E8
:1025E50098450408000000000000000000000000FD
:1025F50000000000A84504080D000000457603080A
:102605007C1E002004000000B44504080D000000F5
:102615006D720308701E002004000000C045040808
:102625000D00000011760308641E00200000000064
:10263500CC45040803000000B97303084C1E0020B4
:1026450008000000D84504080300000081C7010800
:10265500A421002000000000C81A040801000000A1
:102665000000000000000000000000000000000065
:102675000E00000000000000000000000000000047
:10268500BC1A040800000000000000000000000063
:1026950000000000C41A040804000000E5770308E0
:1026A5000000000000000000C81A04080100000036
:1026B5000000000000000000000000000000000015
:1026C5000E000000000000000000000000000000F7
:1026D500284604080000000000000000000000007B
:1026E50000000000242B04080D000000000000007D
:1026F500DC1E002004000000384604080800000025
:1027050000000000D01E002004000000444604081C
:102715000800000000000000C41E002004000000A6
:102725004C4604080800000000000000B81E002008
:1027350004000000544604080800000000000000E2
:10274500AC1E0020040000005C46040808000000E0
:1027550000000000A01E00200400000064460408DC
:102765000800000000000000941E00200400000086
:102775006C4604080800000000000000881E0020C8
:1027850004000000C81A0408010000000000000051
:102795000000000000000000000000000E00000026
:1027A500000000000000000000000000744604085E
:1027B5000F0000003972030800000000000000004F
:1027C500E81E00207C4604080F0000000000000001
:1027D5000000000000000000601F0020844604087F
:1027E5000F000000000000000000000000000000D5
:1027F500002000208BC9002004000000380A0408CE
:1028050070C90020E0150C170000000073C90020F6
:1028150008000000E809040872C90020050000004E
:102825004C0A04088C4604080F0000000000000054
:102835000000000000000000502000200100000002
:102845004300000000000000000000000000000040
:102855000000000000000000000000000000000073
:102865004300000000000000000000000000000020
:102875000000000000000000000000000000000053
:102885004300000000000000000000000000000000
:102895000000000000000000000000000000000033
:1028A50043000000000000000000000000000000E0
:1028B5000000000000000000000000000000000013
:1028C50043000000000000000000000000000000C0
:1028D50000000000000000000000000000000000F3
:1028E50043000000000000000000000000000000A0
:1028F50000000000000000000000000000000000D3
:10290500430000000000000000000000000000007F
:1029150000000000000000000000000000000000B2
:1029250041B7030881B503080000000052470408B9
:10293500C81504082C2404082C2404082C24040895
:102945002C2404082C2404082C2404082C24040812
:102955002C2404082C240408FFFFFFFFFFFFFFFFC2
:10296500FFFFFFFFFFFF00000100415343494900FE
:102975000000000000000000000000000000000052
:1029850000000000000000000000415343494900D9
:102995000000000000000000000000000000000032
:1029A50000000000000000000000000030230020AF
:1029B5000000000000000000000000000000000012
:1029C5000000000000000000000000000000000002
:1029D50000000000000000000000000000000000F2
:1029E50000000000000000000000000000000000E2
:1029F50000000000000000000000000000000000D2
:102A050000000000000000000000000000000000C1
:042A150001000000BC
:10800000436B826A816930B41C68456A24F00104BC
:108010001144AA421C60D9600DD3016900248A1A58
:108020005A6084621A68002142F0010280F84C1004
:1080300030BC1A607047AA1A5A608562F2E700BF26
:10804000436A8269F0B4D154436A0469426B0133D4
:10805000A34228BF00234362FAB1116811F0010165
:1080600001D0F0BC7047856A1768866927F0010760
:108070002E449D421760D6600BD3641B546081620E
:108080001368002143F0010380F84C10F0BC13602A
:1080900070475D1B55608362F2E7826DD36843F0E1
:1080A0008003D360DDE700BF026B10B462B1836C64
:1080B000C2684469D11A013B615C5DF8044B08BF9A
:1080C00013468364C8B27047016A4369C4685B5C45
:1080D0000131A14228BF114601625DF8044BD8B2BC
:1080E000704700BF436B13B190F84C007047836A30
:1080F000406A181AB0FA80F040097047416A836AF2
:1081000099420AD3CB1A416B026961B14968501E8A
:108110000B4483420AD2C01A704702691144CB1A39
:10812000416B0029F2D1501EC01A704700207047E1
:10813000036B43B1826C5B6893422FBF981AC0688F
:108140009B1AC0187047C269036A9A422FBFD01A9F
:10815000C0688018C01A70470A4B30B503F110048C
:1081600093F900205D78072AC8BF143A81180433B8
:108170008D7213F8025C855413F8012C0A75A34222
:10818000EED130BD3CDD030803682DE9F041DF6925
:108190001FB13B46BDE8F0411847002A164611DDE5
:1081A00004460D460E4400E023689B68204698472D
:1081B0000028F9D0236815F8011B1B682046984752
:1081C000AE42F1D1BDE8F081002325220270437058
:1081D0008370C370704710B5074B03F10C0193F91E
:1081E00000205C78845402449C78D470DC789471CC
:1081F00004338B42F3D110BD4CDD0308F0B5446865
:1082000014B12568A4886C8341F08001046840F2B1
:10821000E93501E0002D58D02689013D16F0020F06
:10822000ADB2F7D089B2A18140F2E93101E0002975
:1082300060D02589013915F0010F89B2F7D0A189E5
:10824000A1894FF0000C4FF47A714FF6FF764FF092
:10825000FF0E624502D131E0B1421BD025890139C0
:1082600015F0020589B2F7D0A4F80CE04FF47A714A
:1082700002E0B9B2B1420DD0258915F0010501F136
:10828000FF37F6D0A589ADB20BB11D7001330CF1EB
:10829000010CDEE7244B9C4208D0A3F578439C42B6
:1082A0003CD003F580639C4208D102251F4B03EBB1
:1082B00005156B8901339BB26B816B89436813B1E0
:1082C0001A689B8813830120F0BD17498C4208D09F
:1082D000A1F578418C4223D001F580618C42AFD169
:1082E0000225124901EB05156989013189B26981BD
:1082F0006989A5E70C4DAC4207D00D498C4211D0DD
:1083000001F580618C429BD10221084D05EB0111E2
:108310004D890135ADB24D81498991E70125C5E708
:108320000125DEE70121F0E70030014010C5002003
:108330000038004030B4446814B12368A5885D83D8
:10834000036840F2E93001E0002833D01D8901388C
:1083500015F0020F80B2F7D089B2998140F2E9316D
:1083600001E0002950D01889013910F0010F89B2BD
:10837000F7D0998940F2E93101E000292FD018891E
:10838000013910F0020F89B2F7D092B29A8140F20F
:10839000E93201E0002A4BD01989013A11F0010FAE
:1083A00092B2F7D09B8914B12368A2881A83012066
:1083B00030BC70472C498B4208D0A1F578418B42E4
:1083C0004CD001F580618B42D4D10220274901EBCA
:1083D00000104189013189B241814189CAE7224AAD
:1083E000934208D0A2F57842934235D002F58062DC
:1083F0009342D8D102211D4B03EB01114B8901336C
:108400009BB24B814B89CEE71748834207D018496E
:108410008B4227D001F580618B42ABD102211348FA
:1084200000EB01114889013080B248814989A1E7F8
:108430000D498B4207D00E4A934211D002F580625B
:108440009342B0D10222094B03EB0212538901334C
:108450009BB253815389A6E70121CCE70120B5E700
:108460000122F0E70121DAE70030014010C50020C9
:1084700000380040002870B51EDB0928044620DDC6
:10848000012303EB83035B00B0FBF3F2092AF8D866
:108490007BB10E4EB4FBF3F00928CCBF572230223B
:1084A000A6FB03E5024403FB1044EB0801F8012B93
:1084B000F0D100230B7070BD2D230B7040420131B1
:1084C000DBE7303001F8010BF3E700BFCDCCCCCCBB
:1084D000884230B44FF001042ED301FB04F4B0FB0A
:1084E000F4F58D42F9D284B1AAB901E0B0FBF4F5FC
:1084F000092DCCBF572230222A4404FB150003F873
:10850000012BB4FBF1F4002CF0D100221A7030BC26
:108510007047B0FBF4F5092DCCBF372230222A4436
:1085200004FB150003F8012BB4FBF1F4002CF0D18F
:1085300000221A7030BC70470546002AEBD1D7E7FD
:1085400003685A1C02601970704700BF2DE9F0479C
:10855000089C2578002B804689460CBF4FF0200AE6
:108560004FF0300A661C35B3002A29DD334601E09E
:10857000024698B113F8011B501E0029F8D1971E2E
:1085800060B13D46013D51464046C8476B1C002B3B
:10859000F8DC257827EAE770013055B1041B29463D
:1085A0004046C847301916F8015B002DF7D1BDE8E9
:1085B000F087BDE8F087002A04DC2846BDE8F08794
:1085C0000020EBE7571EDCE70A44914251D030B45B
:1085D00041F2210411F8013B80EA0320430010F42A
:1085E000004F84EA03059BB2ADB208BF1D466B0085
:1085F00015F4004F84EA03009BB280B208BF18460E
:10860000430010F4004F84EA03059BB2ADB208BFEB
:108610001D466B0015F4004F84EA03009BB280B244
:1086200008BF1846430010F4004F84EA03059BB2CC
:10863000ADB208BF1D466B0015F4004F84EA03007D
:108640009BB280B208BF1846430010F4004F84EA82
:1086500003059BB2ADB208BF1D466B0084EA030060
:1086600015F4004F85B298B218BF28468A42B1D19E
:1086700030BC704783684268D0ED037A00EB830119
:108680000133934281ED040A836004BF00238360B9
:1086900000EB830393ED047A036870EE277A9A4225
:1086A000C0ED037A77EEC77AC0ED037A0CDA0133B6
:1086B00007EE103AF8EEC76AB7EE007A87EEA60A20
:1086C000036030EE070A704707EE102AB8EEC77A4B
:1086D00087EE870A704700BF90ED097A90ED004A57
:1086E000D0ED0A6AD0ED014AD0ED047A90ED035A3C
:1086F000D0ED025AA4EE007AB0EE406AB0EE470A1E
:10870000B0EE667AA6EE247A67EEC07AA0EE457ADD
:10871000E6EE257A80ED097AC0ED0A7A704700BF4F
:10872000D0ED057A90ED013AD0ED003AD0ED064A51
:1087300090ED024A90ED077A90ED035A90ED086AA9
:10874000D0ED045AC0ED067AF0EE406A27EE830AB7
:10875000C0ED056AA3EEA60A80ED087AA4EE240A0D
:10876000A5EE470AA5EEC60A80ED070A704700BFCE
:10877000D0ED007A90ED017A30EE670AE7EE007AEC
:10878000B0EE670AC0ED007A704700BF704700BFC7
:108790004FF480530382704750F8043C012280F864
:1087A0003520143803B11847704700BFBFF34F8F0F
:1087B0000549064BCA6802F4E0621343CB60BFF37D
:1087C0004F8F00BFFDE700BF00ED00E00400FA0599
:1087D000F8B5027B466903681F2A2DD9A2F120054E
:1087E0005F682024AC402742114617D01022AA40CF
:1087F000DC60DA605A68EA40D40749D4716B756A64
:108800000A68B46A22F00102A5420A6037D1012247
:1088100086F84C20027B11461F2A20D920390822D5
:1088200058688A40024200D0DA600422586802FA8E
:1088300001F1014221D1F8BD20241D689440254258
:1088400011460CD0102191409C6099601968D1406C
:10885000C907D3D5012101FA02F29A60CEE70822B6
:1088600018688A40024200D09A600422186802FA0E
:1088700001F101420BD09960F8BDD960F8BD044602
:108880003046FFF7BDFB227B23681146C4E7F8BDE5
:10889000012202FA05F5DD60B0E700BF70B4037B8A
:1088A00004681F2B08D9203B2021626801FA03F3DA
:1088B0001A421CD170BC70472021226801FA03F3D0
:1088C0001A42F7D042691449582000FB021251683D
:1088D0005689CD680868296821F0010129608289DC
:1088E00092B222EA06028281A36070BC704742699C
:1088F0000949582000FB021251685689CD68086862
:10890000296821F001012960828992B222EA0602D7
:108910008281E36070BC7047B0BB002030B4094B6B
:108920001C786CB1084A002502EBC40411689388D6
:108930004D628889083203439BB2A2428B81F5D1F4
:1089400030BC7047D0BF0020D4BF002010B4037BE0
:1089500001681F2B09D9203B20224C6802FA03F33F
:108960001C4214D15DF8044B704720220C6802FAB7
:1089700003F31C42F6D00C4A4068002414700268CD
:108980005DF8044B22F0010202608B607047064ADA
:1089900040680024147002685DF8044B22F0010264
:1089A0000260CB60704700BFD362002090F849306E
:1089B00013B1002280F849201846704770B504466C
:1089C00082B00830256A6B4606223B21A847A8B131
:1089D0009DF804009DF800609DF801109DF802507C
:1089E0009DF803209DF8053041EA062143EA002363
:1089F00042EA05226182A282E382012002B070BDB8
:108A0000F8B50468C4F30D0405460E4604B32F6898
:108A100023F084F8092840F08880454C236923F42A
:108A200040732361236943F400732361236943F096
:108A3000010323613E6023F071F82369092823F0C4
:108A40000103236171D12B6804332B600020F8BD32
:108A5000384B394A93422BD902F58042934226D9AA
:108A600002F5804293422AD902F58042934228D9E6
:108A700002F58032934226D902F50032934224D97E
:108A800002F50032934222D902F50032934220D9F6
:108A900002F5003293421ED902F5802293421CD97E
:108AA000B3F1016F1BD3052008F0F4FEFBE70824A7
:108AB00023F034F8092814D04FF0FF30F8BD10240B
:108AC000F6E71824F4E72024F2E72824F0E730241E
:108AD000EEE73824ECE74024EAE74824E8E75824A6
:108AE000E6E7134F3B6923F440733B613B6943F472
:108AF00000733B613B6923F0F8033B613B6943F042
:108B000002031C433C613B6943F480333B6123F027
:108B100005F83B6923F002033B613B69092823F018
:108B2000F8033B613FF473AFC6E76FF00100F8BD97
:108B3000003C024000400008FF3F0008F8B5044632
:108B40000D468E180027B54201D12069F8BDE368B3
:108B5000591CE160234415F8012B1A720429F2D143
:108B6000206918B9A1682046FFF74AFF2061E76035
:108B7000E9E700BF70B582B00446694618302AF0B4
:108B80005BFCA8B19DF805009DF801609DF80210FE
:108B90009DF803509DF804209DF8063041EA062117
:108BA00043EA002342EA0522A184E28423850120CE
:108BB00002B070BD38B5254B5C69236B73B1A36DF2
:108BC000626BCAB1998A1A88C90592B201D5D207D7
:108BD00000D438BD4FF6F7721A8038BDA36D99895D
:108BE0001A88890692B2EBD59206E9D5E26ACAB133
:108BF000988880B29047E2E799891A880D0692B268
:108C0000E0D51006DED5A26A616A8A4219D0A16950
:108C10002569885C98800132B2FBF5F105FB1122D1
:108C2000A262CFE79B88E2696169DBB28B54E2699B
:108C3000E068A36D0132B2FBF0F100FB1122E261AA
:108C4000BEE7DA6822F08002DA60BBE78C3F0020E2
:108C500038B5254BDC68236B73B1A36D626BCAB169
:108C6000998A1A88C90592B201D5D20700D438BDB5
:108C70004FF6F7721A8038BDA36D99891A88890654
:108C800092B2EBD59206E9D5E26ACAB1988880B271
:108C90009047E2E799891A880D0692B2E0D510064E
:108CA000DED5A26A616A8A4219D0A1692569885C09
:108CB00098800132B2FBF5F105FB1122A262CFE7E9
:108CC0009B88E2696169DBB28B54E269E068A36D5D
:108CD0000132B2FBF0F100FB1122E261BEE7DA687B
:108CE00022F08002DA60BBE78C3F002038B5254BCC
:108CF0009C68236B73B1A36D626BCAB1998A1A88A1
:108D0000C90592B201D5D20700D438BD4FF6F7722B
:108D10001A8038BDA36D99891A88890692B2EBD55D
:108D20009206E9D5E26ACAB1988880B29047E2E734
:108D300099891A880D0692B2E0D51006DED5A26A8E
:108D4000616A8A4219D0A1692569885C98800132DC
:108D5000B2FBF5F105FB1122A262CFE79B88E26925
:108D60006169DBB28B54E269E068A36D0132B2FB4A
:108D7000F0F100FB1122E261BEE7DA6822F0800226
:108D8000DA60BBE78C3F002038B5254B1C68236BAD
:108D900073B1A36D626BCAB1998A1A88C90592B280
:108DA00001D5D20700D438BD4FF6F7721A8038BD0E
:108DB000A36D99891A88890692B2EBD59206E9D5F6
:108DC000E26ACAB1988880B29047E2E799891A8826
:108DD0000D0692B2E0D51006DED5A26A616A8A421B
:108DE00019D0A1692569885C98800132B2FBF5F140
:108DF00005FB1122A262CFE79B88E2696169DBB2C1
:108E00008B54E269E068A36D0132B2FBF0F100FB24
:108E10001122E261BEE7DA6822F08002DA60BBE785
:108E20008C3F002003685B6A03B11847704700BF9E
:108E300003681B6A03B11847704700BF03682DE938
:108E4000F041DF691FB13B46BDE8F0411847002AF9
:108E5000164611DD04460D460E4400E023689B686B
:108E6000204698470028F9D0236815F8011B1B6895
:108E700020469847AE42F1D1BDE8F08103689B6976
:108E8000184700BF03685B69184700BF03681B6988
:108E9000184700BF0368DB68184700BF03689B687A
:108EA000184700BF03685B68184700BF03681B686A
:108EB000184700BF014B1868F8E700BF58D00020E2
:108EC00038B50C46097849B1054601342B68284667
:108ED0001B68984714F8011B0029F7D138BD00BF63
:108EE000064B53F820302BB11A689B8851690B420E
:108EF00001D1138370475383704700BF28C70020F8
:108F0000026802F13F4303F57E032DE9F04F9B0A0F
:108F1000544DEB5C03F01F055B090124032B04FA9D
:108F200005F400F09980042B00F09180022B3ED0D4
:108F300001F00306731E012BC1F3810CC1F300186D
:108F40008588C1F3411137D90024234601274FF00A
:108F5000030E03E0102B04F1020426D007FA03F0FD
:108F6000A84303F10103F5D1D2F800C00EFA04F0D2
:108F7000C04300EA0C0CC2F800C0D2F8008006FA28
:108F800004FC4CEA080CC2F800C0D2F80CC000EA9D
:108F90000C00D060D2F80CC001FA04F040EA0C00DA
:108FA000102BD06004F10204D8D1BDE8F08F2E4B15
:108FB0005D6C2C435C64BBE7002003464FF0010E60
:108FC0004FF0030904E00133102B00F102003CD004
:108FD0000EFA03F737EA0504F5D1D2F800A009FA32
:108FE00000F4E4430AEA040AC2F800A0D2F800B090
:108FF00006FA00FA4AEA0B0AC2F800A0D2F808A062
:1090000004EA0A0AC2F808A0D2F808B00CFA00FA7A
:109010004AEA0B0AC2F808A0D2F804A02AEA070715
:109020005760D2F804A008FA03F747EA0A07576026
:10903000D7683C40D460D76801FA00F401333C4360
:10904000102BD46000F10200C2D1BDE8F08F064BB6
:109050001D6B2C431C636BE7034B1D6C2C431C6482
:1090600066E700BF200804080038024010B5040974
:10907000013C032C17D80D4B33F8142000F00F00DF
:1090800042FA00F313F001030DD0012303FA00F0BC
:109090000138104032F080F9054A064B125D104449
:1090A00003EBC00010BD002010BD00BFF408040891
:1090B000F008040840C500202DE9F04F4A484B490C
:1090C0004B4B4C4C4FF0010A4FF002094FF0040893
:1090D0004FF0080C4FF0100E20274026802530F866
:1090E000022B12F0010F03D01960A3F804A008337B
:1090F00012F0020F03D01960A3F80490083312F0A5
:10910000040F03D01960A3F80480083312F0080F8D
:1091100003D01960A3F804C0083312F0100F03D075
:109120001960A3F804E0083312F0200F02D0196090
:109130009F80083312F0400F02D019609E800833E0
:1091400012F0800F02D019609D80083312F4807FE6
:1091500005D04FF4807B1960A3F804B0083312F4F3
:10916000007F05D04FF4007B1960A3F804B00833EA
:1091700012F4806F05D04FF4806B1960A3F804B02F
:10918000083312F4006F05D04FF4006B1960A3F898
:1091900004B0083312F4805F05D04FF4805B19608F
:1091A000A3F804B0083312F4005F05D04FF4005B5D
:1091B0001960A3F804B0083312F4804F05D04FF4BF
:1091C000804B1960A3F804B00833D20B04D04FF4DD
:1091D000004219609A80083301F58061A1427FF452
:1091E0007EAFBDE8F08F00BFF40804080000024025
:1091F00040C500200010024000286AD003682DE915
:10920000F04F03F13F4404F57E045F4EA40A0125AC
:10921000345D04F01F066409032C05FA06F559D0E5
:10922000042C00F0AC80022C59D08588B5FA85F06A
:10923000C0F11F0080B2C40803EB840400F00700F3
:10924000266A80000F27874026EA07062662276ADB
:1092500001F003068240701E3A430128C1F3810CDD
:10926000C1F300182262C1F341113DD90024224606
:1092700001274FF0030E03E0102A04F1020426D068
:1092800007FA02F0A84302F10102F5D1D3F800C0B9
:109290000EFA04F0C04300EA0C0CC3F800C0D3F887
:1092A000008006FA04FC4CEA080CC3F800C0D3F8AE
:1092B0000CC000EA0C00D860D3F80CC001FA04F02E
:1092C00040EA0C00102AD86004F10204D8D1BDE8AD
:1092D000F08F70472D4C266C35432564A5E72B4C49
:1092E000666C35436564A0E7002002464FF0010E2E
:1092F0004FF0030904E00132102A00F102003CD0D3
:109300000EFA02F737EA0504F5D1D3F800A009FAFE
:1093100000F4E4430AEA040AC3F800A0D3F800B05A
:1093200006FA00FA4AEA0B0AC3F800A0D3F808A02C
:1093300004EA0A0AC3F808A0D3F808B00CFA00FA45
:109340004AEA0B0AC3F808A0D3F804A02AEA0707E0
:109350005F60D3F804A008FA02F747EA0A075F60E3
:10936000DF683C40DC60DF6801FA00F401323C4316
:10937000102ADC6000F10200C2D1BDE8F08F034C7E
:10938000266B3543256350E7200804080038024067
:10939000002855D0026802F13F4303F57E032DE912
:1093A000F04F9B0A544DEB5C03F01F055B09012451
:1093B000032B04FA05F444D0042B00F09780022B11
:1093C00044D001F00306731E012BC1F3810CC1F3DD
:1093D00000188588C1F341113DD900242346012797
:1093E0004FF0030E03E0102B04F1020426D007FA1D
:1093F00003F0A84303F10103F5D1D2F800C00EFA3F
:1094000004F0C04300EA0C0CC2F800C0D2F800809F
:1094100006FA04FC4CEA080CC2F800C0D2F80CC0F2
:1094200000EA0C00D060D2F80CC001FA04F040EA67
:109430000C00102BD06004F10204D8D1BDE8F08FED
:1094400070472E4B1D6C2C431C64BAE72B4B5D6C94
:109450002C435C64B5E7002003464FF0010E4FF04B
:10946000030904E00133102B00F102003CD00EFA96
:1094700003F737EA0504F5D1D2F800A009FA00F4A1
:10948000E4430AEA040AC2F800A0D2F800B006FADF
:1094900000FA4AEA0B0AC2F800A0D2F808A004EACF
:1094A0000A0AC2F808A0D2F808B00CFA00FA4AEA90
:1094B0000B0AC2F808A0D2F804A02AEA07075760EE
:1094C000D2F804A008FA03F747EA0A075760D768FA
:1094D0003C40D460D76801FA00F401333C43102BC0
:1094E000D46000F10200C2D1BDE8F08F034B1D6BC8
:1094F0002C431C6365E700BF2008040800380240C5
:10950000F0B5044690F84D0083B0002840F0A480E8
:10951000674E3778002F40D004F11805A06929F074
:109520003FFE94F846201A212846FEF703FF01204B
:1095300008F004FEA06929F01FFE284694F85C108C
:10954000256D6B460622A847D0B19DF802609DF8B4
:1095500003309DF800509DF801109DF804009DF81F
:10956000052043EA06231BB2E3845BB241EA0521EE
:1095700042EA00220133A184228506D003B0F0BD67
:10958000B4F926305BB20133F8D194F924300133B9
:10959000F4D1062008F07EF9F0E7254655F8180FBB
:1095A00029F0FEFD80226B212846FEF7C3FE96209F
:1095B00008F01EFE032268212846FEF7BBFE962017
:1095C00008F016FE03226B212846FEF7B3FE0F209B
:1095D00008F0B4FD10226A212846FEF7ABFE0F20EA
:1095E00008F0ACFD3A466C212846FEF7A3FE0F209A
:1095F00008F0A4FD94F8482019212846FEF79AFEA9
:109600000F2008F09BFD18221B212846FEF792FE32
:109610000F2008F093FD10221C212846FEF78AFE39
:109620000F2008F08BFD102237212846FEF782FE1E
:109630000F2008F083FD012238212846FEF77AFE2C
:109640000F2008F07BFDA06929F096FD012008F0AD
:1096500075FD0123337061E7FFF708FD0546D8B1BA
:10966000202300218371C171FFF792FE2146114B27
:1096700041F8143F284629F071FEAB88B3FA83F312
:10968000C3F11F03012212FA03F33FF441AF0A4969
:109690000A6813430B603BE70146FFF779FE21465A
:1096A000044B41F8143F284629F058FE30E700BF2C
:1096B0009423002099870008003C014010B1036802
:1096C00082885A83704700BF10B1036882881A836A
:1096D000704700BF18B10368828809B95A83704780
:1096E0001A83704710B40A4B0A4A1C78012383403E
:1096F000234052F8200029B9B3FA83F149095DF8F3
:10970000044BE7E7191C18BF01215DF8044BE1E7A2
:1097100026C7002028C7002030B1036882881B6953
:109720001A4214BF01200020704700BF2DE9F0410C
:109730000B4E346873691C400FD0DFF82880012776
:10974000B4FA84F3C3F11F0307FA03F558F82300B2
:1097500003689847AC437561F2D1BDE8F08100BF62
:10976000003C014098C600202DE9F0410B4E3468C2
:1097700073691C400FD0DFF828800127B4FA84F306
:10978000C3F11F0307FA03F558F82300036898474D
:10979000AC437561F2D1BDE8F08100BF003C0140EF
:1097A00098C600202DE9F0410B4E346873691C40C7
:1097B0000FD0DFF828800127B4FA84F3C3F11F0328
:1097C00007FA03F558F8230003689847AC4375611E
:1097D000F2D1BDE8F08100BF003C014098C60020F6
:1097E0002DE9F0410B4E346873691C400FD0DFF84F
:1097F00028800127B4FA84F3C3F11F0307FA03F5A5
:1098000058F8230003689847AC437561F2D1BDE86E
:10981000F08100BF003C014098C600202DE9F041D6
:109820000B4E346873691C400FD0DFF82880012785
:10983000B4FA84F3C3F11F0307FA03F558F82300C1
:1098400003689847AC437561F2D1BDE8F08100BF71
:10985000003C014098C600202DE9F0410B4E3468D1
:1098600073691C400FD0DFF828800127B4FA84F315
:10987000C3F11F0307FA03F558F82300036898475C
:10988000AC437561F2D1BDE8F08100BF003C0140FE
:1098900098C60020084A094808B5536C43F4804331
:1098A00053640021402234F094F9054B4FF0FF320D
:1098B0001A60C3F8032008BD0038024098C6002093
:1098C000D8C600202DE9F041044618460D4616463C
:1098D000984631F097F82768E6722844A072294626
:1098E0007D69434632462046AC46BDE8F0416047BC
:1098F000036810B504461B689847236820469B6898
:109900009847A37B0133A37310BD00BF10B5036854
:1099100004469B689847FF2301226373227310BD9E
:1099200008B5FFF7A3FB38B12C2282710022C27167
:109930002021BDE808402BE508BD00BF30B44568D4
:1099400015B12B68AA885A83026841F0800140F261
:10995000E93301E0002B47D01089013B10F0020FE2
:109960009BB2F7D089B2918140F2E93301E0002B3C
:109970003AD01189013B11F0010F9BB2F7D09389C6
:10998000938940F2E93300E0D3B11189013B11F032
:10999000020F9BB2F8D0FF23938140F2E93300E03D
:1099A00073B11189013B11F0010F9BB2F8D094897A
:1099B000E4B215B12B68AA881A83204630BC7047E0
:1099C00015498A4207D0154B9A4221D003F580638E
:1099D0009A42EED10223124A02EB03135A89013252
:1099E00092B25A815B89E4E70B498A4207D00B4B5C
:1099F0009A420FD003F580639A42C1D102230849ED
:109A000001EB03135989013189B259815B89B7E7A9
:109A10000123E0E70123F2E7003001400038004075
:109A200010C50020F8B50501684C694B62596119F1
:109A30009A4204EB050704BF01230B730646387AEC
:109A400029F0E4FB3B7A03F01F015B090122032BA1
:109A500002FA01F26DD0042B66D0022B5CD06319A0
:109A600001361879FFF702FBF6B2074610B1122350
:109A7000C671837163195879FFF7F8FA10B113238F
:109A8000C671837163199879FFF7F0FA10B1142346
:109A9000C671837166190A21F2793846FFF7ACFB6B
:109AA0007079FFF7E3FAF2790A21FFF7A5FBB079A5
:109AB000FFF7DCFAF2790A21FFF79EFB6359454A6A
:109AC000934247D0424A934250D0434A934259D09E
:109AD000424A934262D0424A93426BD0414A9342F7
:109AE0002CD02C44227BE2B901200222198801F4F7
:109AF000415141F445710A4302431A809A8B22F482
:109B000000621204120C07219A8319821A8892B2F9
:109B100042F040021A80F8BD334B596A0A435A6238
:109B20009DE700200246E1E72F4B19690A431A61BD
:109B300095E72D4B196A0A431A6290E702F56442D1
:109B40004FF40010536A43F40013536222F046F8B6
:109B50006359C6E702F584324FF48050536A43F4E8
:109B60008053536222F03AF86359BAE702F50032A3
:109B70004FF48040136A43F48043136222F036F8B6
:109B80006359AEE702F5FE324FF40040136A43F426
:109B90000043136222F02AF86359A2E702F58232E9
:109BA0004FF40050536A43F40053536222F016F806
:109BB000635996E702F568424FF48010536A43F404
:109BC0008013536222F00AF863598AE710C5002017
:109BD0000038004000300140003C004000340140AB
:109BE000005001400054014000380240427A02B95E
:109BF000704710B504460368406804F10A019847AD
:109C00000023637210BD00BF437A5A1C0344D2B2D2
:109C100042729972037A934200D802B9704710B524
:109C200004460368406804F10A0198470023637200
:109C300010BD00BF302827D0312827D0322827D0A8
:109C4000332827D0342827D0352827D0202827D0DC
:109C5000212827D0102827D0112827D0122827D034
:109C6000132827D0142827D0152827D0162805D048
:109C7000172808BF0F2202D0002070470E22104B79
:109C800003EB4203587F70470022F8E70122F6E712
:109C90000222F4E70322F2E70422F0E70522EEE7CE
:109CA0000622ECE70722EAE70822E8E70922E6E7CE
:109CB0000A22E4E70B22E2E70C22E0E70D22DEE7CE
:109CC0003CDD030870B5448806460D46C4F30B041A
:109CD00022460021284633F07CFF3369094A93422B
:109CE00009D3094A934206D2224628461946BDE8BE
:109CF000704031F057BC23B121462846BDE8704082
:109D0000184770BDD405000885060008064B0749B2
:109D10008B4202D30023184670471A88C2F30B0205
:109D20009042F8D01433F3E788010008D405000806
:109D3000024A136823EA000010607047F8500020C0
:109D4000F8B51A4D2B789F2B2ED16B78BE2B2BD1CB
:109D500005221749A81C33F087FF28BB0722294694
:109D60004FF6FF70FEF730FC124FEC1D22884AB10F
:109D7000A618BE4218D2052A16D92146FEF724FCA1
:109D80003446F3E721460222FEF71EFC0222A11808
:109D9000FEF71AFC0634084B641B1C8041F60F5377
:109DA000C31A58425841F8BD0020F8BD00400008D1
:109DB000A00A040800800008084100202DE9F04FA7
:109DC000DFF85891504F8DB00326A7EB09071822F2
:109DD0000DEB0200002133F0FCFE4C4BCDF8189047
:109DE00007971A69002A04DA494A5A6002F1883250
:109DF0005A6001228DF82C20F322DA60454B464C44
:109E000018689A8804909B79ADF8142004A9072259
:109E100006A88DF81630FEF791FE072204A94FF62A
:109E2000FF70FEF7D1FBDFF8F8B080464FF0000A74
:109E30005C4539D30CAC002524F82C5D0222214668
:109E400006A8FEF77BFE022221464046FEF7BCFB39
:109E500040BAC043ADF80800022202A906A8FEF7E6
:109E60006DFE099878B108ABC0F104022946184488
:109E700033F0AFFE0A9818B9089906A8FEF7C0FD9E
:109E800000230A9009939DF82C300A9A23B11F49A8
:109E90000B6943F000430B61013E2DD0002A96D19F
:109EA000FFF74EFF50B32CE065888DF80DA0C5F389
:109EB0000B05AA1DADF808202288C2F30B01120B76
:109EC000ADF80A108DF80C2002A9062206A8FEF7AC
:109ED00035FE062202A94046FEF776FB6168804601
:109EE0002A4606A8FEF72AFE616840462A46FEF783
:109EF0006BFB143480469BE7002AD1D0052007F085
:109F0000C9FC0DB0BDE8F08F00800008003C0240A5
:109F10002301674578DD0308880100080040000838
:109F2000D40500080378202B024600F10100F9D087
:109F3000092BF7D02D2B2CD02B2B03BF5378B7EE4A
:109F4000000A0246B7EE000AA3F13001C8B20928A0
:109F50009FED467A10D8F2EE046A07EE901AF8EEFA
:109F6000E77A12F8013FE7EE267AA3F13001C8B292
:109F70000928B0EE677AF0D92E2B4CD003F0DF031E
:109F8000452B0BD0F7EE007A67EE276A20EE260A03
:109F900070475378BFEE000A0246D5E710B45178F7
:109FA0002D2959D02B290ABF9178501C901C0024D0
:109FB000A1F13003092B53D8002303EB830301EBFA
:109FC000430310F8011FA1F13002092AA3F1300365
:109FD000F3D9B3F59A7F28BF4FF49A73072B42D970
:109FE000DFED236A1A46F7EE007A083A072A67EE91
:109FF000A67AFAD803F007032BB1F2EE046A013B0C
:10A0000067EEA67AFBD124B3C7EE276A5DF8044B4E
:10A0100020EE260A70475378A3F13001C8B2092810
:10A0200002F10102AAD8F2EE046AF0EE665A07EED7
:10A03000901AF8EEE77A12F8013F87EEA66AA3F1CC
:10A040003001C8B2092866EEA56A37EE067AEED965
:10A0500094E767EE276AD9E7901C91780124A7E777
:10A06000F7EE007ACFE7F7EE007AC5E700000000D0
:10A0700020BCBE4CB5EEC00ADFED317AF1EE10FA2D
:10A08000CCBF30EE270A30EE670ADFED2E7A20EEE5
:10A09000270A30B5FDEEC07A87B017EE904A054624
:10A0A00084EAE470002303A9A0EBE4700193009319
:10A0B000029327F0ABFA002CACBF20232D2303A87A
:10A0C0008DF8003030F09EFC012803A924D002282E
:10A0D0002DD0032805BF3023684668468DF801302F
:10A0E00033F09DFD684630F08DFC0338C4B2224643
:10A0F0006946284633F0F1FD00232B55284630F001
:10A1000081FC2E22431C2A540DEB0401E81833F085
:10A11000A3FD284607B030BD302368468DF80130D6
:10A120008DF802308DF8033033F079FDDAE7302313
:10A1300068468DF801308DF8023033F070FDD1E7BC
:10A140006F12033A00007A442DE9F04106461546A5
:10A150000846B6FBF2F43CB905FB1464124B1B5DD8
:10A1600000F8013BBDE8F081B4FBF2F767B90E4B94
:10A1700005FB174705FB1464DA5D00F8012B1B5D36
:10A1800000F8013BBDE8F081B7FBF2F8B8F1000F31
:10A1900002D04046FFF7D8FF05FB1878024B13F8B2
:10A1A000082000F8012BE3E7A80A040830B402688D
:10A1B0001146531C036011F8024B0160D31C517807
:10A1C00003609378151D05601B0443EA0123D078D2
:10A1D000234343EA006030BC704700BF0368591C4A
:10A1E0001A46016012F8021B0260587841EA00200A
:10A1F000704700BF38B504460068154631F0D2F903
:10A2000022682A44226038BD036810B40A0E5C1C20
:10A2100004601A7003680A0C5C1C04601A700368FE
:10A220000A0A5C1C04601A7003685A1C02601970E8
:10A230005DF8044B704700BF036810B40A0A5C1C49
:10A2400004601A7003685A1C026019705DF8044BB0
:10A25000704700BF03685A1C026010B4197003688D
:10A260000A0A5C1C04601A7003680A0C5C1C046017
:10A270001A700368090E5A1C026019705DF8044BCD
:10A28000704700BF03685A1C026019700368090A0E
:10A290005A1C0260197070472DE9F047002488B0FD
:10A2A00080460F461E46A14605AD531C0393117808
:10A2B00039B3252933D1931CCDF8109003935078EE
:10A2C00030284ED04FF0000AA0F13003DBB2092B4A
:10A2D00042D96C2819D0642800F0938024D825280E
:10A2E0001CD063D9582876D063281BD131784046DA
:10A2F000B847039A531C039311780436013400299C
:10A30000D7D1204608B0BDE8F087039B5A1C0392C2
:10A310001B78642B7CD02AD8252B54D1252140468C
:10A320000134B847039AC0E7732833D044D975285D
:10A330004FD106F1040E30682B4600220A217646E2
:10A34000FEF7C6F8049A0095534639464046FEF794
:10A35000FDF8039A0444A8E704AA03A924F04CF8E2
:10A36000B7E7D31C039390784FF0010AACE7732B47
:10A3700010D05BD9752B3AD0782B96D1A3F1580227
:10A38000B2FA82F2306852092B4610210436FEF7E9
:10A390009FF8D7E73368049A009339460023404674
:10A3A000FEF7D4F804360444039A7EE70028B9D1B6
:10A3B000204608B0BDE8F0876E28B3D1039A336811
:10A3C00004361C6071E72AD9582BD7D0632B8DD067
:10A3D0006BE77828A6D1A0F15802B2FA82F2306871
:10A3E00052092B461021FEF773F80436AAE706F14E
:10A3F000040E30682B4600220A217646FEF768F8E4
:10A40000A0E7331D306829461E46FEF733F899E76A
:10A41000331D306829461E46FEF72CF892E7002BC4
:10A420007FF443AF204608B0BDE8F0876E2BC6D05E
:10A430003BE700BF0EB400B584B005AB019053F804
:10A44000042B0649039301A8FFF726FF019B002276
:10A450001A7004B05DF804EB03B070474185000842
:10A460000FB430B583B006AB0A490B4853F8042B40
:10A47000096800680193FFF70FFF084C0546206844
:10A48000FEF700FD0028FAD0284603B0BDE83040B2
:10A4900004B07047803F0020843F002058D0002047
:10A4A000DFED2B7AB4EEE70AF1EE10FA4ADDDFEDCC
:10A4B000296A9FED297A01E0B0EE670AB4EEC70A77
:10A4C000F1EE10FA70EE667AF6DC9FED247AF4EE87
:10A4D000C77AF1EE10FA38D5DFED1E6A9FED207ACB
:10A4E00001E0F0EE407AF4EEC77AF1EE10FA37EEC2
:10A4F000A60AF6D4DFED1B7AB4EEE70AF1EE10FA05
:10A5000014DDDFED137A37EEC00A60EE006A9FEDCE
:10A51000166A9FED167ADFED167AA6EE867A20EEA1
:10A52000266AE6EE877AA6EE270A7047DFED117AF3
:10A53000B4EEE70AF1EE10FA44BFDFED087A37EE29
:10A54000C00AE2E7F0EE407ABFE7B0EE670AD1E773
:10A55000DB0F4940DB0FC940E4CB1641DB0F49C09C
:10A56000E4CB16C1DB0FC93F92E741B99730083CF5
:10A5700015A82ABEDB0FC9BF41404A0011F0800F69
:10A5800082F0D503D2B2DBB208BF1346590013F0F4
:10A59000800F81F0D502C9B2D2B208BF0A4651007D
:10A5A00012F0800F81F0D503C9B2DBB208BF0B46B1
:10A5B000590013F0800F81F0D502C9B2D2B208BFA2
:10A5C0000A46510012F0800F81F0D503C9B2DBB208
:10A5D00008BF0B46590013F0800F81F0D502C9B2B5
:10A5E000D2B208BF0A46510012F0800F81F0D503A5
:10A5F000C9B2DBB208BF0B465A0082F0D50013F097
:10A60000800FD2B2C0B208BF1046704709B909E046
:10A61000194690FBF1F301FB13030846002BF7D119
:10A62000084670470146FBE7F0EEC07AB0EEE07AEC
:10A63000B4EEE77AF1EE10FAB4BFB0EE676AB0EEAE
:10A64000476AB5EE406AF1EE10FA46D0B4EEE77A0A
:10A65000F1EE10FA8CBFF0EE675AF0EE475AC5EEF5
:10A66000866A9FED1F3A9FED1F6A9FED1F4A9FED7F
:10A670001F5ADFED1F3ADFED1F4ADFED1F5AA6EE2E
:10A68000C36AE6EEA34AA6EE864AB7EE006AA6EED5
:10A69000845AA6EEA46AE6EE855AC5EE866AB4EE42
:10A6A000E77AF1EE10FA48BFDFED147AF5EEC00A52
:10A6B00048BF77EEE66AF1EE10FA48BFDFED107A98
:10A6C000B5EEC00A48BF77EEE66AF1EE10FA48BF71
:10A6D000F1EE666AB0EE660A7047DFED076ADEE704
:10A6E00039094E3DE3B59E3E88FA163E45FE7F3F52
:10A6F00099FB243F69A2163EA7DFA834DB0FC93FB0
:10A70000DB0F4940DFED317A30EE277AFDEEC76A84
:10A7100016EE903A2033402B02D99FED2D0A704758
:10A72000B4EEE70AF1EE10FA4DDD9FED2A6ADFED97
:10A730002A6A01E0B0EE677AB4EEE67AF1EE10FA3A
:10A7400077EE467AF6DC9FED257AF4EEC77AF1EEE5
:10A7500010FA35D5DFED1F6A9FED217A01E0F0EEAA
:10A76000407AF4EEC77AF1EE10FA37EEA60AF6D484
:10A77000DFED167AB4EEE70AF1EE10FA1BDCDFED3E
:10A78000197AB4EEE70AF1EE10FA44BFDFED137A5E
:10A7900037EEC00A60EE006A9FED136A9FED137AF0
:10A7A000DFED137AA6EE867A20EE266AE6EE877A49
:10A7B000A6EE270A7047DFED0F7A37EEC00AE9E709
:10A7C000B0EE670AD4E7F0EE477ABCE7DB0FC93F8B
:10A7D00000000000DB0FC940E4CB1641DB0F49C08D
:10A7E000E4CB16C1DB0FC9BF92E741B99730083CF3
:10A7F00015A82ABEDB0F4940FDEEC07A17EE903A4D
:10A800002033402B51D8DFED2D7AB4EEE70AF1EE7C
:10A8100010FA50DDDFED2A6A9FED2A7A01E0B0EEF2
:10A82000670AB4EEC70AF1EE10FA70EE667AF6DC4B
:10A830009FED257AF4EEC77AF1EE10FA38D5DFED08
:10A84000206A9FED227A01E0F0EE407AF4EEC77ABA
:10A85000F1EE10FA37EEA60AF6D4DFED1D7AB4EE6B
:10A86000E70AF1EE10FA1BDCDFED1A7AB4EEE70A24
:10A87000F1EE10FA44BFDFED147A37EEC00A60EE55
:10A88000006A9FED156A9FED157ADFED157AA6EE49
:10A89000867A20EE266AE6EE877AA6EE270A7047C9
:10A8A000DFED067A37EEC00AE9E79FED0E0A704742
:10A8B000B0EE670AD1E7F0EE407AB9E7DB0F494026
:10A8C000DB0FC940E4CB1641DB0F49C0E4CB16C116
:10A8D000DB0FC93FDB0FC9BF92E741B99730083C96
:10A8E00015A82ABE0000000010B507EE901A2DED45
:10A8F000028BB8EE678ADFED227A28EE008A0446E2
:10A9000028EE278AB0EE480A31F0A2F8F0EE408A2D
:10A91000B0EE480A30F0FEFFF7EE007A9FED197AAC
:10A92000F0EE675AE8EE875A0023A361B0EE676A3B
:10A93000C7EEA56A63612362E361A3626362A8EE66
:10A94000C76ABDEC028B77EEC07AB6EE007AF8EEFD
:10A95000005A27EE877A20EE250A27EE267A26EE81
:10A96000266A67EEA67A20EE260A84ED046AC4ED14
:10A97000017A84ED007A84ED027A84ED030A10BD39
:10A9800027D4D236F304353F10B44C09012250F8D5
:10A99000243001F01F0102FA01F10B4340F824308A
:10A9A0005DF8044B704700BF4B0901F01F0150F8E0
:10A9B0002320012303FA01F1114214BF184600209D
:10A9C000704700BF2DE9F84FDFF8B480DFF8B4908E
:10A9D000DFF8B4A0274E0123102088F8003028F0BB
:10A9E000F3FBD9F80000FEF769FE052028F09CFB78
:10A9F000002028F099FB062028F096FB002028F084
:10AA000093FB9AF80040042044F0010428F08CFBEA
:10AA1000204628F089FB33888BB1174D174F00244F
:10AA200015F804B0072028F07FFB584628F07CFB7F
:10AA30002A5D33883A550134A4B2A342F0D80720E6
:10AA400028F072FBFF2028F06FFB9AF800400420EA
:10AA500028F06AFB204628F067FBD9F80000FEF7D3
:10AA600033FE042028F0B0FB002388F80030BDE856
:10AA7000F88F00BF80160020586500201CCA0020F7
:10AA80007D6A0020247C00200CCA00202DE9F041C2
:10AA90004A4E102028F098FB3068FEF70FFE484B16
:10AAA0001B78012B7BD062D3022B0AD1DFF83081D7
:10AAB000082388F800300D254FF4C373414F3B80C5
:10AAC00010E0DFF81C813F4F98F8003003F040039E
:10AAD000002B14BF4FF4F0734FF4C3733B8014BFCB
:10AAE00010250D25002404F11000C0B228F01CFB35
:10AAF0000134012028F018FBA3B2AB42F3D398F83D
:10AB00000040314D002028F00FFB204628F00CFBC0
:10AB10002E4B1C78022028F007FB204628F004FB6F
:10AB20002B4B1C78032028F0FFFA204628F0FCFA73
:10AB3000284B1C780420044328F0F6FA204628F01D
:10AB4000F3FA3068FEF7C0FD042028F03DFB3A8898
:10AB50002148002133F03DF82B7833B11F4B1B788F
:10AB600033B300232B70BDE8F081BDE8F081A02055
:10AB700028F0DAFA002028F0D7FA00F00603022BBA
:10AB8000DFF85C8007D000F00500012803D14823DE
:10AB900088F8003008E0082388F800308BE7DFF8F9
:10ABA0004080482388F8003010254FF4F07385E783
:10ABB000FFF708FF00232B70BDE8F081247C002004
:10ABC000287C002080160020000000202F7C002020
:10ABD000307C00200CCA00201CCA00207D6A0020A6
:10ABE000881600200C4B984213D0A3F5806398423E
:10ABF0000FD003F5804398420BD003F58063984251
:10AC000007D003F58063984203D0044B18684008CE
:10AC10007047024B186870470004014080BB002059
:10AC2000F0B5774B774A87B01968914200AF00F0D2
:10AC3000DB800023744A3B607B60136843F48033FD
:10AC4000136003E03B68B3F5A04F09D0136803F429
:10AC500000337B603B6801333B607B68002BF1D0A5
:10AC6000694B1B6813F4003318BF01237B607B68BA
:10AC7000012B7BD0654D644B654AEA606549586F8E
:10AC8000654A0860AA605E6B644C654A654826F0B8
:10AC900080065E635E6F46F080765E67196B0C43DC
:10ACA0001C63596B5963996B9963196C41F05B5143
:10ACB00041F47B1141F41F6141F00F011964596C9B
:10ACC00007F118040A4348F2FF715A6444F8101D52
:10ACD000002621460123FB733E737E73BE7320F072
:10ACE00031FF21464FF6FF734F48BB6020F02AFF2B
:10ACF0004FF6FF7321464D48BB6020F023FF2146ED
:10AD00004B4820F01FFF21464A4820F01BFF2146F8
:10AD1000494820F017FF2146484820F013FF2146FC
:10AD2000474820F00FFF2146464820F00BFF204601
:10AD300021F012F8444B454C1B68BA684448454919
:10AD4000A4FB03439B09A0FB0202013B920CB3F15D
:10AD5000807F0A6007D2404AF0200721536085F8BF
:10AD60002300966011601C37BD46F0BD264B3B4C5E
:10AD70001A6C3B4942F080521A6420688A684D6818
:10AD8000C96840F44040206098689860986812064E
:10AD900040F40040986042EA8512986842F48002CC
:10ADA000490842F00802013942EA014240F4A05049
:10ADB00098605A601A6842F080721A601A689201AC
:10ADC000FCD52849104A40F205700860996821F0C6
:10ADD00003019960996841F002019960936803F05A
:10ADE0000C03082BFAD145E700221A6062B61E4B0D
:10ADF0001B6883F308881D4B1B689847FEE700BF5C
:10AE0000FCFF0120EFBEADDE0038024000ED00E0A7
:10AE10000005FA0584C0002000000008FF916700CB
:10AE2000335F0700000002400004024000080240B7
:10AE3000000C0240001002400014024000180240C2
:10AE4000001C02400020024080BB0020D34D621055
:10AE500083DE1B4360C7002010E000E0007000406C
:10AE600000000020003C02400000FF1F0400FF1F04
:10AE700008B5054B1B6803B19847044B044A1A6098
:10AE800072B6FDF793FC00BFAC840020FCFF0120EC
:10AE9000EFBEADDE08B5034B1B6803B1984772B631
:10AEA000FDF784FCAC840020084B10B507281B6814
:10AEB000C8BF143818440C46007DFEF7D7F820B1FF
:10AEC0002146BDE81040FEF705BC10BD04C70020B8
:10AED00030B50446806D61718389A26823F4005304
:10AEE0001B041B0C838185B0A379009213F004022C
:10AEF00030D04FF4805213F00203ADF804205CD13F
:10AF0000ADF806304FF480630022ADF8083011F040
:10AF10000103ADF80C2028D1ADF80A3008238D07C5
:10AF2000694648BFADF80A3020F060FFA279A36DF2
:10AF3000D10724D412F0080F9A8A1BD122F00802FC
:10AF40001204120C9A829A8992B242F400529A81A7
:10AF500005B030BD13F00203ADF804202AD04FF441
:10AF600000551346ADF80650CEE70423ADF80A307D
:10AF70000C23D4E792B242F008029A82E3E7104928
:10AF80008B4215D0A1F548418B420FD001F580616D
:10AF90008B4209D00B498B42CCD105200121FFF710
:10AFA00083FFA279A36DC5E70320F7E70220F5E749
:10AFB0000020F3E7ADF80630A6E74FF400539FE713
:10AFC000001001400014014010B50446806DA160DE
:10AFD000838923F400531B041B0C8381A37984B061
:10AFE00013F00402009135D04FF4805213F00203A5
:10AFF000ADF804205CD1ADF806304FF4806362797F
:10B00000ADF80830D1074FF00003ADF80A30ADF8C5
:10B010000C3045BF0423ADF80A3008230C236946E1
:10B02000920748BFADF80A3020F0E0FEA279A36D88
:10B03000D1071FD412F0080F9A8A16D122F0080205
:10B040001204120C9A829A8992B242F400529A81A6
:10B0500004B010BD13F00203ADF8042025D04FF466
:10B0600000511346ADF80610C9E792B242F008024B
:10B070009A82E8E710498B4215D0A1F548418B42EE
:10B080000FD001F580618B4209D00C498B42D1D1A0
:10B0900005200121FFF708FFA279A36DCAE703206D
:10B0A000F7E70220F5E70020F3E7ADF80630A6E762
:10B0B0004FF400539FE700BF00100140001401400F
:10B0C00038B50D4B07281B68CCBFA0F1140404460B
:10B0D00023440546187DFDF7C9FF58B101342722E6
:10B0E000C47182710121FEF753F928460021BDE8A1
:10B0F0003840D9E638BD00BF04C70020064A002307
:10B100005168814202F11C0204D00133102BF7D1A7
:10B1100000207047D8B27047E000002070B50F4C97
:10B120000F4DC0EBC00004EB8004286B2669304350
:10B13000286382B09209667BA1600025012101A8E5
:10B1400063618DF804608DF805208DF806508DF848
:10B15000071028F0E1F802B070BD00BFE000002049
:10B1600000380240074BC0EBC00030B403EB800056
:10B17000054C0569236B2B4323630176427630BC73
:10B18000704700BFE0000020003802402DE9F04F7A
:10B19000534C54F8204083B0002C00F09C80E56DA7
:10B1A000002D00F09A8017464E4A9846064604F154
:10B1B00062032869226004F262226361A2614FF493
:10B1C00000736A68A160E3602361A265A24668B16A
:10B1D000FFF794FF721CD2B20C21FFF7C3FFA36DDF
:10B1E000A9682A6922630433A1636365E868A0B192
:10B1F000FFF784FF721C8146D2B20B21FFF7B2FF2A
:10B200002346EA7F38494846FFF788FFA36DA968BF
:10B21000EA6862630433E163236594F86100FDF733
:10B2200025FF814694F86000FDF720FF8346287FC4
:10B2300000284DD118F0080F36D1BA070DD5B9F155
:10B24000000F0AD00B22731C89F8062089F80730FA
:10B2500048466A7F2221FDF7CFFFFB0715D4A36B79
:10B260007BB995F82020A97F8DF8063001A89309B5
:10B2700001228DF805308DF804108DF8072028F094
:10B280004BF8504603B0BDE8F08FBBF1000FE6D09D
:10B2900001360C238BF807608BF8063058466A7F1E
:10B2A0002221FDF7A9FFDAE70136F6B2B9F1000F66
:10B2B00004D00B2389F8076089F8063018F0100FC6
:10B2C000484614BF022112216A7FFDF795FFC6E7A9
:10B2D00027F09CFFAEE7A246D3E7AA46D1E700BF1E
:10B2E0008C3F002080DD0308D18700080348D0F898
:10B2F000AC3113B100F5D27018477047E000002060
:10B300000348D0F8903113B100F5C4701847704766
:10B31000E00000200348D0F8743113B100F5B67096
:10B3200018477047E00000200348D0F8583113B1A7
:10B3300000F5A87018477047E00000200348D0F8D7
:10B340003C3113B100F59A7018477047E0000020B7
:10B350000348D0F8203113B100F58C7018477047BE
:10B36000E00000200348D0F804310BB1FC3018474E
:10B37000704700BFE00000200348D0F8E8300BB170
:10B38000E0301847704700BFE00000200348D0F8C5
:10B39000CC300BB1C4301847704700BFE00000202C
:10B3A0000348D0F8B0300BB1A8301847704700BF41
:10B3B000E00000200348D0F894300BB18C301847DF
:10B3C000704700BFE00000200248836F0BB170306F
:10B3D00018477047E00000200248C36D0BB154309D
:10B3E00018477047E00000200248036C0BB138306A
:10B3F00018477047E00000200248436A0BB11C3038
:10B4000018477047E00000200248836803B11847DE
:10B41000704700BFE00000201549164B16484A68E7
:10B4200010B4CC681549B2FBF4F203FB02F30360DD
:10B43000D1F88820124B134C42F47002C1F88820D6
:10B440001A68002042F001021A6098601A6822F01F
:10B45000847222F480321A605C601A684FF00064D3
:10B4600022F480221A60D8608C605DF8044B70472B
:10B470000000002040420F0080BB002000ED00E0F3
:10B480000038024010300024044B4FF4F0700221C9
:10B490000A225860D9609A60FFF7BEBF0000002002
:10B4A0002DE9F04F05462DED048BB0F90800088119
:10B4B0005FFA80F897B040460C46914605F034F8A4
:10B4C00040B101231A461846628117B0BDEC048BC7
:10B4D000BDE8F08FA8F10A03E72B00F2EA80DFE86D
:10B4E00013F06606E800E800E800E800E800E8007D
:10B4F000E800E800E800E800E800E800E800E8000C
:10B50000E800E800E800E800E800E800E800E800FB
:10B51000E8007806E800E800E800A906E800E8008E
:10B52000E8006D05E8009705E800D805E800F1059A
:10B53000E800FD05E8000206E8002806E800E8004B
:10B54000E8008D019401E8009C01E800E800A501F5
:10B55000E800E800E800E800E8008001E800E80012
:10B56000E800E800AD01E800C801E800E9011102C7
:10B57000E800E800E800E800E800E800E80043022E
:10B58000E8008602E800B002E8001303E800DE02EB
:10B59000E800E800E800E800EE025C038E03960392
:10B5A000BE03CF0325043B045404E800600499045F
:10B5B000E800E800E800E800B604E800E800C2049B
:10B5C000E800E800E800E404F5040E051E05E800C4
:10B5D000E800E8005C052507E800E800E800E8006E
:10B5E000E800E800E800E800E800E800E800E8001B
:10B5F000E800E800E800E800E800EE02E800E80003
:10B60000E800E800E800E800E800E800E800E800FA
:10B61000E800E800E800BA06E800E800E800E80012
:10B62000E800E800E800E800E800E800E800E800DA
:10B63000E800E800E800E800E800E800E800E800CA
:10B64000E800E800E800E800E800E800E800E800BA
:10B65000E800E800E800E800E800E800E800E800AA
:10B66000E800E800E800E800E800E800E800E8009A
:10B67000E800E800E800E800E800E800E800E8008A
:10B68000E800E800E800E800E800E800E800E8007A
:10B69000E800E800E800E800E800E800E800E8006A
:10B6A000E800E800E800E800E800E800E800F30649
:10B6B0003B06B8F1740F58D0B8F1770F0DD12B6855
:10B6C0006A689A421EBF5A1C2A601978994A08BFB4
:10B6D0000021204605F0B4FAF3E6B8F1F50F01F0C9
:10B6E0004687B8F1760F4ED095E88400A8F1210383
:10B6F000BF1A362B00F23E87DFE813F0F0063C0756
:10B700003C073C073C073C073C073C0711073C074C
:10B710003C073C073C073C073C073C073C073C0711
:10B720003C073C073C073C073C073C07B2063C078C
:10B730003C073C073C073C073C073C073C073C07F1
:10B740003C073C073C073C073C073C073C073C07E1
:10B750003C073C073C073C073C073C073C073C07D1
:10B76000BD063C0790063C072C062B686A689A4287
:10B770001EBF5A1C2A6019786F4A08BF0021204654
:10B7800005F05EFA9DE62B685A1C2A601B78002B98
:10B7900001F05687102B07BF684A92E82200002567
:10B7A00029462268501C206013702046FEF752FD87
:10B7B00029462046FEF74EFD614B2046D968FEF72C
:10B7C00049FD00212046FEF75DFD00212046FEF7E1
:10B7D00059FD216800204A1C012322601A46087086
:10B7E00071E6236800255A1C2260294620461D70F8
:10B7F000FEF730FD29462046FEF72CFD00212046AD
:10B80000FEF728FD01231A465DE6216801200A188B
:10B81000226003460246087055E62268494B501CD8
:10B8200099782060117021685878D4E70822464939
:10B830002046FEF7DFFC01231A4644E62368434D09
:10B84000591C2A7821601A7023686A78591C216073
:10B850001A7069882046FEF715FD23682A79591C5D
:10B8600021601A70E9882046FEF70CFD2168287ACD
:10B87000B1E7374E3378002B3FF423AE354D002728
:10B88000A846236815F81720591C21601A7098F8EB
:10B89000011001EB810101EB810101F2EE2189B27E
:10B8A0002046FEF7EFFC337801379F4208F102088B
:10B8B000E7DB06E62368284A284D591C012621604B
:10B8C0001E701068FDF728FF002841F00287244B06
:10B8D0002268511C21601070226841F2B410511C82
:10B8E000185C216041F27811107059582046890A7D
:10B8F000FEF7B0FCE96B20464908FEF7ABFC0123DC
:10B900001A46E0E52168174A0123481C20600B70A5
:10B9100021689078CD182560087021681078CD18BE
:10B920002560087021685078CA1822601A4608708D
:10B93000C9E500BF750101083D040108982C0020ED
:10B9400098230020B441002058C00020EC4E002075
:10B95000F02800203C6100207061002004B8002025
:10B960007CA3002018C800202DF066F9FF280646A9
:10B9700001F0B88616A9002501F84A5D0DF10D0009
:10B980008DF80D502DF038F916A800F8495D2DF00E
:10B9900027F916A800F8485D2DF016F916A820F82A
:10B9A000405D2DF005F923685A1C22601E70236843
:10B9B0009DF80D20591C21601A7023689DF80E20F7
:10B9C000591C21601A7023689DF80F20591C2160B2
:10B9D0001A7023689DF81020591C21601A70BDF858
:10B9E00018102046FEF74EFC01231A466BE5B74EB1
:10B9F000F378002B01F0178623680822591C216078
:10BA00001A7023680122991821601A702368B04DBA
:10BA1000591C2A7921601A702368AA78591C216060
:10BA20001A7029882046FEF72DFC698A2046FEF709
:10BA300029FC2368F279591C21601A702168E87882
:10BA4000C9E6A24D23686A79A24E591C21601A707A
:10BA500033682046198CFEF715FC33682046598C54
:10BA6000FEF710FC69892046FEF70CFCA9892046E8
:10BA7000FEF708FC33682046998CFEF703FC336818
:10BA80002046D98CFEF7FEFBE9892046FEF7FAFB3B
:10BA9000298A2046FEF7F6FB01231A4613E52368A0
:10BAA0008D4A8E49D0788E4A5D1C256018702368B7
:10BAB0000978581C206019702168D0788BE60DF148
:10BAC000180900250695DFF858A2864B04950595C0
:10BAD000C9F8045001214FF6FF7B05E001350B2D1D
:10BAE00001F0B0841AF9011F4E1CF7D04BFA05F291
:10BAF000D007F3D51A882A41D207EFD548460193DB
:10BB0000FEF742FF019BE9E700212046FEF7BAFB62
:10BB100000212046FEF7B6FB00212046FEF7B2FBCF
:10BB200022686C4D0023511C216013702268296823
:10BB3000501C91F82F102060117022682968501C49
:10BB400091F83A102060117022682968501C91F811
:10BB50003B10206011702268511C21601370226814
:10BB6000511C216013702268511C216013702B68D6
:10BB70002046D98FFEF786FB2B682046998FFEF76B
:10BB800081FB23682A68591C92F8312021601A70C1
:10BB90002B68216893F832001DE6534E338AB3F5C3
:10BBA000007F06F1340594BF01270427403655F87D
:10BBB000041B91FBF7F1204689B2FEF763FBB54207
:10BBC000F5D14A4D4A4F05F10C06B5EC010AD7ED07
:10BBD000087A80EE270A2FF0EFFE81B22046FEF7AA
:10BBE00051FBB542F1D1434D05F10C0655F8041B4C
:10BBF000204689B2FEF746FBB542F7D161E4102238
:10BC00003D492046FEF7F6FA01231A465BE43B4D18
:10BC10003B4EDFF81081DFF81091DFED3A8ADFED5F
:10BC20003A9A9FED3A9A05F1200708E0204604353C
:10BC3000FEF728FBBD4206F118063FF442AC717CCA
:10BC40000029F3D095ED008AB0EE480A2FF0B4FE3B
:10BC500098F80030002B41F0F88481B2E6E72C4ED2
:10BC60003378002B3FF42DAC2A4F002537F8021F04
:10BC70002046FEF707FB337801359D42F6DB20E4D2
:10BC8000254B22681B78254D511C03F002032160CF
:10BC9000137023682A78591C21601A70696820463D
:10BCA000FEF7D8FAA9682046FEF7D4FAA9892046FB
:10BCB000FEF7E8FA698A2046FEF7E4FAA98A2046E8
:10BCC000FEF7E0FA01231A46FFF7FDBB647C002073
:10BCD00084BB00204027002090410020A04100208C
:10BCE000A84100203C27002010250020A08400202F
:10BCF000787C0020484F00204C4400205C44002009
:10BD00003C890020000040420040744400E082442E
:10BD1000F0280020FA2800206A2500206C25002049
:10BD2000D8DD0308ACBB002088C00020A54B20460E
:10BD30001988FEF7A7FAA44B20461988FEF7A2FA45
:10BD4000A24B20681978421C01F0010101232260F6
:10BD50001A460170FFF7B7BB9D4D20462988FEF7B4
:10BD600091FA69882046FEF78DFAB5F904309949B1
:10BD7000DA1781FB0313C2EBA30399B22046FEF747
:10BD800081FA01231A46FFF79EBB00212046FEF7E9
:10BD900061FA00212046FEF775FA01231A46FFF7E3
:10BDA00092BB8D4D23682A68591C127821601A7045
:10BDB0002B6822689978531C2360002311702A682D
:10BDC00021681A4401335279481C032B20600A7001
:10BDD000F5D123682A68591C127A21601A702368E9
:10BDE0002A68591CD27821601A7023682A68591C65
:10BDF000127921601A702B6820465989FEF742FAA1
:10BE000023682A68591C527A21601A702B682168AD
:10BE10005878E0E4714E00232268306803EB430158
:10BE2000551C405C25601070326820680A44451C2F
:10BE3000527825600270326820680A440133927893
:10BE4000411C0A2B21600270E6D1FFF73ABB64491E
:10BE500052232268501C2060137011F8013F002B00
:10BE6000F7D1FFF72EBB5F4D05F16006A98820468C
:10BE7000FEF708FAE9882046FEF704FA29892046E9
:10BE8000FEF700FA2368AA7A591C21601A70236809
:10BE9000EA7A591C21601A7055F80C1B2046FEF7EF
:10BEA000D9F9AE42E2D1FFF70CBB4F4D20462988AD
:10BEB000FEF7E8F969882046FEF7E4F9A9882046EC
:10BEC000FEF7E0F901231A46FFF7FDBA2268474B57
:10BED00045491878551C2560107022685878551C03
:10BEE0002560107022689B78501C20601370C988F0
:10BEF0002046FEF7C7F901231A46FFF7E4BA236884
:10BF00003B4A3C4910783C4A5D1C25601870236808
:10BF10008978581C20601970216890785BE4DFF8FC
:10BF2000ECE00027FEB2714600232268501C20601E
:10BF300016702268501C20601370226811F8010FDF
:10BF40000133551C062B25601070EED10137062FEA
:10BF50000EF1060EE6D1294900232268501C20600C
:10BF600017702268501C20601370226811F8010FAE
:10BF70000133551C0B2B25601070EED12368204A2D
:10BF8000581C07212060197023680021581C20606C
:10BF90001970216892F8F0001DE41A4D2046A98A14
:10BFA000FEF770F9E98A2046FEF76CF9298B2046E6
:10BFB000FEF768F901231A46FFF785BA124B21688C
:10BFC000187808E4EC250020EE250020806700208A
:10BFD000542500206766666644270020402700201D
:10BFE000A8DD030860C20020C44100208841002071
:10BFF000647C002090410020A8410020B362002012
:10C00000D061002084BB0020202900208F62002006
:10C01000B44D23682A7A591C21601A70A98B2046D6
:10C02000FEF730F9298B2046FEF72CF9698B204664
:10C03000FEF728F92368EA7C591C21601A70E98C04
:10C040002046FEF71FF9298D2046FEF71BF92368CD
:10C05000AA7F591C21601A70236895F82020591C6A
:10C0600021601A70A98C2046FEF70CF92368EA7A41
:10C07000591C21601A70E9682046FEF7EBF8236826
:10C080002A7C591C21601A70216895F82100FFF75D
:10C09000A2BB954D05F14006B5F880102046FEF78D
:10C0A000F1F8236895F88220591C21601A702368E2
:10C0B00095F883200435591CAE4221601A70EBD1EB
:10C0C000FFF7FFB9894D05F1800655F8041F20469A
:10C0D000FEF7C0F8B542F8D1FFF7F3B9814B2168FC
:10C0E000587DFFF778BB824B03F15A0522685979D6
:10C0F000501C2060117022681978501C206011704B
:10C1000022685978501C2060117022689978501C60
:10C11000206011702268D978501C2060117022684C
:10C1200019790633501C9D4220601170DED1FFF753
:10C13000C8B9704D704E05F1280795F9021000231B
:10C14000F2568A4201F060810C333C2BF8D108355D
:10C15000AF42F2D1FFF7B5B9684B03F17005226821
:10C160001978501C2060117022685978501C20608A
:10C17000117022689978501C206011702268D9785B
:10C18000501C2060117022681979501C20601170B9
:10C1900022685979501C2060117022689979073300
:10C1A000501CAB4220601170D9D1FFF78AB95448B6
:10C1B0002EF028FC00287FF784A9514B1D18226817
:10C1C00013F8011B501CAB4220601170F7D1FFF730
:10C1D00078B94C4D4C4F05F15006002128784B4A58
:10C1E0000B4607E00133242B02F10C0201F0098118
:10C1F00012F80C1C8842F5D103EB4303226807EBCD
:10C200008303511C93F844302160137023686A78CB
:10C21000591C21601A702368AA78591C21601A7071
:10C220002368EA780435591CB54221601A70D4D1CC
:10C23000FFF747B9364D20462988FEF723F8A9882D
:10C240002046FEF71FF829892046FEF71BF8012338
:10C250001A46FFF738B92368DFF8CCC0591C9CF8A0
:10C26000002021601A709CF80030002B3FF429A9AF
:10C27000284E294D29482A490022236816F8017FB3
:10C2800003F1010EC4F800E01F70236815F8017F68
:10C2900003F1010EC4F800E01F70236810F8017F5D
:10C2A00003F1010EC4F800E01F70236811F8017F4C
:10C2B00003F1010EC4F800E01F709CF80030013259
:10C2C0009A42DADBFFF7FDB8164D2046A989FDF743
:10C2D000D9FF69892046FDF7D5FF01231A46FFF7EC
:10C2E000F2B800BF58C00020D0610020CC6100200F
:10C2F0001C480020387C002018C0002054C30020B7
:10C3000005630020D4460020A8DD0308F0DD030803
:10C31000B03F0020A7680020B7680020D768002041
:10C32000C768002090410020A56800202268874B44
:10C33000501C19782060117022685978501C2060B8
:10C34000117022689978501C206011702168D8788B
:10C35000FFF741BA531C2B6012F8377B0DF1170120
:10C3600001332B6013F8010C01F8010F9A42F7D149
:10C37000DFF8F89199F80050002DFDD1DFF8F0A119
:10C380000126102089F8006026F01EFFDAF8000070
:10C39000FDF794F96E4B28461E7026F0C5FE284620
:10C3A00026F0C2FE092026F0BFFE384626F0BCFE6D
:10C3B00006AF3D460DF14E08EE1BF6B20A2026F000
:10C3C000B3FE304626F0B0FE15F8016B0B2026F0C8
:10C3D000ABFE304626F0A8FE0020FCF781FDA84504
:10C3E000EAD1082026F0A0FEA02026F09DFEA02085
:10C3F00026F09AFE002026F097FE10F02005F6D1D8
:10C40000DAF80000FDF760F9042026F0DDFE4FF0B9
:10C41000FF3389F800501A46FFF755B8531C2B60BC
:10C420001678FF2E01F04D82FE2E01F0CB812846BA
:10C43000FDF7D4FE2B686A68D21A002A06DD5A1C62
:10C440002A601B7813B90B2E41F21382242E0DD8CB
:10C45000404A4FF0FF3322F816001A46FFF733B870
:10C46000531C2B6013780A2B01F0EC814FF0FF3343
:10C470001A46FFF728B8531C2B6010787A1E032841
:10C48000D2B2F3D8411EC9B2334E344B01EB410155
:10C4900006EB4101187049780028E7D08A42E5D1BF
:10C4A0000021C3F80610C3F8021099725AB1013284
:10C4B00029681A4401330131296011F8010C03F88D
:10C4C000010F9342F7D1264B1B78002BCED021F0E1
:10C4D00073FF4FF0FF331A46FEF7F5BF1346511CAA
:10C4E0002960204E13F8021B71702B605378337053
:10C4F000D31C2B609378B3702846FDF76FFE2B6832
:10C50000F0801A46591C296012F8021B31712A600A
:10C510005B7873714FF0FF331A46FEF7D4BF531C9C
:10C520002B6013780A2B01F01E81502B9ED12846D8
:10C53000FDF754FE0C4E30802846FDF74FFE4FF0BD
:10C54000FF3370801A46FEF7BEBF00BF8C68002024
:10C550000DCA0020B0C70020E4E00308AC70002042
:10C56000AC2C00205C250020002D00207D6A0020DE
:10C57000247C0020A8F10B00EF283FF677AF01A341
:10C5800053F820F0F1CF00086DC400086DC4000816
:10C590006DC400086DC400086DC400086DC40008B7
:10C5A0006DC400086DC400086DC400086DC40008A7
:10C5B0006DC400086DC400086DC400086DC4000897
:10C5C0006DC400086DC400086DC400086DC4000887
:10C5D0006DC400086DC400086DC400086DC4000877
:10C5E0006DC4000839CF00086DC4000837D20008B8
:10C5F0006DC4000815D200086DC400086DC40008A1
:10C600006DC4000803D200086DC4000863D100089F
:10C610006DC4000877D200086DC4000851D200082C
:10C620006DC40008A9D200086DC400089DCF0008A1
:10C630006DC40008E7D000086DC400086DC4000890
:10C640006DC400086DC40008C3B400086DC40008C0
:10C65000CBD000086DC400086DC40008B1D000083C
:10C660006DC400086DC400086DC400086DC40008E6
:10C670006DC400086DC400086DC400086DC40008D6
:10C680006DC400086DC4000871D000086DC40008B6
:10C69000B9D300086DC400086DC4000835D1000886
:10C6A0006DC400086DC400086DC400086DC40008A6
:10C6B0006DC400086DC400086DC40008BBD200083A
:10C6C0006DC40008C9CE00086DC400082FCE000854
:10C6D0006DC40008D1CD00086DC40008A9CD0008C4
:10C6E0006DC400086DC400086DC400086DC4000866
:10C6F0006DC400086DC400086DC400086DC4000856
:10C700006DC400086DC400086DC400086DC4000845
:10C710006DC400086DC400086DC400086DC4000835
:10C720006DC400086DC400086DC400086DC4000825
:10C730006DC400086DC400086DC400086DC4000815
:10C740006DC400086DC400086DC400086DC4000805
:10C750006DC400086DC400086DC400086DC40008F5
:10C760006DC400086DC400086DC400086DC40008E5
:10C770006DC400086DC400086DC400086DC40008D5
:10C780006DC400086DC400086DC400086DC40008C5
:10C790006DC400086DC400086DC400086DC40008B5
:10C7A0006DC400086DC400086DC400086DC40008A5
:10C7B0006DC400086DC400086DC400086DC4000895
:10C7C0006DC400086DC400086DC400086DC4000885
:10C7D0006DC400086DC400086DC400086DC4000875
:10C7E0006DC400086DC400086DC400086DC4000865
:10C7F0006DC400086DC400086DC400086DC4000855
:10C800006DC400086DC400086DC400086DC4000844
:10C810006DC400086DC400086DC400086DC4000834
:10C820006DC400086DC400086DC400086DC4000824
:10C830006DC400086DC400086DC400086DC4000814
:10C840006DC400086DC400086DC400086DC4000804
:10C850006DC400086DC400086DC400086DC40008F4
:10C860006DC400086DC400086DC400086DC40008E4
:10C870006DC400086DC400084FCD000877CE0008D5
:10C8800017CD00086DC4000895CC00082BCC00081B
:10C890000FCC00086DC40008F5CB00088FCB000852
:10C8A00067CB000859CB0008FBCA00086DC400081C
:10C8B000CDCA00086DC400086DC40008ABCA0008EA
:10C8C0007DCA000869CA000841CA000821CA0008D8
:10C8D000FFC90008D3C900086DC400086DC4000872
:10C8E0006DC400086DC400086DC400086DC4000864
:10C8F0006DC400086DC400086DC400086DC4000854
:10C900006DC400086DC400086DC400086DC4000843
:10C910006DC40008B9C900086DC400086DC40008E2
:10C920005FC900086DC400086DC400086DC400082C
:10C930006DC400086DC400086DC400086DC4000813
:10C9400045C90008BF4B1B78DB073FF58FAD04F0EE
:10C9500043FA05F0C5F801231A46FEF7B4BD531C8F
:10C960002B6013780F2B3FF681AD911C2960C3EB30
:10C97000C303B5495078C854D01C28600B44917843
:10C980005970111D2960D1789970511D2960117954
:10C99000D970911D296051791971D11D2960917942
:10C9A000597102F108012960D2799A7126F06AF86A
:10C9B00001231A46FEF787BD2846FDF70FFCA34E5C
:10C9C000B0812846FDF70AFC012370811A46FEF764
:10C9D0007ABD1146531C2B609D4B11F8020B187049
:10C9E000296051785970D11C296091789970111D76
:10C9F0002960D278DA7001231A46FEF764BD284612
:10CA0000FDF7ECFB934EB0822846FDF7E7FBF08282
:10CA10002846FDF7E3FB012330831A46FEF753BD9A
:10CA20001346511C296013F8020B2B60D31C51785C
:10CA30002B6092781CF054FE00287EF442AD15E580
:10CA40001346511C2960844913F8020B08702B60AF
:10CA50007E4953788B70D31C2B60804B92789A70F0
:10CA600001231A46FEF72FBD7D4B7E4918684A22E6
:10CA70002EF098FD01231A46FEF725BD1146531CE2
:10CA80002B60794B11F8020B18702960517859709E
:10CA9000D11C296092789A702846FDF79FFB734A53
:10CAA0000123D0801A46FEF70EBD2846FDF796FBFF
:10CAB0006E4E30802846FDF791FB70802846FDF7CA
:10CAC0008DFB0123B0801A46FEF7FDBCDFF8BC8168
:10CAD00098F80030002B3EF4F4AC654F0026284651
:10CAE000FDF77CFB15F082FF98F80030A7EC010AF7
:10CAF00001369E42F3DBFEF7E4BC0F2F7FF4B6ACA9
:10CB0000531C2B601678072E3FF6B0ACDFF88081FF
:10CB100028460C27FDF762FB07FB06F708EB070624
:10CB2000B0802846FDF75AFBF0802846FDF756FBFB
:10CB30002B6830811A46591C296012F8021BB17209
:10CB40002A605B78F3722846FDF730FB012348F832
:10CB500007001A46FEF7B7BC2846FDF73FFB012346
:10CB60001A46FEF7B0BC531C2B601078060600F185
:10CB7000F786344B1B78DD073EF5A3AC032828BFAE
:10CB8000002004F00DF901231A46FEF79CBC531C4B
:10CB90002B60284692F80090FDF708FB8046284657
:10CBA000FDF704FB07462846FDF700FB064628462E
:10CBB000FDF714FB2846FDF711FB2B6801332B60B2
:10CBC000B9F1000F00F0B786B9F1100F7EF479AC1F
:10CBD000284BC3F800805F600EB1274BDE60274909
:10CBE000274B0222081F1A702BF018FF01231A4648
:10CBF000FEF769BC134B1B78D8073EF562AC04F016
:10CC00009FF904F06DFF01231A46FEF75CBC0D4B43
:10CC10001B78DA073EF555AC1A490A78012342F031
:10CC200004020A701A46FEF74EBC064B1B78D90761
:10CC30003EF547AC144A4FF4C871012311801A46DF
:10CC4000FEF741BC4C65002054C3002090410020F9
:10CC50008C68002084BB0020647C0020A841002058
:10CC60004027002024E7030888410020C441002019
:10CC7000CC410020982C0020982300209C2C0020E0
:10CC8000826700206A250020D0D00020D1CE00206D
:10CC900060C20020092F7FF6E9ABDFF8D08313468E
:10CCA000511CD8F80060296013F8021B31702B600A
:10CCB0005378B370D31C2B609378642B02F104017A
:10CCC000A8BF642373712960D378642B02F1050136
:10CCD000A8BF6423B37129601379F371931D2B608E
:10CCE0005379642B28BF6423D11D33722960937953
:10CCF000F37002F108032B60D37933712846FDF7F6
:10CD00006DFA0A2F708140F0368612F0B1FA0123D5
:10CD10001A46FEF7D8BBC34B1868D31C0146213214
:10CD20009E1E2E6013F8036C0E705E1E2E6013F8AC
:10CD3000026C4E702B6013F8016C8E7003339A42B4
:10CD400001F10301ECD126F077F8FEF7BABBC7F387
:10CD50004707122F3FF68AABB7B116AB0DF1160895
:10CD600003EB4706C146423E2846FDF737FA29F84D
:10CD7000020F4E45F8D1AC4B38F8022F23F8022FA2
:10CD8000C845F9D1112F09D8A84A7B00023B1344AA
:10CD90000021223223F8021F9A42FBD1A44901222A
:10CDA00013460A70FEF78FBB1346511C2960A14938
:10CDB00013F8020BC8702B609F4953780B70D31C7B
:10CDC0002B609E4B9278DA7001231A46FEF77BBBEC
:10CDD0002846FDF703FA2846FDF700FA2846FDF736
:10CDE000FDF92B688F4E9A1CD6F800802A605A787D
:10CDF00088F82F20DA1C2A609A7888F83A201A1DC1
:10CE00002A60DA7888F83B2007332B602846FDF744
:10CE1000E5F9A8F83E002846D6F80080FDF7DEF9CF
:10CE2000112FA8F83C0000F26E8530688BE7531C88
:10CE30002B607C4EDFF814821378D6F8009088F8C7
:10CE400005302846FDF7CAF9A9F820002846D6F88B
:10CE50000090FDF7C3F9052FA9F8220000F29B8589
:10CE600003F0C4FF21F08CFB306815F0F3FB0123C5
:10CE70001A46FEF728BB531C2B6013787049002B11
:10CE800000F01A850B7843F00203901C0B706D4E76
:10CE90002860537833702846FDF788F9706028467B
:10CEA000FDF784F9B0602846FDF798F9B08128466F
:10CEB000FDF794F9644970820A78012342F0020276
:10CEC0000A701A46FEF7FFBA1346511C29605F4EDE
:10CED00013F8021BB1702B605D4953780B70D31CA3
:10CEE0002B605C4F93783B71131D2B60D378092B1B
:10CEF000A8BF09232846BB70FDF770F92B686A6844
:10CF00003880D11A012905DD2846FDF767F92B681D
:10CF10006A6878829A4240F0058503F067FF2B68C3
:10CF20006A689A423EF4CDAA5A1C2A601B78FB70AC
:10CF300001231A46FEF7C7BA531C2B60107813283A
:10CF40003FF694AA931C2B605678434B002105E0D2
:10CF50000131242903F10C033FF488AA1F7AB74258
:10CF6000F6D13E4E3E4B0C2707FB0161D61C91F8D3
:10CF70003C1003F820102E6003EB80039178597069
:10CF8000111D2960D0789870501D286025491279AC
:10CF90000868DA7012F0FAF8FEF793BA531C2B60A7
:10CFA00013780E2B3FF662AA911C29605678032E47
:10CFB0003FF65CAA2B48062101FB03F14318D71C5E
:10CFC0005E712F6096784654111D2960D178597092
:10CFD000511D296011799970911D29605179D9707D
:10CFE000D11D296092791A7101231A46FEF76BBA96
:10CFF0001D4B102F4FF0000228BF10271A605A60F7
:10D000009A60DA601A74002F3EF45BAA2A6817440B
:10D0100001322A6012F8011C03F8011BBA42F7D151
:10D02000FEF74FBA402700206A5F00206C5F0020A7
:10D03000905F002090410020A0410020A8410020E6
:10D040006A2500206C25002080670020647C002079
:10D050008441002084BB0020E4DD0308A8DD030830
:10D06000D44600201C4800200563002044270020EF
:10D070001346511C2960C44E13F8021B31702B60FB
:10D08000537873702846FDF7A9F82B6870805A1CF6
:10D090002A601B7833712846FDF7A0F82B68F080D2
:10D0A0005A1C2A601B78337201231A46FEF70BBA0A
:10D0B000B64B02F1080101322A6012F8010C03F8A4
:10D0C000010F9142F7D1FEF7FCB91346511C2960BC
:10D0D000AF4913F8020B88702B6053784B70012313
:10D0E0001A46FEF7F0B90723B7FBF3F3C3EBC3010E
:10D0F000791A7FF4BBA9DBB203F1FF395FFA89F932
:10D10000002B3EF4DEA9DFF88CA209F10109884664
:10D11000531C2B6092F900209E4B002693F90210BD
:10D12000914200F062830136052E03F10803F5D128
:10D13000FFF79CB9984B1B78012B3EF6C2A911460C
:10D14000531C2B60954B11F8020B98702960517895
:10D150001970D11C296092785A7001231A46FEF783
:10D16000B2B9531C8E4E2B60137833722846FDF7EC
:10D1700035F8B0832846FDF731F830832846FDF7AF
:10D180002DF82B6870835A1C2A601B78F374082FC3
:10D190007EF697A92846FDF721F8F0842846FDF78A
:10D1A0001DF80C2F30857EF68CA92B681A46591C69
:10D1B000296012F8021BB1772A605B7886F820306C
:10D1C0002846FDF70BF8102FB0847EF67AA92B685D
:10D1D0005A1C2A601B78F3722846FCF7E7FF2B687D
:10D1E000F0605A1C2A601A783274162F7EF669A9EC
:10D1F0009A1C2A605B7886F8213001231A46FEF7D4
:10D2000062B9531C2B60674B12781A7001231A46BF
:10D21000FEF759B92846FCF7E1FF634E3060284617
:10D22000FCF7DCFF70602846FCF7D8FF0123B060F4
:10D230001A46FEF748B95D4E002333602846FCF7D6
:10D24000B5FF32680123024332601A46FEF73BB94C
:10D25000531C2B6016781F2E3FF608A9052F7FF46C
:10D2600005A92846FCF7A2FF514B43F8260020F001
:10D27000D7FAFEF726B94E4E06F140072846FCF7CE
:10D28000ADFF2B68A6F88000591C1A46296012F8D9
:10D29000021B86F882102A605B7886F88330043699
:10D2A000B742EBD1FEF70DB9531C2B603C4B127803
:10D2B0005A7501231A46FEF706B92846FCF78EFF79
:10D2C00006462BF0B9FCFF283EF4FBA8B6F57A7FA2
:10D2D00080F0DB820DF15809002309F8403DF70882
:10D2E000494604A88DF8103001372BF085FC9DF8D5
:10D2F0001030FFB206F00706BB4206F1010603D16B
:10D300009DF81830B34203D0314638462BF080FCEC
:10D310002B686A68D21A012A7EF7D3A85A1C16A86D
:10D320002A6000221E7800F8482D2BF059FC9DF849
:10D330001030B3420AD01F4B1B683BB19A79B242FE
:10D3400004D31B681B690BB1304698472B685A1CE5
:10D350002A60484600221D788DF818202BF034FCF6
:10D360009DF81830AB423EF4ACA8124B1B68002B62
:10D370003EF4A7A81B685B69002B3EF4A2A82846D0
:10D380009847FEF79EB800BFEC4E002057C0002023
:10D39000B4410020387C0020FC50002018C8002038
:10D3A00058C0002020290020B03F0020F850002065
:10D3B000D061002018630020531C2B601778112FB8
:10D3C0003FF654A8931C2B60CA4E537806F81730CA
:10D3D0002846FCF703FF40F6CA039842A8BF184648
:10D3E00040F2EE23984206EB4706B8BF18460123E9
:10D3F000A0F2EE211A46192091FBF0F17170FEF7B0
:10D4000062B800231B7AFFDE23685A1C2260197061
:10D4100029882046FCF736FF2368EA78591C2160EA
:10D420001A7023682A79591C21601A702368AA7916
:10D43000591C21601A7023686A79591C21601A707E
:10D44000FEF785BEDFF8ECB200254FF0080A013583
:10D45000242D1AD0C5F120020AFA02F22BFA05F6A1
:10D46000A5F1200316432AFA03F31E4306F0010236
:10D4700000231343EBD0E8B211F082FE0028E6D07F
:10D4800029464846FDF780FAE1E79B4B1B78DF070A
:10D4900000F15D810025994E2F4602E00135242DD3
:10D4A0000DD029463046FDF77FFA0028F6D02946F0
:10D4B0004846FDF779FA002854D10137EEE7904B42
:10D4C000904DB3F850102046FCF7DCFE00212046BA
:10D4D000FCF7D8FE8C4B1A68530103F02001C2F30D
:10D4E00040030B43C2F3800143EA4103C2F3C0018E
:10D4F00043EA8103C2F3401143EAC10102F0100282
:10D5000011432046FCF7BEFE04A904222046FCF786
:10D5100071FE236829787D4A581C20601970118893
:10D520006429A8BF64212046FCF7ACFEB8F1960F31
:10D5300000F0028100212046FCF7A4FE2168B7F12B
:10D54000190348BFA7F11203A3F3C4034A1C2260C6
:10D5500020461A460B7005A9FCF74CFE01231A461B
:10D56000FDF7B1BF394604A8FDF70EFAA5E72B6811
:10D570006A689A4240F0FD80604BFF221A724FF0B9
:10D580000008634D1DF0C8FB41463022614885F814
:10D59000008030F01EFB8DF818809DF818300B2BA2
:10D5A00000F265815C4F5B4E42469DF8183003EBFC
:10D5B000430307EBC3035B7CE3B19DF8183003EB37
:10D5C000430307EBC3035B69A3B19DF8183003EB7A
:10D5D000430307EBC3032021586946F82200FBF7F9
:10D5E000D7FE2B7856F82300FCF76EF82A78013224
:10D5F000D2B22A709DF818300133DBB28DF81830A2
:10D600009DF818300B2BD0D92368591C21601A7053
:10D61000B9F1000F3DF455AF404BC9F8003001237C
:10D620001A46FDF750BF2368B1783D4A581C206068
:10D63000197023681278591C21601A70FEF7E6B938
:10D64000384A92E82200FEF7ACB8D9F8003013F45B
:10D650008053B4EEE88A7FD0F1EE10FAC0F2EF808A
:10D66000B4EEC98AF1EE10FA0DD8DFED2F7A9FEDF6
:10D670002F7A77EEC87AB4EEC78AF1EE10FAB0EEE0
:10D68000678A00F2DC80F7EE007A78EE677AB6EE11
:10D69000007AF0EE696AE7EE876A40F2E932FDEE61
:10D6A000E67A17EE901AB1F5FA6FA8BF4FF4FA6157
:10D6B0009142B8BF114689B2002B3EF4B7AAB5EE2D
:10D6C000408AF1EE10FA40F2DC5308BF1946FEF72B
:10D6D000ADBA95F82420164B002A40F0A7803046BA
:10D6E000FEF7F6B821680123CA1822601A460870AE
:10D6F000FDF7E9BE3C6100204C6500209823002026
:10D70000DC16002000630020B08400200A410020C5
:10D71000FBC00020606000203C890020411C030801
:10D72000844100207C27002000C0884400C082443F
:10D730007CA3002090E33FF423680322591C21605E
:10D740001A7023686A78591C21601A70F6E6069BE5
:10D7500043F0010306939DE6F1EE10FA93DA4FF4DD
:10D760007A71FEF763BA2846FCF738FD9D4EFEF746
:10D77000E2BE5A1C19462A609B4811F8022B02721D
:10D7800029605B784372042A03D9FF2A7EF421A81A
:10D79000F5E696490978994205D8022A7EF419A837
:10D7A000FF2B7EF416A822680123D1182160137084
:10D7B000B9F1000F3DF485AE8D4AC9F800201A4634
:10D7C000FDF781BE931C2B605678022E3EF64EAEBE
:10D7D0002846FCF703FD874A02EB46024FF0FF3371
:10D7E000A2F85E001A46FDF76EBE0AEBC607284691
:10D7F000BA70FCF7F3FC2B682AF836001A46591C5D
:10D80000296012F8021BF9702A605A783A71DA1C02
:10D810002A609A78BA711A1D2A6008F10108DB782B
:10D820007B71C1457FF474ACFDF74BBE597802297A
:10D8300017D003290CBF04203046FEF749B84FF437
:10D840007A713CE7931C2B606B4B51781970D11C9B
:10D85000296091785970111D2960D2789A70FEF76D
:10D8600005BE042A34BF02200320FEF731B8424629
:10D87000CAE6604B00301E4418BF01204FF0FF3352
:10D8800086F84A001A46FDF71EBE0DF118094846F3
:10D890002BF08EF9BDF81830B3423FF439AD574B39
:10D8A0001B68002B3FF434AD1B689B69002B3FF4D1
:10D8B0002FAD304698472BE50B7803F0FD03FFF7BB
:10D8C000E4BA931C2B604E4B51781970D31C2B601B
:10D8D000484E937886F85C30131D2B60D37886F819
:10D8E00056302846FCF77AFCA6F858002846FCF784
:10D8F00075FC2846FCF772FC4FF0FF33A6F85A007F
:10D900001A46FDF7E0BD2B683168581C1A4628609E
:10D9100012F8020B81F831002A605B7881F832300E
:10D92000FFF783BA5A1C2A601B78003318BF012303
:10D93000F371FFF7F2BA334B1020C3F800805F6039
:10D9400028F00CFA304A137843F001031370002ECC
:10D950003DF4B7AD244A0123D6601A46FDF7B3BDA6
:10D9600000F07F00032828BF00201DF015FA0123D6
:10D970001A46FDF7A8BD2B68D8F80020591C29606D
:10D98000197851720B2F3FF4C0A9991C29605B785C
:10D990005370FFF7BAB92846FCF720FCA8F80A0034
:10D9A0002846FCF71BFCA8F80C002846D6F8009087
:10D9B000FCF714FCA9F824002846D6F80090FCF7E0
:10D9C0000DFC0D2FA9F826007FF64AAA2846FCF781
:10D9D00005FCA8F80E002846FCF700FCA8F810008B
:10D9E000FFF73EBA8041002098230020D1CE0020CE
:10D9F00065040108B0C70020B34F00201863002061
:10DA00002C7C00207C2700206A2500202DE9F04F87
:10DA1000A34CDFF8C09294F85C312DED028B834665
:10DA20008FB0002B40F05A8194F8DD31002B39D0B3
:10DA3000D4F8E0319B4AABEB0303934200F2348409
:10DA400094F84862002E00F0B780D4F850324BB3FF
:10DA5000D4F8583240F6B732ABEB0303934221D9E6
:10DA600094F85432002B00F061858F4F013BDBB2FC
:10DA700084F85432002B00F06985D4F8505294F8A1
:10DA80005C2215F8011B94F85D323868C4F85052D6
:10DA90000A44013384F85C2284F85D32FBF706FA0D
:10DAA000C4F858B294F85E32D9F8005043B17F4EB2
:10DAB000306828B194F85F32013B012B40F2F384C7
:10DAC00094F8A03353B17A4E33683BB1D9F8007063
:10DAD000D4F8A433FB1A632B00F22A8294F8DC33C7
:10DAE000022B00F0D482734D95F87430032B00F0B4
:10DAF000488794F8F8336BB1D4F8FC3353B104F091
:10DB0000D1FAD4F8003444F61F62C31A9342074690
:10DB100000F2E88294F87A35002B40F08B8194F87B
:10DB20008B3533B1D4F88C3503F5C333A0339B4523
:10DB300078D294F8C235BBB15F4D2E46D4F8C405F7
:10DB4000FBF7B0F980B1D4F8C405FBF7A3F994F85A
:10DB5000C83507465A1E63B1D4F8C40584F8C825F1
:10DB6000FBF7A0F90028EED10FB0BDEC028BBDE8A9
:10DB7000F08F03225149284630F011F894F8CC3543
:10DB800094F8CD2584F8CF7583F47F4383F0FF03A9
:10DB90009B1ABFB29BB2B7EB132FCFD194F8CE250F
:10DBA000DBB29A42CAD130462BF0A0FE94F8C835B9
:10DBB000184484F8C805C1E73B4F3868FBF772F991
:10DBC000C0B201280FD902283A4D40F0CE842B78FC
:10DBD000002B41F0A087D4F84C32ABEB0303B3F534
:10DBE0007A6F81F09A85D4F85032002B3FF45AAF07
:10DBF00094F84832002B7FF42BAF314B1B689B7895
:10DC000001211E3B00228B4284F8481284F85C22DA
:10DC100041F2D2873868022104302BF08DFF94F84E
:10DC2000543223E794F89035264AC4F88CB502EBB9
:10DC30008302526C42B3244F244E0EADFB1C45F8B8
:10DC4000203D07F1150300210793A523318084F8B7
:10DC500094358021152384F89635284684F8951547
:10DC6000904728463188FCF70DFB069DED1B152DCE
:10DC7000A8BF15252A46394607F118002DF092FC59
:10DC800094F8903584F8C155114A013382FB031290
:10DC9000A2EBE37202EB42029B1A84F8903548E74C
:10DCA000A82300203F0D0300E8CF00209CCF0020D8
:10DCB000E0CF0020200000207429002075290020DA
:10DCC000ECCF002098DF03083C29002086CF0020FD
:10DCD000565555555CC7002000007A44D4F8603191
:10DCE000D9F80020D31A7C2B7FF69EAE94F86431CD
:10DCF0001FED078AC4F86021013384F8643104F50C
:10DD0000CE77242528462BF08FFFB4F87831F7EC36
:10DD1000016A07EE103AF8EEE66AB8EEC77A013506
:10DD2000C6EE877AEDB267EE887AFDEEE77ACDED42
:10DD3000007ABDF90060F0B22BF04CFFC6F307206B
:10DD40002BF048FF272DDDD130202BF06DFFD94E71
:10DD500000202BF03FFF00202BF03CFF30685E21BD
:10DD6000FBF7A4F894F8643113F0030528D1D4F834
:10DD7000602141F288339A4201F2C98714202BF0C6
:10DD800053FFCD4AB4F9B031DD1782FB0323C5EB55
:10DD9000A3052DB2E8B22BF01DFFC5F307202BF031
:10DDA00019FF1C202BF040FF00202BF013FF002058
:10DDB0002BF010FF5E213068FBF778F894F864319F
:10DDC00013F0070501F02E85282B7FF42DAE0025DA
:10DDD0001720D9F8008084F864512BF025FF2846DD
:10DDE0002BF0F8FEB54BB64FA3FB08239B0BA7FB0C
:10DDF00003125209C2EB0212A3EB8203D8B22BF03A
:10DE0000E9FE18202BF010FFAE4BA3FB08239B0963
:10DE1000A7FB03125209C2EB0212A3EB8203D8B292
:10DE20002BF0D8FE28462BF0D5FE30685E21FBF79C
:10DE30003DF8F9E5A44D2A7832B1A449D4F87C051F
:10DE4000FAF7FCFF00232B70D4F8803503F5C333B9
:10DE5000A0339B45FFF463AE94F88935C4F880B5D0
:10DE6000234493F88455E80701F10B86A90701F1D3
:10DE7000CD856A0701F191852A074DD5944B07930B
:10DE80000EAA1046A3F1210240F8202DA3F124028E
:10DE900006460090002003F8240C1125022355703B
:10DEA0009370D4F8C8113046FCF7AEF93046D4F878
:10DEB000CC11FCF7A9F9B4F8D6317F4903EBC303C1
:10DEC0009B00053381FB0321DB17C3EBA10189B262
:10DED0003046FCF7B1F9B4F8D83103EB83035900AD
:10DEE00089B23046FCF7A8F994F8C231009D9B072F
:10DEF00043BFB4F8D01101F57A7189B24FF47A7149
:10DF00002846FCF799F9069B94F8C421591C069100
:10DF100028461A702BF0F2FE94F8893594F88A1589
:10DF2000013393FBF1F201FB123384F88935F6E5F6
:10DF300041202BF0B1FD604DB4F9AE31DFF8A08186
:10DF400085FB0320DB17C3EBA00080B22BF088FD1C
:10DF5000B4F9AC3185FB0320DB17C3EBA00080B222
:10DF60002BF07EFDB4F9B03185FB0320DB17C3EB4A
:10DF7000A00080B22BF074FD98F800103068FAF71A
:10DF800095FF94F8A85315F0010200F0B585514BA8
:10DF90001B689A0668D594F8C2319B0701F1B583D6
:10DFA000012547202BF078FDD4F8C8012BF024FD83
:10DFB000D4F8CC012BF020FD474AB4F8D6313068B4
:10DFC000A2FB0323C3F3471A5146FAF76FFFB4F8D5
:10DFD000D02198F80030642000FB02F08AEA0303A5
:10DFE00088F800302BF008FD94F8C431306845EA19
:10DFF0008305EDB22946FAF759FF98F800303068EA
:10E000005D40294688F80050FAF750FF94F8A8536D
:10E0100055BB4F202BF040FDD4F8D4032BF0ECFC83
:10E02000D4F8D8032BF0E8FC28462BF0E5FC0121BE
:10E030003068FAF73BFF94F8C25198F80030306826
:10E0400005F00105294683F0010388F80030FAF74E
:10E050002DFF98F8003030685D40294688F8005060
:10E06000FAF724FF94F8A8531C4AC4F8A4736B1C55
:10E07000DBB2A2FB0312D20802EB8202A3EB420343
:10E0800084F8A83394F8DC33022B7FF42CAD04F031
:10E0900009F8D4F8E06340F6B833861B9E4201F2DB
:10E0A0004E8294F8EC333A2B01F03A85002384F841
:10E0B000DC331EE5F0CF00206766666673B2E74585
:10E0C00089888888D34D62103CD0002018D0002069
:10E0D00018D00020B08400201F85EB51CDCCCCCCD3
:10E0E000E4CF002094F80634002B40F0CB846A4B38
:10E0F0001B6848F6034113F0080F49F607464FF036
:10E10000190208BF0E46580784F8062403D546F4C2
:10E11000005646F00806990648BF46F4804694F833
:10E12000B85148BF46F02006C6F30908002D41F05B
:10E130001B8394F8B931002B41F024861D466420DE
:10E140004FF0FF3A4FF0000C06960796ADF82650B8
:10E15000CDF82080ADF828A08DF83600ADF824C0A9
:10E16000ADF82AC0ADF82CC0ADF82EC0ADF830C067
:10E17000ADF832C0ADF834C00DF1180EBEE80F0096
:10E18000464E35460FC59EE80F0007C525F8023BF1
:10E19000180C0121FE221F23287084F8531084F8E4
:10E1A0004E2084F84F3094F8162484F851C051184A
:10E1B000C82084F8161484F85020311F84F85200C7
:10E1C0004FF6FF7501E011F8013B6B4083EA031342
:10E1D000DBB21A0982EA152242EA03228E4282EA5F
:10E1E000C305F0D12D49A4F84C5001F11F0011F8DE
:10E1F000013B6B4083EA0313DBB21A0982EA152262
:10E2000082EA032282EAC3031BB29DB28142A4F8D0
:10E210004C50ECD183F07C0383EA0313DBB21A0980
:10E2200082EA152282EA032282EAC3031BB29AB26F
:10E230004FEA122C5FFA83FE194EA4F84C2084F8A2
:10E2400074C084F873E004F14E0804F16E0AD8F843
:10E250000000D8F80410D8F80820D8F80C3035465B
:10E260000FC508F11008D0452E46F0D1D8F80000AF
:10E2700028600C4D98F80430337105F1270684F8B6
:10E2800065E484F866C415F8011FD4F8FC03FAF7B6
:10E290000DFEAE42F7D1F8E3B0840020FC2300204D
:10E2A000E8270020E7270020D94ADA4BD07AD9F8AE
:10E2B0000010D4F810221B88891A4FF47A7202FBDE
:10E2C00000F2DDB200201B0A914284F8025284F869
:10E2D000F85184F8033284F8F93184F8E60184F8BF
:10E2E000E80181F0F480CC4BCC491A689B6894F823
:10E2F000C20181FB026581FB0361D217DB17C2EB10
:10E30000A502C3EBA10315121912F42684F800220A
:10E31000012284F8015284F80432302584F8051271
:10E3200084F8FE617521782384F8FF21860794F82C
:10E33000C42184F8065284F8071284F8083284F85D
:10E34000322241F1BF80D4F8C851B549D4F8CCC1CC
:10E35000B448B54BDFF8E8A281FB0567EE1781FBF7
:10E360000CE1C6EBA7564FEAEC77C7EBA15100FBD7
:10E37000065707EB47077F0000FB01C083FB07E858
:10E3800000EB400040004FEAA848052A4FEAD57547
:10E390004FEAE77201EB810183FB00E301EB8101AE
:10E3A00006EB860684F82152A8EB02054FEAA34E3D
:10E3B00000912A464FEAE0716DB206EB860605EB46
:10E3C0008606B4F8D631AEEB010529464FEADC7C6F
:10E3D0000AFB127203EBC303944FDFF868E284F880
:10E3E00026C24FFA81FC00990AFB15054FEA830308
:10E3F000B4F8D0010CEB81018EFB03CE87FB028CBD
:10E400004FEAE27287FB0587C2EB6C12B6B289B2A3
:10E410004FEAE373B4F844C284F8226200F5FA705C
:10E420004FEAE5754FEA112AC3EBAE1EC5EB67153F
:10E430004FEA162380B24FEA222884F828A284F8F3
:10E4400023324FEA252784F82712CEF307264FEA16
:10E45000102184F8242234BF4FF0320A4FF0330ADF
:10E460004FEA1C22B4F8463284F8258284F82952F7
:10E4700084F82A7284F81FE284F8206284F82D025E
:10E4800084F82E1284F833A284F82BC284F82C224C
:10E4900084F8343294F84862C4F8E0B1002E7FF476
:10E4A000D4AAFFF789BB624F4FF0010A4FF0000872
:10E4B00008E01B2B00F07B820D2B00F0878187F892
:10E4C00001A03068FAF7EEFC00285BD03068FAF75C
:10E4D000E1FC83B27E2BD9F800204CD07A78002A58
:10E4E000EFD194F860120029E3D07D2B00F0468232
:10E4F00094F864E2BEF1000F04D080F02003DBB298
:10E5000084F864224A1CD2B2092A635484F8602237
:10E5100000F02A82082AD4D8B4F86222134403EB0C
:10E52000132303F0FF03A4F86232CAE7C4F85032A1
:10E5300084F848322BF034FB94F854323D4F013BC1
:10E54000DBB284F85432002B7FF497AA94F85C1263
:10E5500094F85D3238684A1C013384F85C2284F8F0
:10E560005D32FAF7A3FCFFF79BBA2BF009FB0123FE
:10E570002B70FFF738BB84F8608284F8618287F8DB
:10E5800001809EE794F865322BB1637884F86502C8
:10E59000302B01F0398394F86122274B274FDFF8A5
:10E5A000A8E0DFF86CC00126002A3FF489AAD9F858
:10E5B0000000401B012825D894F87883B8F1000F9B
:10E5C00040F0068294F890A303EB4A0000890028EB
:10E5D0003CD184F8906338688106E5D594F8C2018F
:10E5E0008007E1D5B4F8D62110494FF4F36303FB5B
:10E5F00002F381FB0321DB17C3EB61114FF40360CE
:10E600002BF080FA002384F86132FFF759BA00BF7B
:10E6100078CF002088CF00208CCF00206766666608
:10E620006BCA5F6B806967FF83DE1B431F85EB51FD
:10E6300020000020E8CF002098DF0308B0840020ED
:10E6400040420F00D34D621088C000200AF1010A39
:10E650005FFA8AFAB0F5E06F84F890A300F0998031
:10E660001AD8B0F5047F00F0318136D8B0F5887F34
:10E6700000F00981B0F5007F00F0EF80B0F5807FF9
:10E6800092D1396849078FD500212BF03BFA00233E
:10E6900084F86132FFF714BAB0F5026F00F001811F
:10E6A0006CD8B0F5E46F00F08380B0F5006F00F037
:10E6B0009380B0F5E26F7FF477AFD4F8A021B4F87F
:10E6C0007811642303FB02F393FBF1F12BF01AFAA8
:10E6D000002384F86132FFF7F3B9B0F5826F00F0E0
:10E6E0002481B0F5C06F00F01081B0F5806F7FF429
:10E6F0005BAF94F891330133DBB2032B00F26281FC
:10E7000042F2107184F8913301FB03F1B4F89233B3
:10E71000002B40F055810131D24B1B78DF07B4F854
:10E72000943348BF0431DD0748BF0A31980748BF1A
:10E7300014311A0648BF2831DF0548BF28315D076C
:10E7400048BF6431180748BFC8319A0548BF01F572
:10E75000C8719F0648BF01F57A71DD0648BF01F513
:10E76000FA61580648BF01F57A614FF480602BF0DA
:10E77000C9F9002384F86132FFF7A2B9B0F5046F3C
:10E7800019D0B0F5116F4DD0B0F5036F7FF40CAF19
:10E7900021E7D4F89C21B4F87811642303FB02F339
:10E7A00093FBF1F12BF0AEF984F86182FFF788B9A1
:10E7B000D4F8A421EFE7B4F9B01101EB81014900CD
:10E7C0002BF0A0F984F86182FFF77AB984F860A28F
:10E7D0002370A4F8621274E6386881067FF5E4AE0F
:10E7E00094F8C20180077FF5DFAE1AF0010F40F008
:10E7F0007887D4F8C8219C4982EAE273A3EBE273DC
:10E8000003EB5303A1FB0331C908002AB8BF41F051
:10E8100080414FF400602BF075F9002384F86132D9
:10E82000FFF74EB994F8B80100283FF4BDAE8F4908
:10E83000087800283FF4B8AE8D4B1B8803EB8303A8
:10E84000590080464FF4116091FBF8F12BF05AF912
:10E85000002384F86132FFF733B994F8B901002836
:10E860003FF4A2AE834B84491B6881FB0321DB1775
:10E87000C3EBA1014FF400702BF044F9002384F89E
:10E880006132FFF71DB9386841077FF58DAE002171
:10E890004FF488702BF036F9002384F86132FFF7CB
:10E8A0000FB9396889067FF57FAE94F8C2A11AF0D6
:10E8B000020F3FF479AEB4F8D031642101FB03F1CB
:10E8C0002BF020F984F86182FFF7FAB894F8B801C8
:10E8D00000283FF469AE6549087800283FF464AE2B
:10E8E000664B5B7B002B01F04982614B198891FBE1
:10E8F000F0F101EB810149004FF404702BF002F9B3
:10E90000002384F86132FFF7DBB894F8B9010028DE
:10E910003FF44AAE574B4FF4C06099682BF0F2F8C1
:10E92000002384F86132FFF7CBB83868810640F1E4
:10E93000F18594F8C22194F8C41112F0020F0CBFB3
:10E9400000234FF47A7312F0010F0CBF00224FF432
:10E95000FA62134419444FF482602BF0D3F8002379
:10E9600084F86132FFF7ACB8B4F86222C2F1FF025A
:10E9700093427FF4A4AD84F865A2A0E584F864A274
:10E980009FE5D4F8F40303685B69984700283FF4D7
:10E99000B0A8D4F8F403036801219B6998470222C8
:10E9A000002385F8742084F8DC33FFF7A2B83068C0
:10E9B000FAF778FA00287FF482AD84F861A280E546
:10E9C0000231A9E6012384F8913342F210719DE6E9
:10E9D000D4F868322A4E94F88E23B34201F0B08105
:10E9E000511C94F88F03D4F86C7284F88E1302F0E3
:10E9F0000F028DF818200DF11902F91A002941F3C0
:10EA0000008306A900910DF11E0502E0002E40F3DF
:10EA1000A0850133C4F8683213F8011C02F8011B09
:10EA2000AA42A7EB030680EA0100EFD384F88F0324
:10EA300001F0E182531CAB42107038BF002203D2B8
:10EA400003F8012BAB42FBD1009932202BF03EF8AA
:10EA50004FF00008002384F8788384F86132FFF7D0
:10EA60002FB800BF4C6500201F85EB51CFCF002091
:10EA700088CF00208CCF00206766666678CF0020A4
:10EA800020260020013B84F8063494F80734002B3C
:10EA900040F0958094F84815D9F800E00A2284F8EF
:10EAA0000724002900F059850129B4F854A541F242
:10EAB00021830229B4F8568501F06A810329B4F84C
:10EAC00058C501F04283B4F85A250092042901F098
:10EAD00037830529B4F85C5501F02E830629B4F874
:10EAE0005E0501F026830729B4F8602500F03D8516
:10EAF000B4F8623500F039BDB4F89433D80513D4B6
:10EB0000D90601F1EF809D0601F14981580601F116
:10EB10006F82190701F17B82DD0701F1D78213F0C3
:10EB2000020F0CBF04220C22B24994F8AF3391F8C3
:10EB300000A00AF0010A0BB14AF0020A5320009229
:10EB40002AF0AAFFAC4B1B8803EB830303EB830380
:10EB5000980080B22AF084FF00202AF081FFB4F8E8
:10EB6000D033A6493068C3EBC3135B0081FB03219C
:10EB70001944DD17C5EB6125EDB22946FAF796F980
:10EB800098F80030009A306842EA0A0A5D40002195
:10EB900088F80050FAF78AF951463068FAF786F992
:10EBA00098F8003030688AEA0303DBB2194688F827
:10EBB0000030FAF77BF994F8A853FFF729BA013B24
:10EBC00084F8073494F80A34002B40F06E848C4BA0
:10EBD0001B68192284F80A249A0640F11A8294F8D4
:10EBE000C2319B0700F1B885012603F05BFAB4F847
:10EBF000D811B4F8D051D4F8C831069001EB810196
:10EC0000019349004FF47A70ADF83210D4F8CC215A
:10EC1000B4F8D68194F8C4C101998DF8346000FB32
:10EC200005F04FF0000E06AB4FF6FF75ADF83080E3
:10EC30008DF835C0CDF81CE00A9008910992ADF826
:10EC40002C50ADF82E5098460093B8E80F006D4E4A
:10EC5000B446ACE80F0098E80F00ACE8070094F861
:10EC60001624ACF8003084F851E0A6F1040A02F151
:10EC7000010E1820FE211E234FF0C80CD04684F848
:10EC8000502084F816E484F8530084F84E1084F879
:10EC90004F3084F852C001E018F8013B6B4083EA22
:10ECA0000313DBB21A0982EA152242EA032246451F
:10ECB00082EAC305F0D1534AA4F84C5002F11E0178
:10ECC00012F8013B6B4083EA0313DBB2180980EAB8
:10ECD000152080EA032080EAC3031BB29DB28A425A
:10ECE000A4F84C50ECD183F0180383EA0313DBB291
:10ECF0001A0982EA152585EA032282EAC3031BB2B8
:10ED00009AB2DBB24FEA122E019384F87230DFF828
:10ED100000C1A4F84C2004F16E0384F873E004F100
:10ED20004E060293F36830687168B26865460FC595
:10ED3000029B10369E42AC46F4D13068CCF80000FD
:10ED4000314D9DF8043084F8643484F865E42E462F
:10ED500016F8011FD4F8FC03FAF7A8F82B4BB342BE
:10ED6000F6D103F09FF9B4F9B011DFF8A8E0B4F8D8
:10ED7000D06106908EFB010EC9174FF47A7000FB2C
:10ED800006F0D4F8C821D4F8CC31009E0990C1EB2C
:10ED9000AE014FF0000EADF82CE0ADF82EE0ADF86E
:10EDA00030E0ADF832100A90079208930FCE04F1CC
:10EDB000540CACE80F0096E8070021231C268CE8D1
:10EDC000070084F85330C8226FF0010384F851E043
:10EDD00084F84E3084F84F6084F8522094F816344A
:10EDE00084F850305A1C84F8162433464FF6FF7EC0
:10EDF000564613E04C65002088CF00200308208091
:10EE0000B0840020FC230020E72700200D280020EC
:10EE1000E82700206766666616F8013B83EA0E0362
:10EE200083EA0313DBB21A0982EA1E2242EA0322B2
:10EE3000B04582EAC30EEFD1D248A4F84CE000F10D
:10EE40001C0110F8013B83EA0E0383EA0313DBB2D3
:10EE50001A0982EA1E2282EA032282EAC3031BB253
:10EE60001FFA83FE8842A4F84CE0EAD183F06803DD
:10EE700083EA0313DBB21A0982EA1E2282EA032222
:10EE800082EAC3031BB29AB2DBB2110A019384F87F
:10EE90007030DFF800C3029104F16E03A4F84C2037
:10EEA00084F8711004F14E080393D8F80C30D8F8A8
:10EEB0000000D8F80410D8F80820E646AEE80F00A5
:10EEC000039B08F110089845F446EED1B8F80030DD
:10EED000AEF800309DF8043084F862349DF80830B4
:10EEE00084F86334A84618F8011FD4F8FC03F9F736
:10EEF000DDFFA54B4345F6D1D4F8D433D4F8D8235D
:10EF000006934FF0000E009BCDF820E0079293E8A7
:10EF1000070004F1540383E8070094F8162484F8EA
:10EF200051E0312002F1010EFE210C2384F8502023
:10EF3000C82284F816E484F8530084F84E1084F84C
:10EF40004F3084F852204FF6FF7E01E01AF8013B63
:10EF500083EA0E0383EA0313DBB21A0982EA1E2254
:10EF600042EA0322564582EAC30EEFD18549A4F84E
:10EF70004CE001F10C0011F8013B83EA0E0383EA37
:10EF80000313DBB21A0982EA1E2282EA032282EA12
:10EF9000C3031BB21FFA83FE8142A4F84CE0EAD1FE
:10EFA00083F0270383EA0313DBB21A0982EA1E2ED9
:10EFB0008EEA032E8EEAC30EA2460FFA8EFE1FFAC9
:10EFC0008EF65AF84E0FDFF8CCC1A4F84C604FEA29
:10EFD00016285FFA8EFE84F860E084F86180DAF823
:10EFE0000410DAF80820DAF80C30BAF810A0ACE80F
:10EFF0000F0004F25346ACF800A084F8538484F860
:10F0000052E415F8011FD4F8FC03F9F74FFFAE42A4
:10F01000F7D194F80E64002E40F0BE80B4F9AC2114
:10F02000B4F9AE319FED596AD9F80010069106EE99
:10F03000902AB4F9B021534D84F851605B4207EE39
:10F04000102A07EE903AF8EEE66AF8EEE77AB8EEA4
:10F05000C77A67EE867A66EE866A27EE067A00221F
:10F06000CDED087ACDED076A8DED097A0A920B9203
:10F070000C920DF1180EBEE80F002E460FC69EE84A
:10F08000070094F816C486E807004FF00508FE2034
:10F09000C8214FF01E0E1C230CF1010284F84E0013
:10F0A00084F8521084F80E8484F853E084F84F30CA
:10F0B000291F84F850C04FF6FF7084F8162401E031
:10F0C00011F8013B434083EA0313DBB21A0982EAD9
:10F0D000102242EA03228D4282EAC300F0D1294D78
:10F0E000A4F84C0005F11C0115F8013B434083EAEC
:10F0F0000313DBB21A0982EA102282EA032282EAAF
:10F10000C3031BB298B28D42A4F84C00ECD183F03B
:10F11000270383EA0313DBB21A0982EA102282EA88
:10F12000032282EAC3031BB29AB24FEA122C5FFA9F
:10F1300083FEDFF86080A4F84C2084F871C084F866
:10F1400070E004F14E0604F16E0930687168B2682F
:10F15000F36845460FC510364E45A846F5D10C4D0F
:10F160003388A8F8003005F1240684F862E484F8B6
:10F1700063C415F8011FD4F8FC03F9F797FEAE42FB
:10F18000F7D10CE0FC2300200B28002088C3E43AD0
:10F19000E7270020E8270020731E84F80E3494F837
:10F1A0000F340193002B40F08481D24B1B68052261
:10F1B0009D0684F80F2400F18382DFEDCF7AB0EE54
:10F1C000677AB4F95A35B4F9B011CC4DCC48CDEDCD
:10F1D000077AB3F5FA6FA8BF4FF4FA63B3F57A7FF5
:10F1E000B8BF4FF47A73A3F57A72642303FB02F37A
:10F1F00085FB032580FB0120DB17CA170026C3EB24
:10F20000A51306A9C2EBA0028DED087AADF82A304D
:10F21000ADF82820069609960D4600910FCDDFF82F
:10F22000E4E22E6894F816C484F850C075460FC501
:10F230004A212E60AEF1040800250CF10100FE22E7
:10F24000142384F85310C82184F85150464684F89A
:10F25000160484F84E2084F84F3084F852104FF68C
:10F26000FF7501E016F8013B6B4083EA0313DBB244
:10F270001A0982EA152242EA0322B64582EAC30548
:10F28000F0D1A049A4F84C5001F1140011F8013B51
:10F290006B4083EA0313DBB21A0982EA152282EA81
:10F2A000032282EAC3031BB29DB28142A4F84C50F0
:10F2B000ECD183F0140383EA0313DBB21A0982EA68
:10F2C000152282EA032282EAC30325461BB21FFAF3
:10F2D00083FC55F84E0FDFF838E2A4F84CC0DBB2DF
:10F2E0004FEA1C2A84F869A084F8683069680293A0
:10F2F000AA68EB68AEE80F00286969692B8BAEE855
:10F30000030004F23F45AEF800309DF8083084F861
:10F310005BA4A94684F85A3404F25B4A19F8011F29
:10F32000D4F8FC03F9F7C2FDCA45F7D1764A94F840
:10F3300078351278013BDBB212F0010214BFC02114
:10F340004021172B9BBF71481B184FF0000E93F8FC
:10F350002CE0B4F89433980706BF0120019041F0E7
:10F36000100113F4027F019818BF022013F0100F50
:10F3700018BF062013F0200F0CBF03461023019383
:10F38000002A40F0B2840322019B069303234FF02E
:10F39000000C8DF82030009B8DF81CE08DF81E10BD
:10F3A0008DF81F208DF81DC093E80700DFF854E1A9
:10F3B00084F853C0AEE8030094F816148EF80020C9
:10F3C00001F1010A4FF0FE090923C82084F851C059
:10F3D00084F8501084F816A484F84E9084F84F30C6
:10F3E00084F852004FF6FF7E01E018F8013B83EAF3
:10F3F0000E0383EA0313DBB21A0982EA1E2242EAF1
:10F400000322464582EAC30EEFD13E49A4F84CE000
:10F4100001F1090011F8013B83EA0E0383EA0313AB
:10F42000DBB21A0982EA1E2282EA032282EAC303BD
:10F430001BB21FFA83FE8142A4F84CE0EAD183F0AC
:10F44000320383EA0313DBB21A0982EA1E2282EA3C
:10F45000032282EAC303A6461BB21FFA83FC5EF8AE
:10F460004E0F2B4EA4F84CC0DBB24FEA1C2884F898
:10F470005D3084F85E80DEF80410DEF8082007C6F0
:10F48000BEF80C109EF80E203180B27004F58A662A
:10F4900084F8508484F84F3415F8011FD4F8FC0325
:10F4A000F9F704FDAE42F7D108E0013B84F80A34D5
:10F4B000AFE5019B03F1FF3984F80F94C4F80074A1
:10F4C000FEF728BB2D2384F83332FEF7E3BF94F810
:10F4D0001432D9F80020C4F81022013B012B3EF66B
:10F4E00002AF1022022384F8E62184F8E831FEF707
:10F4F000FABE00BFB084002000000000D34D6210AF
:10F5000067666666FC2300204C65002098DF0308D0
:10F51000E8270020DEF80000000600F1CC839CF80C
:10F520000C0000283FF440A894F89613032900F239
:10F53000B485DFE811F05F01550146012F01B4F8F1
:10F54000E43300220133A4F8E43384F8DC23FEF72B
:10F55000D0BA84F88F03FFF76DBA0A4608460D4605
:10F5600000918C4688468A460B46B4F8D013A64EC6
:10F57000CDF818E0C1EB012186FB016E8E44C9175E
:10F58000C1EB6E21BDF80060ADF81E804FF0000E9B
:10F59000ADF820C0ADF82260ADF824508DF82CE015
:10F5A000ADF81CA0ADF82600ADF82820ADF82A3043
:10F5B0008DF82D1006AD0FCD944E84F851E0B6466F
:10F5C000AEE80F0095E8030094F816C44EF8040B5B
:10F5D00023250CF10108FE201623C822AEF80010E6
:10F5E00084F8535084F850C084F8168484F84E0090
:10F5F00084F84F30311F84F852204FF6FF7501E038
:10F6000011F8013B6B4083EA0313DBB21A0982EA6B
:10F61000152242EA03228E4282EAC305F0D17B49D9
:10F62000A4F84C5001F1160011F8013B6B4083EA3D
:10F630000313DBB21A0982EA152282EA032282EA64
:10F64000C3031BB29DB28142A4F84C50ECD183F0AD
:10F65000F40383EA0313DBB24FEA131E8EEA152E7E
:10F660008EEA032E8EEAC30E25460FFA8EFE1FFA8F
:10F670008EF855F84E0F664EA4F84C805FFA8EFE59
:10F680004FEA182C84F86AE084F86BC06968AA68AD
:10F69000EB680FC628696969AA6904F23F4507C685
:10F6A00004F25D4684F85DC484F85CE415F8011F3B
:10F6B000D4F8FC03F9F7FAFBAE42F7D1FFF782BAB0
:10F6C000B4F8D631DFED536A07EE903AB4F8D03192
:10F6D000F8EEE77A07EE103A67EEA67AB8EE477AC8
:10F6E0006FE5D4F8CC214C4982EAE273A3EBE273D4
:10F6F00003EB5303A1FB0331C908002AACBF41F05F
:10F70000004141F04041FFF784B894F8C431042B24
:10F710008CBF03250225FEF744BC012338682B70FB
:10F72000F9F7B8FB05463868F9F7B4FB6D067EF4C7
:10F730005AAA8A2800F09F848E287EF454AA94F84E
:10F740004832002B7EF481A9344BC4F850322D236B
:10F7500084F85432FEF751BA94F8C431042B8CBFAC
:10F7600003260226FFF741BA2D4B94F8B9211B88D6
:10F7700003EB830303EB83039D00ADB2002A40F04B
:10F78000B1844FF0FF330FFA83FA0AF0E3FB40B283
:10F79000FEF7D8BCD4F89C2353799079D17903F142
:10F7A000407303EB002303EB0141002384F89633FD
:10F7B0004FF482602AF0A6F9002384F86132FEF744
:10F7C0007FB9D4F89823137A507992781B0403EB0D
:10F7D000002313444A1C84F8962303EB0161E7E7F6
:10F7E000D4F89823D379107952781B0403EB0023C3
:10F7F0001344EFE7D4F898239379D07812781B0458
:10F8000003EB00231344E5E703082080FC230020DA
:10F81000E82700200AD7233C1F85EB518C250020C8
:10F8200088CF002002202AF0FFF9FF2029F0E8FF0E
:10F830000378FF2B00F0D58390F90100C517EDB2D6
:10F84000C0B22AF0C7F928462AF0C4F903202AF0EA
:10F85000EBF9FF2029F0D4FF0378FF2B00F057834A
:10F86000B0F90850E8B2C5F307252AF0B3F92846E5
:10F870002AF0B0F994F8B831002B40F09382D24BC3
:10F880001B68980640F1398294F8C231990700F15B
:10F890006D8300252F4601202AF0C6F938462AF04C
:10F8A00099F928462AF096F909202AF0BDF9002096
:10F8B0002AF090F900202AF08DF9B4F8DA2194F8B2
:10F8C000C451B2F5967F0AD994F8643103F00F035E
:10F8D000072B04D842F20F75954228BF1546BB4F3F
:10F8E00005202AF0A1F93B7A002B00F0BD83A5F199
:10F8F000200307EE903A9FEDB67AF8EEE77AF6EE3F
:10F90000006A67EE877ABEEE007AF5EEC07AF1EE15
:10F9100010FA58BFB0EE667A77EE877AFDEEE77A96
:10F92000CDED007ABDF90050E8B22AF053F9C5F3E5
:10F9300007202AF04FF994F8C2210023049305937D
:10F94000930700F1BD8294F8DC31012B00F0B882FE
:10F95000B7F90030DFED9F6A07EE103AB7F90230D1
:10F9600007EE903AB8EEC77AF8EEE77A27EE267AF5
:10F9700067EEA67ABDEEC77AFDEEE77A06A88DEDB2
:10F98000067ACDED077A2AF061F95E213068F9F741
:10F990008DFA94F86431FEF717BA8F4B0793A3F1F1
:10F9A000240600222121A3F1210703F8242CB170A1
:10F9B000727006970FF0D6FB884B8949B4F89423F0
:10F9C000002814BF99468946530500F1B481D00739
:10F9D00000F19882910740F10683DFF828924FF0FA
:10F9E0000308424649467F482BF0DCFD07EB08033D
:10F9F0000EA87D4A013340F8203D9B1A002207F8EB
:10FA0000082073702AF07AF9FEF736BA724B7749FC
:10FA100007930EAEA3F1210046F8200D0A2003F84B
:10FA2000230C0027082003F8220C03F8247C30461E
:10FA30000988FAF701FC6E4B6E491B6881FB0321B4
:10FA4000DB17C3EBA101304689B2FAF7F5FB0AF0E8
:10FA500081FA069BB4F8BA21591C06911F70069BC7
:10FA6000110A5F1C06971970069B591C06911A70A3
:10FA7000069B5A1C0692187030462AF03FF9FEF792
:10FA8000F8B9B4F9AE319FED5C8A534A079207EE9C
:10FA9000903AF8EEE77A0EAE67EE887AA2F121018D
:10FAA000FDEEE77A46F8201DA2F124030020CDEDFB
:10FAB000007A02F8240C1E2208209A70BDF800106B
:10FAC00058703046FAF7B8FBB4F9AC3107EE903A0B
:10FAD000F8EEE77A304667EE887AFDEEE77ACDED0C
:10FAE000007ABDF80010FAF7A7FBB4F9B03107EEC1
:10FAF000903AF8EEE77A304667EE887AFDEEE77ADC
:10FB0000CDED007ABDF80010FAF796FB30462AF0EA
:10FB1000F5F8FEF7ABB9C4F84CB22E70FEF763B837
:10FB200094F8EA03C0B10138C0B2344D0130284422
:10FB3000002215F8013B534083EA0313DBB2120A9B
:10FB4000D90042EA0322A84281EA131382EA03029F
:10FB5000EFD1002A7EF4AAAA244B294D244AD4F8D6
:10FB6000F4031B881168EB619268036BE962EA6435
:10FB70000021B4F8E423EE66E963EA65002B00F0A7
:10FB80009D825B68816C8B423BBFC2685B1A5B1ACB
:10FB90009B18002B7DF4A8AF036802219B6998474E
:10FBA000042394F8EB0385F8743016F09DF90323D1
:10FBB00084F8DC33FDF798BF02213868F9F75EF965
:10FBC00094F85432FDF752BFB084002078CF002063
:10FBD000E4380E3F0050C34718D000206C0C0408D6
:10FBE000640C0408F7CF0020F5CF002088CF002058
:10FBF0008CCF00206766666658A08B419027002056
:10FC0000200000207C0C0408A3785E09012E40F03F
:10FC1000648103F00F0E13F0100300F07B81C64ADD
:10FC2000E3782779A4F88603D11887EA0300C4F89B
:10FC30007C23134684F86662C4F88013073A84F87C
:10FC40008C03A4F8847394F88C03BC4F0CE012F876
:10FC5000011BC4F87C63BA4280EA0100197007D224
:10FC6000D4F88013D4F87C33994203F10106EED125
:10FC7000BA4284F88C0300F03982127894F88C33FD
:10FC80009A4200F0C781AE4BC4F8683201330122BA
:10FC9000B4F88413C4F86C3200204FF6F67384F87D
:10FCA0006602A4F8701284F8782284F87823A4F805
:10FCB0007232FEF770BC102300250422184606A9F4
:10FCC0008DF818308DF819208DF81A508DF81B50CA
:10FCD0008DF81C508DF81D5029F0F8FE84F8615203
:10FCE000FDF7EEBE3422FEF71FBF94F8AF33002BB2
:10FCF0000CBF04220522FFF747BB924B93E8030099
:10FD000006AB83E80300184629F0A0FF3DE610206B
:10FD100029F08AFF284629F05DFF284629F05AFF7E
:10FD2000212029F081FF284629F054FF284629F098
:10FD300051FFFEF723B84FF00308DFF8289250E692
:10FD4000B4F97212D4F86C72501C02F00F0242F037
:10FD500010020029B8BF42F0200284F88E0394F804
:10FD600070028DF81820BA1B5040C0B28DF81920CF
:10FD700084F88F030DF11A02FEF73FBE724B19880B
:10FD8000FEF7B7BD714B6420B3F900A0FEF7DAB9F6
:10FD90001A4618461D4600939C46FFF7E6BB2422F0
:10FDA000FEF7C2BE6A4F97F80080B8F1000F3FF42B
:10FDB00066ADDFF894A1B4F8C051BAF800302D0157
:10FDC0006422ADB202FB03834FEA4802B3FBF2F3B5
:10FDD00045EA0325ADB2C3F303231D43062029F0F2
:10FDE00023FFE8B229F0F6FE280A29F0F3FEB4F862
:10FDF000C0315849BAF8005001339BB293FBF8F276
:10FE000008FB12334A7AA4F8C031012A00F0878136
:10FE10006E23514A497B03FB05F382FB0302DB1788
:10FE2000C3EBA203002940F075814C4D9FB2A5FBA6
:10FE300007356D093A201FFA85F829F0F5FE5FFABB
:10FE400088F029F0C7FE4FEA182029F0C3FE3B20B6
:10FE500029F0EAFE642303FB15739BB24048053387
:10FE600080FB0320DB17C3EBA000C0B229F0B2FE79
:10FE7000002029F0AFFE354F394D282029F0D4FE5F
:10FE80003B6885FB0325DB17C3EBA505E8B229F02A
:10FE9000A1FEC5F3072029F09DFE042029F0C4FE31
:10FEA000B4F8BA31002B40F01481BD6885F3100519
:10FEB000E8B229F08FFEC5F3072029F08BFEDEE4BF
:10FEC0000121D4F8C821D4F8CC3184F8DC1104A87D
:10FED0000492059329F0BAFE57E5194B84F866029F
:10FEE0005E1C4FF6F6710122A4F8700284F87802C5
:10FEF000C4F86832C4F86C62A4F8721284F87823EB
:10FF0000FEF749BB4FF00408DFF85C9069E5002577
:10FF10002846AAE494F86622002A3EF43CAB94F802
:10FF20008D23013202F00F02724500F0C18084F887
:10FF30006632FEF730BB00BFB4230020B0230020A0
:10FF40002026002098DF030888CF00208CCF0020D7
:10FF5000CFCF002078CF0020310CC3301F85EB516C
:10FF600067666666700C0408740C0408112029F09A
:10FF70005BFEB4F8D621784D4FF4F36707FB02F22D
:10FF800085FB0235D217C2EB6535E8B229F022FEB7
:10FF9000C5F3072029F01EFE192029F045FEB4F80C
:10FFA000D6316E4A07FB03F382FB0301DB17C3EB79
:10FFB000611382FB0321DA17C2EB6112642101FB9A
:10FFC0001233D8B229F006FE002029F003FE94F87F
:10FFD000C231B4F8D0519A077FF55BACEFB22D0A6D
:10FFE00059E428462DE448462AF00CFD8046F8E402
:10FFF0001022FEF799BD0099322029F067FDFEF727
:020000040801F1
:1000000029BD06AB00930DF11E05FEF713BD20229E
:10001000FEF78ABD524BD4F87C23C4F88023002716
:1000200003F55B7203F51B76C4F86C2203F51771B8
:1000300003F55C703A46C4F86862C4F87C3384F80F
:100040006672A4F87072A4F87272FBF729FA013094
:1000500058D0D4F86832C4F86C320123C4F868620E
:1000600084F87833FEF797BAE8B229F0B3FD280A8E
:1000700029F0B0FD5FE43B4B1B6898067DF5B3ADFE
:1000800094F84832002B7DF4E0AC374BC4F8503282
:100090002D2384F85432FDF7B0BD4B1CDBB2042B8A
:1000A00084F896334FEA01613FF47FABFFF780BBE2
:1000B000D4F88013D4F87C332C4AC4E5C269036AAF
:1000C0009A423CBFC1685218D31A62E50822FEF773
:1000D0002BBD09F03FFF29F07DFD002029F07AFDBE
:1000E000FFF7CDBB224B1B68FFF74DBB84F88DE3B8
:1000F000FEF751BA1A4618461D4600939C4698468C
:10010000FFF733BAD4F868320222591CC4F86812D7
:100110001A709EE79BB23A7893FBF2F385E639209A
:1001200029F082FDE8B229F055FD280A29F052FD98
:10013000A1E61A46FFF719BA1A461846FFF715BA8C
:100140001A4618461D46FFF710BA1A4618461D46AD
:100150000093FFF70ABA00BF89B5F8141F85EB5169
:10016000B4230020B0840020C0250020AB23002051
:100170008CCF002003680A7A591C01601A707047FE
:1001800038B50B4C23688BB15A68821A002A054691
:1001900004DA0CE05A68AA1A002A07DB9A6822607F
:1001A00018461A6890472368002BF3D138BD38BD34
:1001B0002C4500200B4B002210B4027203F1900476
:1001C000012102E0072A09DC9979890702D519790A
:1001D000815401329C4203F11803F3D15DF8044BC2
:1001E000704700BF4808040829230370704700BF08
:1001F000012310B431213224332244704171C27082
:100200000370037183705DF8044B70472DE9F04172
:100210000B78047BDB43DEB200F1100200F13803FF
:1002200042F8044F9342FBD1DFF89CC000F160011B
:10023000002243F8042F8B42FBD14FF0140E05210E
:10024000002546FA01F303F00103002B1D4414BFFF
:100250004FF019084FF00A0811F0010FEDB214BF6A
:100260002746002700220EEB02039BB200EB83031C
:10027000013242455F61F6D1013A92B20132013951
:100280000EEB02034A1C9BB201D09E46D9E715F043
:10029000010F14BF19250A2500215A1892B200EB4C
:1002A00082020131A9425461F7D10B449BB21A1D5D
:1002B00000EB8202013300219BB25160ACF80030A8
:1002C0000361BDE8F08100BF8C290020254B5B88CD
:1002D0000B332DE9F04F8A4601F1060B1FFA83F923
:1002E0004FF00108002100271AF801EB3E464C466A
:1002F0000122A4F10B039BB207E001339BB2B0F8DB
:100300000CC0C5F814C09C420AD000EB8305002A3B
:10031000F3D100EB830501339BB29C426A61F4D1B7
:10032000231D00EB83030136092FF6B259600CD070
:10033000092E14D008FA07F313EA0E0F14BF012296
:1003400000220C34A4B20137D3E709F17809DA4569
:100350001FFA89F9C7D1034B5980BDE8F08F0022FD
:10036000EFE700BF8C2900202DE9F047DFF85C8023
:10037000B8F8043004338A461FFA83FC01F10909F6
:100380004FF0010E1AF8017B64460026231F0EFA77
:1003900006F29BB23A40BAB1818900EB8305013382
:1003A0009BB29C426961F6D101360434082EA4B296
:1003B000ECD10CF1200CCA451FFA8CFCE2D10023D1
:1003C000A8F80430BDE8F0871146E6E78C29002044
:1003D00010B4037B01681F2B09D9203B20224C68F5
:1003E00002FA03F31C4214D15DF8044B704720223B
:1003F0000C6802FA03F31C42F6D00C4A4068002451
:10040000147002685DF8044B22F0010202608B60F8
:100410007047064A40680024147002685DF8044B77
:1004200022F001020260CB60704700BFA87000207C
:1004300008B512F011FBFAF72DFD00BF70B54E683C
:10044000054630462AF0DEFA314604460246286860
:100450002BF0A8F82A68131901333B212B601155A2
:1004600070BD00BF024A034B1278197828F000BC17
:10047000A0230020A1230020038A2DE9F0478589CD
:10048000ADB21D4029D00F4606464FF000484FF050
:100490000009B5FA85F328FA03F2D24391B21B3B67
:1004A00015403182042B16D8DFE803F031292119D9
:1004B00003007B6A002B32D003F1FF3A1FFA8AFA5D
:1004C000C7F824903C6A34B12368204651469847C7
:1004D0006468002CF8D1002DDBD1BDE8F0873868C6
:1004E000716B036889B29847002DD2D1F5E778681F
:1004F000B16B036889B29847002DCAD1EDE7B8689F
:10050000F16B036889B29847002DC2D1E5E7F8681E
:10051000316C036889B29847002DBAD1DDE7F36AE0
:100520001FFA83FACEE700BF38282DE9F04700F024
:1005300097810C462ED9802800F0F68074D8522876
:1005400000F0898040F24C81542800F0B2816E287E
:1005500040F0AC81B04B0A681B88B04DFF2BA8BFA0
:10056000FF23511C21601370A96881F310012046FC
:1005700089B2F9F787FEAA4B20461988F9F782FE5F
:10058000296801F30F01204689B2F9F77BFE0120AB
:10059000BDE8F087042800F04E8240F2EE8020286B
:1005A00000F0A18040F22481242800F0D381282883
:1005B00040F07C810B68DFF89C829A4E591C022225
:1005C00021601A70236806275A1C22601F70236856
:1005D0000A22591C21601A70236801255A192260C9
:1005E0001D70B8F800102046F9F74CFEB8F802105C
:1005F0002046F9F747FE23685A1922601F702368C6
:100600005022591921601A7023680022591921605B
:100610001A7031882046F9F735FE20467188F9F7BF
:1006200031FE2846BDE8F08782282FD0C0F0AC818B
:10063000A02800F09781FE2840F038817A4D05F11E
:10064000080635F8021B2046F9F71CFEB542F8D122
:100650000120BDE8F0870A68744E531C0321236013
:1006600006F10C0711703346062001212268551C43
:100670002560117022689F4202F101012160107013
:1006800000F0EA819979D8790633EFE70B68684A78
:10069000624D1178674A581C20601970D188204635
:1006A000F9F7F0FD5C4B22681B88FF2B02F101017A
:1006B000A8BFFF2321601370A96881F310012046B1
:1006C00089B2F9F7DFFD296801F30F01204689B2ED
:1006D000F9F7D8FD2368584A591C127821601A701E
:1006E0000120BDE8F0870B68524D591C6A782160E3
:1006F0001A7023682A78591C21601A702368AA7816
:10070000591C21601A70E9882046F9F7BBFD23685F
:100710002A79591C21601A7023686A79591C216052
:100720001A700120BDE8F087DFF82C81434F444E5A
:10073000DFF828A108F10D090A2515E0322D34D083
:10074000A5F13C00C0B2132835D900232268511C02
:10075000216015702268C84502F101012160137003
:100760003FF476AF18F8015B0A2DE7D1BAF80030F4
:10077000FF2BA8BFFF23DBB2E8E7022800F09C8133
:1007800000F28981012840F091800B680022591CF9
:1007900021601A7023685A1C226018702368242272
:1007A000591C21601A70BDE8F0873388FF2BA8BF61
:1007B000FF23DBB2CAE729F023F80028C5D003786D
:1007C0000A2B00F28181B0F9023087FB0312DB179C
:1007D000C3EBA2039BB2FF2BA8BFFF23DBB2B5E79D
:1007E000442863D1002A3FF433AF164B13602FE740
:1007F00005285BD120460B221349F9F7FBFC204664
:1008000008221249F9F7F6FC204607221049F9F7A9
:10081000F1FC0120BDE8F08788CF00208CCF0020BC
:1008200078270020002D0020E4CE0020E4E003081B
:10083000CFCF00205C250020BC25002067666666BF
:10084000182D002031040108EC0C0408F80C0408F1
:10085000040D040880410020FDDF0308482D00201E
:100860000B689A4A01205C1C0C6018700B68052408
:100870001D180D601C700B680A241D180D601C707B
:100880000B6800241D180D601C700B6814781D186F
:100890000D601C700B6854781D180D601C700B687F
:1008A00092781C180C601A70BDE8F0870020BDE833
:1008B000F0870B68864A874F581C112120601970F9
:1008C00023681278591C21601A70236897F85C20FD
:1008D000591C21601A70236897F85620591C216012
:1008E0001A70B7F858102046F9F7CCFC00212046C2
:1008F000F9F7C8FCB7F85A102046F9F7C3FCBD1E3B
:1009000007F1480635F8021F2046F9F7BBFCAE4256
:10091000F8D12268704B0C21501C20605D181170BA
:10092000226813F8011F501C9D4220601170F7D1FE
:1009300023680222591C21601A70B7F85E10204605
:10094000F9F7A0FC2046B7F86010F9F79BFC0120EE
:10095000BDE8F087614B08461968F9F77BFC012078
:10096000BDE8F0875E4B08461968F9F773FC5D4BEC
:1009700020461968F9F76EFC5B4B20461968F9F7B9
:1009800069FC0120BDE8F087DFF87891574F09F145
:100990000E064FF00A081DE0B8F1500F32D0B8F142
:1009A000320F31D0A8F13C00C0B213282FD9002556
:1009B000294623685A1C2260204683F80080F9F7F4
:1009C00061FC29462046F9F75DFC4E453FF440AEF8
:1009D00019F8018BB8F10A0FDED1454B9D681968F3
:1009E00005EB85054FF6FF736D009D42A8BF1D46C0
:1009F0009942A8BF194625EAE57521EAE171ADB231
:100A000089B2D6E73B4BE9E797E82200E8E728F010
:100A1000F7FE0028CBD003780A2BC8D8B0F90430F1
:100A2000B0F9061003EB830383F3500521EAE1716B
:100A3000ADB289B2BDE702462F492046F9F7DAFB8D
:100A400020460021F9F71EFC23680222591C216070
:100A50001A700120BDE8F087284B21681A78481CDD
:100A600020600A70002A3FF4F3AD013AD2B202EBE3
:100A7000420206EB42025278002A3FF4E9AD01320D
:100A8000D5180133226813F8011F501C9D422060C5
:100A90001170F7D1DCE50B680222591C21601A7035
:100AA000236801201A182260187023680022191880
:100AB00021601A70BDE8F087084604221049F9F752
:100AC00099FB0120BDE8F087002387E6B34F0020A3
:100AD0002C7C0020B0C70020F9C70020F85000206F
:100AE000107AFF1F147AFF1F187AFF1F102D0020A5
:100AF000C42C0020042D0020E40C0408AC7000205D
:100B0000DC0C0408EDDF0308F0B5464B1A6883B02F
:100B10000123500200935CBF03F180530093D10086
:100B2000414909685CBF43F0100300938F0748BF39
:100B300043F0C6033D4948BF0093160648BF43F43F
:100B40004063097848BF0093D40548BF43F0006371
:100B500001F0EF0048BF009308286D4655D00E29DC
:100B600053D0D0033248009B00784CBF43F420435D
:100B700043F40053D7044CBF43F0C84343F08843C9
:100B800000280CBF07200F20960648BF43F480734F
:100B9000540748BF43F4003343F400245205009443
:100BA00002D5244A1279A2BB182936D00190002719
:100BB000012639462846FCB2F9F7F6FE60B11E4B15
:100BC000002203F5D87103E08B420FD013F80C2CF0
:100BD000944203F10C03F7D10137242FE9D195E8B2
:100BE0000300164B83E8030003B0F0BD7A0904F05C
:100BF0001F0455F8223006FA04F4013723EA0404EE
:100C0000242F45F82240D4D1E9E743F480530093E0
:100C1000A7E743F4C0130093C6E7009B43F060735B
:100C20000093C3E788C00020B08400202029002062
:100C3000ACBB002078CF0020F0DD03089823002013
:100C40002DE9F84F4E014FF0000B174D81469046AD
:100C500006F120075C46594628465FFA8BFAF9F7F9
:100C6000A3FEC0B1A64215D8A74213D900200F4A4F
:100C7000014604E00131242914D012F80C0C50452F
:100C800002F10C02F6D10A4B01EB410103EB8101A9
:100C90004846C04701340BF1010BBBF1240FDAD1F8
:100CA000BDE8F88F0021F3E798230020F0DD03086A
:100CB000E4DD030800210A4A0B4604E00133242B3B
:100CC0000BD012F80C1C884202F10C02F6D1054838
:100CD00003EB430300EB830070470020704700BF25
:100CE000F8DD0308E4DD030800210A4A0B4604E0AE
:100CF0000133242B0BD012F80C1C884202F10C0299
:100D0000F6D1054803EB430300EB83007047002056
:100D1000704700BFF0DD0308E4DD03081C4C08B594
:100D200001210220F8F7DEFC237803F00502052AF2
:100D300029D003F00903092B08D000210120F8F77E
:100D4000D1FC00210846F8F7CDFCFEE7114A124B12
:100D500011681A680B68114C23F001030B601388AB
:100D6000206823F001031B041B0C138018B12922F7
:100D700000238271C37103224A21F8F73DFA2068EB
:100D8000F8F79CFCD9E711F017FF2378D1E700BFF3
:100D9000883F0020B82C0020BC2C00208C2D002087
:100DA000022828BF022010B4084C094B207000EB29
:100DB000C00200EB820207495DF8044B013003EBEF
:100DC0004203C0B20B6024F0B1BF00BF006300203B
:100DD000C44F00204027002008B514F0C9FCF8F7E4
:100DE000EDFFBDE8084014F0ABBC00BF38B5384B90
:100DF0005A899989914224BF00225A81198ADA8935
:100E0000914224BF0022DA81DA788AB1072A0FD012
:100E1000304C3148A27801210025062A01709970D2
:100E2000DD714CD92379DFED2D6A002B36D138BD29
:100E3000DA799B78284807EE103A002A44D0DFED93
:100E4000276A0178234CB8EEC77A07EE901AA27889
:100E5000F8EEE77A27EE267A062A67EE877A2BD80D
:100E60001F4B03EB8203D3ED086AF4EEE76AF1EE61
:100E700010FA10DDC6EE877AFDEEE77A17EE903AAB
:100E8000102BA8BF1023012BB8BF0123DBB28B426C
:100E900028BF0B4603702379002BC8D0013A032AE0
:100EA000C5D8B7EE000A80EE260A2AF085FD238811
:100EB000984238BF208038BDDFED086AD5E7DFED06
:100EC000097AB0EE677ACBE7DFED076AB9E700BFD2
:100ED000647C002084BB0020844100206F12033812
:100EE000ECDF03086F12833A6F12033938B50D4CEB
:100EF0000D4DAC4206D2616820461434F8F7E2FE8C
:100F0000AC42F8D3094B0A4C0A48186000252570FA
:100F100021F04CFE084B094A65701A60BDE8384064
:100F20001CF07EBC88010008D40500084027002082
:100F300000630020C44F002044270020C050002040
:100F400008B5FFF7D3FF14F013FCF8F737FFBDE83F
:100F5000084014F0F5BB00BFF0B50C2934D8DFE829
:100F600001F0893333335E333333343333330700A3
:100F7000048C9689B2F802E01788734D24F48054EB
:100F80002404240C0484038C8488818B23F4005370
:100F900021F4E6411B0409041B0C46EA0E06090C69
:100FA00043EA063341EA0721A8429BB2A4B289B2C0
:100FB00000F09E8005F58065A84200F09980926857
:100FC0008480818302640384F0BD048C9589B2F827
:100FD00002C0B2F800E05C4F24F480742404240CB6
:100FE0000484038C8688818B23F400731B0421F016
:100FF00073011B0C45EA0C04090443EA0423090CA1
:10100000B8429BB2B6B241EA0E015CD04F4CA0424E
:1010100059D0926886808183C2630384F0BD048CBA
:101020009589B2F802C0B2F800E0474E24F01004EF
:101030002404240C0484038C8788018B23F0200370
:1010400021F4E6411B0409041B0C45EA0C04090CBD
:1010500043EA041341EA0E21B0429BB2BFB289B207
:101060005DD03A4CA0425AD0926887800183826357
:101070000384F0BD048C9789B2F802E01688324DE3
:1010800024F001042404240C0484038C8488018B40
:1010900023F002031B0421F073011B0C47EA0E0727
:1010A00009043B43090CA8429BB2A4B241EA0601E1
:1010B00025D005F58065A84221D0926884800183FF
:1010C00042630384F0BDD589148A578A23F40063F0
:1010D00043EA05254FF6FF332B40958826F440560A
:1010E0003C4343EA052346EA04169BB2B6B290E7B6
:1010F000158A24F4804444EA8514A4B25FE7D689B3
:10110000158A578A23F00803334324F440749688E1
:101110003D4323F004032C433343A4B2CDE7D489E9
:10112000158A568A23F0800343EA04134FF6BF74EE
:101130001C40938827F44067354344EA031347EA89
:1011400085079BB2BFB28FE7000001400004014059
:101150002DE9F84FF02200219248934CDFF870926D
:10116000924D934E934FDFF86C822CF032FD9248F3
:101170009249DFF864E2DFF864C200221359834227
:1011800000F0F880B3F1804F00F0F680AB4200F041
:10119000F580B34200F0F480BB4200F0F380734569
:1011A00000F0F280634500F0F180434500F0F080EC
:1011B000DFF82CA2534500F0ED800AF5806A534514
:1011C00000F0EA800AF5806A534500F0E780AAF54E
:1011D000983A534500F0E4800AF5806A534500F0E0
:1011E0009B800AF5806A534508BF0D2300F0958067
:1011F0001832A82AC2D1DFF8B081714E08F1A807D1
:101200004FF0030A4FF0020998F804301C09013C22
:10121000032C03F00F0378D86A4A32F8140040FA1E
:1012200003F2D20771D5012505FA03F3013B1840FB
:101230002AF0B2F8644B1B5D184416EBC00264D070
:1012400056F83030614C98F8081003F13F4000F533
:101250007E00800A205C00F01F044009032805FA84
:1012600004F500F08180042878D0022804D1534886
:10127000406C054351484564B2F804E0BEFA8EF272
:10128000C2F11F0292B2D00803EB800002F0070205
:10129000046A92000F25954024EA05040462046A5A
:1012A00001FA02F22243002502624FF0010C2A46A5
:1012B00003E0102A05F1020527D00CFA02F030EA0B
:1012C0000E0102F10102F4D11C680AFA05F1C943CA
:1012D0000C401C60D3F800B009FA05F444EA0B0492
:1012E0001C609C680C409C609C689C605C6824EA64
:1012F0000000586058685860D8680140D960D968C3
:10130000D960102A05F10205D7D108F11808474520
:101310007FF47AAFBDE8F88F0C2309EBC3034FF0DD
:10132000010A93F8403003F01F0B5B09032B0AFA04
:101330000BFA09D0042B0CD0022B7FF459AF4B6C65
:101340004AEA03034B6453E70B6C4AEA03030B645A
:101350004EE70B6B4AEA03030B6349E71748006B40
:1013600005431648056387E71448006C0543134896
:10137000056481E70023D0E70123CEE70223CCE711
:101380000323CAE70423C8E70523C6E70623C4E707
:101390000723C2E70823C0E70923BEE70A23BCE707
:1013A0000B23BAE72C64002048080408000400401E
:1013B00000080040000C00400000014000380240DE
:1013C00040C50020F4080408F008040820080408B8
:1013D000ECDF03080004014000100040001400404E
:1013E0000040014001490248FFF746B8F46400207C
:1013F0000048014001490248FFF73EB8CC64002094
:101400000004014001490248FFF736B8CC640020CF
:101410000004014001490248FFF72EB8A4640020EF
:101420000008004001490248FFF726B87C6400200C
:101430000004004002494FF08040FFF71DB800BF94
:101440005464002001490248FFF716B82C640020BC
:101450000000014001490248FFF70EB82C6400204B
:1014600000000140F0B504684B4DA30AAB4276D0B2
:1014700009D94A4DAB425CD01135AB4273D0123D15
:10148000AB425AD0F0BDB3F5801F64D0013DAB42F2
:1014900057D14FF0700E02264779B0004FEA970CF3
:1014A000002964D063460227A5899F4083190CEB6D
:1014B00043032F4303F1040C394DBFB245F8231009
:1014C00045F82C20A781EFF31181502282F3128876
:1014D000821905EBC2021369002B33D01362043367
:1014E000821905EBC202576917B11F6053690433B3
:1014F000821905EBC202976917B11F609369043323
:10150000821905EBC202D76917B11F60D369043392
:101510000027CAB21F6082F31188304405EBC00077
:10152000036A93B9A38923F001031B041B0CA38155
:10153000F0BD4FF0C00E0426AEE74FF0200E00269F
:10154000AAE7F0BD05EB0E03CAE7A3899BB243F0FF
:101550000103A381F0BD4FF0480E01269CE74FF038
:10156000980E032698E74FF0E80E052694E702232D
:10157000BF0803FA07F7A389094D9BB223EA0703C3
:1015800087190CEB470CA3810CF1040345F82C10D0
:1015900045F8232097E700BF02001000410010002B
:1015A0002C64002010B5036883480139834282B05F
:1015B00089B200F0CB80A0F58060834200F0C68045
:1015C00000F58040834200F0B88000F580608342DF
:1015D00000F0B38000F58060834200F0AE80774C6D
:1015E000188824686408B4FBF2F4013CA4B282B207
:1015F000B3F1804F0AD07248834207D000F5806073
:10160000834203D000F58060834202D122F0700251
:1016100092B26C48834200F0A28000F58060834261
:1016200000F0A78022F4407200F56C4092B2834231
:101630001A80D9621C854FD05F4A93424CD0012258
:101640009A821A8892B242F001021A80B3F1804F56
:1016500000F099805A4A934200F0978002F5806228
:10166000934200F0948002F58062934200F09180F2
:1016700002F58062934200F08E8002F58062934210
:1016800000F08B8002F57042934200F0888002F5F2
:101690007052934200F0858002F58062934200F020
:1016A000828002F5806293427FD0A2F59832934205
:1016B0007DD002F5806293427BD002F58062934236
:1016C00008BF0D2215D002A84FF0012340F8043DB9
:1016D00021F022FE02B010BD0122002119869A825B
:1016E0001A88394892B242F0010283421A80ADD181
:1016F0000A46364B03EBC20301A893F841408DF82C
:101700000440012300228DF805308DF807308DF854
:10171000062021F001FE1B2C08D02E2CDAD12C4BF8
:10172000019301A821F0F8FD02B010BD294B0193EF
:1017300001A821F0F1FD02B010BD204C18882468EA
:10174000B4FBF2F4013CA4B282B251E71B4C1888FE
:101750002468B4FBF2F4013CA4B282B256E7012043
:101760001A80D9621C8598821A8892B202431A8024
:1017700070E701201A80D9621C8598821A8892B27B
:1017800002431A8062E70122B3E70222B1E7032293
:10179000AFE70422ADE70522ABE70622A9E707225F
:1017A000A7E70822A5E70922A3E70A22A1E70B225F
:1017B0009FE70C229DE700BF0004014080BB002092
:1017C000000400400010004000000140ECDF03086E
:1017D0002C010001190100012C4B98423DD0B0F1C1
:1017E000804F3CD0A3F57C4398423AD003F5806308
:1017F000984238D003F58063984236D003F5806371
:10180000984234D003F58063984232D003F5704398
:10181000984230D003F5705398422ED003F5806380
:1018200098422CD003F5806398422AD0A3F59833D0
:10183000984228D003F58063984207D003F580636F
:10184000984208BF0D2202D0002070470C22104B96
:1018500003EBC20393F8400070470022F7E7012230
:10186000F5E70222F3E70322F1E70422EFE705227E
:10187000EDE70622EBE70722E9E70822E7E709227E
:10188000E5E70A22E3E70B22E1E700BF00000140A1
:10189000ECDF03082DE98048013085B0C3B2039323
:1018A0008A4D8B4F8B4C8C4E0A230293DFF82C927F
:1018B0001CF0E0F84FF4FA7A4FF0100C4FF47A7005
:1018C000D9F80430C3F30803002B40F0C180EFF3D4
:1018D0001183002B40F0BC802968A26800BF2B68F0
:1018E0009942F9D1D7F800E000FB0EF39B1AB3FB45
:1018F000FEF300FB01314FF0010E0191D9F80430E5
:10190000C3F30803002B40F08780EFF31183002B13
:1019100040F082802B68A16800BF2A689342F9D109
:10192000D7F800B000FB0BF2521AB2FBFBF200FB3F
:101930000323019A9B1AB3F57A7FDFD3BAF1010A28
:10194000BED1039B002B40F0BD804FF47A7ADFF8C4
:101950008C9150464FF0100CD9F80430C3F30803B3
:10196000002B40F09280EFF31183002B40F08D802C
:101970002968A26800BF2B689942F9D1D7F800E026
:1019800000FB0EF39B1AB3FBFEF300FB01314FF09B
:10199000010E0191D9F80430C3F3080303BBEFF340
:1019A0001183EBB92B68A16800BF2A689342F9D173
:1019B000D7F800B000FB0BF2521AB2FBFBF200FBAF
:1019C0000323019A9B1AB3F57A7FE3D3BAF1010A94
:1019D000C2D1029B013B02937FF468AFF9F75AFA38
:1019E000EFF311888CF31288A1682368DB0344BFEE
:1019F000C6F800E0A1682B6832685FFA88F888F3BF
:101A00001188D7F800801A4400FB08F35B1AB3FB77
:101A1000F8F300FB0233D4E7EFF311888CF312885C
:101A2000A1682368DB0344BFC6F800E0A1682B6807
:101A300032685FFA88F888F31188D7F800801A4472
:101A400000FB08F35B1AB3FBF8F300FB023370E70B
:101A5000EFF311828CF31288D4F808E02368D903DD
:101A600003D501233360D4F808E02B683168D2B283
:101A700082F311883A68194400FB02F3A3EB0E03CA
:101A8000B3FBF2F300FB013135E7EFF311828CF386
:101A90001288D4F808E02368D90303D50123336002
:101AA000D4F808E02B683168D2B282F311883A6822
:101AB000194400FB02F3A3EB0E03B3FBF2F300FBAC
:101AC000013164E7184621F00DFF3EE75CC70020B6
:101AD00060C7002010E000E058C7002000ED00E0E3
:101AE0002DE9F047AD4FAE4E13F042FEBE421ED27E
:101AF000DFF83883DFF838934446258862197DB1D2
:101B00004A450DD2052D0BD933886188C3F30B03E9
:101B1000994200F0D880144625886219002DEFD133
:101B2000716830461436F8F7CDF8BE42E4D39D4BC9
:101B30005A78022A40F2EC8000225A701A789A48A9
:101B40009A490160022A00F2DD8002EBC201984B43
:101B500002EB810203EB4202964C1046226021F018
:101B600025F8954A1378A3F1170102290FD9934953
:101B700011F83300002840F00381D800014449786F
:101B800029B18F4911F833300BB9182313708D4BDD
:101B90009A78042A00F0EB8032B91A88B2F5F07F07
:101BA00084BF4FF4F0721A80874D884A2B681A4020
:101BB000002A00F0EE80DE0700F1B580580400F145
:101BC000B980190700F1BD809A0100F1C1809B0422
:101BD00000F1C68023689A8CD98C914224BF0022E0
:101BE0009A84FFF703F91FF01BF910B9784823F026
:101BF0008FF80DF03DFB0021302276482BF0E9FFF5
:101C0000754B256803F1500102E0043399427DD001
:101C10001A78002AF9D19C78D8788442F5D26F4995
:101C20006F4B0A7028461D6026F05AFF6D4B6E4AB6
:101C30001E786E496E486F4B1160C825642212FBF6
:101C400006526D4C006B31F8041C5A600022218052
:101C50009A60DA601A615A619A61DA6183F8202029
:101C600083F8212008B10FF0B5FC644B9FED645A56
:101C70001B88644A9FED646A557B644C64496548DF
:101C8000086006EE903AF8EEE66A1389C5EE265A29
:101C900007EE103A5389127BC4ED005A07EE903AD2
:101CA000B8EEC77A5C4BF8EEE77A1D725A7227EEEF
:101CB000067A67EE867ABDE8F04783ED017AC3EDD8
:101CC000007A13F03DBD63799B077FF424AF716800
:101CD00094F804A03046F7F7F5FF3388BAEB133FCA
:101CE0000BD173887068AA1FC3F30B039A4204F1E7
:101CF0000601A8BF1A4629F055FC1436BE42FFF46F
:101D0000FBAE14E700221A70294A25E7012286E774
:101D10002649254802EB420201EB82011A78016054
:101D2000022AEFD811E73D48F8F702F82B6858046B
:101D30007FF547AF3A48F7F7FBFF2B6819077FF5A8
:101D400043AF3848F7F7F4FF2B689A017FF53FAFB0
:101D500046F20900F7F7ECFF2B689B047FF53AAFDA
:101D60003148F7F7E5FF4020F7F7E2FF32E71A8B3B
:101D7000B2F57A7FBFF418AF4FF47A721A8313E783
:101D8000D8000D186D68002D7FF4F8AE172515707A
:101D9000F4E643F008032B600DE700BFD40500080C
:101DA000880100080063002044270020C050002064
:101DB000C44F00204027002020290020FCFF0308FA
:101DC0008406040884BB0020F8500020096000024B
:101DD000387C0020602C0020D4460020F015002024
:101DE000942C0020EC4E0020A8D00020944100202C
:101DF00010250020542700208C440020B42A002005
:101E0000C0C9FB488C29002017B7D138B82A002058
:101E1000F04700203661023DCC47002008600002F8
:101E2000092000020160000209400002074000088A
:101E30000080000808B513F09BFCF7F7BFFF13F014
:101E40007FFCFFF74DFE0120BDE8084023F06EBF88
:101E50002DE9F04F013085B0C3B203930B460291D8
:101E60008B4C8C4E002B00F099808B4D8B4FDFF804
:101E700030921BF0FFFD4FF4FA7A4FF0100C4FF444
:101E80007A70D9F80430C3F30803002B40F0DE80E9
:101E9000EFF31183002B40F0D9802968A26800BFBE
:101EA0002B689942F9D1D7F800E000FB0EF39B1A9A
:101EB000B3FBFEF300FB01314FF0010E0191D9F8A5
:101EC0000430C3F30803002B40F08780EFF3118345
:101ED000002B40F082802B68A16800BF2A689342E3
:101EE000F9D1D7F800B000FB0BF2521AB2FBFBF2AB
:101EF00000FB0323019A9B1AB3F57A7FDFD3BAF173
:101F0000010ABED1039B002B40F0BD804FF47A7ACA
:101F1000DFF88C9150464FF0100CD9F80430C3F321
:101F20000803002B75D1EFF31183002B71D12968C1
:101F3000A26800BF2B689942F9D1D7F800E000FBF6
:101F40000EF39B1AB3FBFEF300FB01314FF0010EC1
:101F50000191D9F80430C3F3080313BBEFF31183E5
:101F6000FBB92B68A16800BF2A689342F9D1D7F862
:101F700000B000FB0BF2521AB2FBFBF200FB032392
:101F8000019A9B1AB3F57A7FE3D3BAF1010AC4D15F
:101F9000029B013B0293002B7FF467AF05B0BDE8C5
:101FA000F08FEFF311888CF31288A1682368DB03AC
:101FB00044BFC6F800E0A1682B6832685FFA88F871
:101FC00088F31188D7F800801A4400FB08F35B1AE5
:101FD000B3FBF8F300FB0233D2E7EFF311888CF385
:101FE0001288A1682368DB0344BFC6F800E0A1683B
:101FF0002B6832685FFA88F888F31188D7F8008078
:102000001A4400FB08F35B1AB3FBF8F300FB02333E
:1020100070E7EFF311828CF31288D4F808E023689C
:10202000D90303D501233360D4F808E02B68316865
:10203000D2B282F311883A68194400FB02F3A3EB91
:102040000E03B3FBF2F300FB01317FE7EFF31182E4
:102050008CF31288D4F808E02368D90303D5012350
:102060003360D4F808E02B683168D2B282F311886B
:102070003A68194400FB02F3A3EB0E03B3FBF2F33F
:1020800000FB013118E7184621F02CFC3EE700BFA9
:1020900010E000E058C700205CC7002060C70020A7
:1020A00000ED00E0204B5B68C3F3080330B4BBB91C
:1020B000EFF31183A3B91D4B1D4C1868A16800BF35
:1020C0001A689042F9D11B4B1C684FF47A7202FBDC
:1020D00004F3591AB1FBF4F130BC02FB0010704755
:1020E000EFF31182102383F3128811498C680B6877
:1020F00013F4803F104B02D0012018608C680B490C
:10210000D2B20D68186882F311880A4B19684FF42F
:102110007A72284402FB01F31B1B30BCB3FBF1F3C2
:1021200002FB0030704700BF00ED00E05CC70020FC
:1021300010E000E060C7002058C700202DE9F84FEC
:102140008046FFF7AFFF254E2549DFF8A0E0254A7E
:10215000254D844610274FF47A740120DEF80430B0
:10216000C3F30803D3B9EFF31183BBB90B68D2F8FB
:1021700008A000BFD1F800904B45F7D1D6F800B0C9
:1021800004FB0BF9A9EB0A09B9FBFBF904FB039368
:10219000A3EB0C034345E1D3BDE8F88FEFF3118ABD
:1021A00087F31288D2F808B01368DB0344BF2860B5
:1021B000D2F808B00B68D5F800905FFA8AFA8AF373
:1021C0001188D6F800A0994404FB0AF3A3EB0B0393
:1021D000B3FBFAF304FB0933DAE700BF60C7002062
:1021E0005CC7002010E000E058C7002000ED00E0D0
:1021F0002DE9F04FDFF830C1474A4849484E494D74
:102200008046102718F1FF38C0F08480DCF80430D5
:10221000C3F30803002B5CD1EFF31183002B58D1DB
:102220000B68946800BF08688342F9D1D6F8009023
:102230004FF47A7000FB09FEAEEB040EBEFBF9FE14
:1022400000FB03EEDCF80430C3F308034FF47A74A8
:102250000120FBB9EFF31183E3B90B68D2F808A0B2
:1022600000BFD1F800904B45F7D1D6F800B004FB81
:102270000BF9A9EB0A09B9FBFBF904FB0393A3EBE8
:102280000E03B3F57A7FBDD2DCF80430C3F3080344
:10229000002BDFD0EFF3118A87F31288D2F808B051
:1022A0001368DB0344BF2860D2F808B00B68D5F888
:1022B00000905FFA8AFA8AF31188D6F800A0994450
:1022C00004FB0AF3A3EB0B03B3FBFAF304FB0933A0
:1022D000D5E7EFF3118487F31288D2F808901368DA
:1022E000D80303D501232B60D2F808900B68286827
:1022F000E4B284F31188D6F800A04FF47A7400EBAE
:10230000030E04FB0AF3A3EB0903B3FBFAF304FB8C
:102310000E3E97E7BDE8F08F10E000E05CC70020BC
:1023200060C7002058C7002000ED00E030B4EFF394
:102330001183102282F312880649074C0A68074865
:10234000013200250A602560DBB2026883F3118840
:1023500030BC70475CC7002058C7002010E000E088
:102360000F4B1B88014643B90E4B0F4A1B78106870
:102370000BB981F00101F7F7ADB90C4B5A691AB1ED
:1023800018B91A68106058747047094A186811889B
:10239000084A92FBF1F2012102605974704700BFB4
:1023A00034C7002036C7002038C700203CC70020B3
:1023B00054C7002020A107002DE9F04FDFF808A145
:1023C0002DED0C8B9AF8003099B0012B089002F09B
:1023D0007383DFF8F8B09BF80021002A41F04083B6
:1023E000072B354C02F0E7820023039363683248E1
:1023F000984700286ED0B4F8A860002284F84920DD
:10240000002E40F09282B4F92600226BB4F92450D9
:10241000E16AB4F92830821A606BE263691A274DC9
:10242000A1631B1A94F84A10254823640FF054F84E
:102430002B6813F0005302F0E182D4ED0F5AD4ED73
:102440000E7A204A9BED656ADBED666A9BED677A42
:10245000DBF8A0311268B8EEE58AD4ED105AF8EE38
:10246000E77AF8EEE58A013377EE867A38EE268A47
:1024700078EE878A9342CBED657A8BED668ACBED59
:10248000678ACBF8A03101F061869AF80080B8F134
:10249000140F03F080820023DBF8A8610493062E5A
:1024A00002F28A83DFE816F0BE179017271374191B
:1024B000DE19EA18821800BF787C002088C000204E
:1024C000B07C0020B4840020E1CE0020A4290020AC
:1024D000DDF810B09AF80080B8F1070F00F0DC8248
:1024E0009BF8B831002B40F0E282CE4B5B79002B99
:1024F00040F0168201239AF800208BF8B831072AA1
:1025000002F05E8400230B93C74B9BED70AA93ED02
:10251000007AC64AC64F12680592F7EE007A77EE47
:10252000CA8AC44AC44BDFF88C93069268EE878A45
:10253000C24A9BED6F9ADFF880839FEDC1BADFED51
:10254000C19ADFEDC1BADFEDC1CADFEDC1AA9FEDCF
:10255000C1CAC14ECDF80C90F4EEE78A0024F1EE2A
:1025600010FA0993079288BFF0EE678A0493254614
:10257000B946BA4B2344D3ED007AB94BF5EE407A15
:102580002344F1EE10FA93ED008A17D0B54B2344A3
:1025900093ED007A78EE476AB0EEE66AF4EEC67A1A
:1025A000F1EE10FA08D5F5EEC06AF1EE10FACCBFE4
:1025B00037EE878A37EE678A83ED008A069B1F888D
:1025C000BB0700F07C82022D04F0C2860599A64B61
:1025D00091F8322006EE902A33F91520234407EEB5
:1025E000102A13ED096A91F83130B8EEC77AF8EE87
:1025F000E66A5A4207EE902AA6EE867A6900F8EE5D
:10260000E77AB4EEE77AF1EE10FA0AD407EE903AE0
:10261000F8EE677AF4EEC77AF1EE10FA88BFF0EEC2
:10262000477A924B0A93924A0B44515EB3F90A30AF
:10263000C81A07EE100AB8EEC77AFF07E7EE697A04
:1026400040F1B0828B4F97ED008A27EE888A9BF885
:10265000D071E7B1874FDBF8D401D7ED007A864F10
:102660005B1A07EE103A089B396867EEA97AB8EE54
:10267000C78A1F1A8F4228EE278A01F3AF81F7EE2F
:10268000007AB4EEE7AAF1EE10FA01F173817B4B08
:102690002344D3ED007A049BD3ED01DA039B69EE6A
:1026A000277A38EE6DDA67EE8D7AC3ED007A079BF4
:1026B00098ED007AD3ED007A714BD6ED006A67EEA3
:1026C000277A234427EEA87AD3ED007A67EE277A9B
:1026D000B0EE667AA7EE8D7AF0EE477A9BED706ADF
:1026E000B7EE007AB4EEC76AF1EE10FAACBF012380
:1026F000002343B1F0EEE66AB0EEE77AB4EEE67A94
:10270000F1EE10FA01D5C6ED007A022D04F04E85E7
:102710005C4A5D4B52F825001B68B0EE6D0A984785
:102720005A4A5B4B52F825001B689847059B93F863
:102730003A30632B04D8069B1B88002B01F0608184
:10274000B0EE6C8A534BD8ED007A38EE400A234441
:1027500093ED008A83ED000A059B30EE480A93F85A
:10276000482080EE278ADAB1F7EE007AB4EEE7AAC5
:10277000F1EE10FA14DB484BD3ED007AB0EEC87AD4
:10278000B4EEE77AF1EE10FA0ADD444BD3ED007AAD
:10279000B0EECDDAB4EEE7DAF1EE10FA01F35B82D7
:1027A0003F4B9BF8E0212344D3ED007A69EE277A72
:1027B00027EE888A89ED008A32B9039BC6ED00CAEC
:1027C000C3ED00CAC9ED00CA039B04330393049B05
:1027D000043404330C2C05F1010509F1040906F158
:1027E000040604937FF4C5AE9AF80030072B02F07C
:1027F000F681012B02F0D48200230393294A0B4B6C
:1028000011681B6893F82F0011F48053049300F0B3
:102810004B82254C254D2378254FED8897ED037A83
:102820004CE000BF647C00201CC400204027002036
:10283000404400203C2700209C8400209800002079
:1028400000009642CDCCCC3DAE47813F0000000059
:102850000000C842610BB63B3444002010C4002085
:10286000A82A0020682B0020342B00209041002053
:1028700054250020F8C3002020C40020CCC3002031
:10288000D8C3002038490020344900209C4900204A
:10289000984900207C2B002030C400202CC400204C
:1028A000E4C3002088C000204C650020C441002003
:1028B000D0CF002028440020C8C3002013F0010F0F
:1028C000A74B1A8B08BFABF8E821571B07EE907A8D
:1028D000F8EEE77AB4EEE77AF1EE10FA42F2C08150
:1028E000561906EE906AF8EEE66AB4EEE67AF1EE74
:1028F00010FA81F2F383BBF8E821974283F25785FF
:10290000984A994D92ED005A95ED003A974A8BED11
:102910007B3A8BED7C5AD2ED006ADFED957ADCE1F3
:10292000944B1B78013BDBB2E5E5934B934909934C
:1029300091F801901B68924F9AF80080B7F9060051
:102940004FF47A71B1FBF3F3C3EB431503EB85034B
:10295000DD00ADB2AE4203F0A480E16FB4F924E033
:10296000236E4A1C07EE90EA7344012AE26723664D
:10297000F8EEE77A03F09F80D4ED1B5AD4ED1D6A80
:1029800007EE102A37EEE56AB8EEC75A012E86EE3A
:10299000057A37EE257A77EEC77A84ED1C7AE6EE73
:1029A000276A84ED1B7AF0EE667AC4ED1E6AC4EDE8
:1029B0001D6A03F0AF85D4F89010B4F926E0636E79
:1029C0004A1C07EE90EA7344012AC4F8902063661B
:1029D000F8EEE77A03F08780D4ED205AD4ED226A2E
:1029E00007EE102A37EEE56AB8EEC75A012E86EEDA
:1029F000057A37EE257A77EEC77A84ED217AE6EE0E
:102A0000276A84ED207AF0EE667AC4ED236AC4ED7D
:102A1000226A03F03885D4F8A410B4F928E0A36E34
:102A20004A1C07EE90EA7344012AC4F8A420A36666
:102A3000F8EEE77A03F07080D4ED255AD4ED276ADA
:102A400007EE102A37EEE56AB8EEC75A012E86EE79
:102A5000057A37EE257A77EEC77A84ED267AE6EEA8
:102A6000276A84ED257AF0EE667AC4ED286AC4ED13
:102A7000276A03F0FB84F880B4F8A8309AF8008045
:102A8000013BA4F8A83009990023B8F1070F4B6067
:102A90008B60CB607FF424ADFFF704FB039B384FC2
:102AA000C01A9BF8B8313880002B3FF41EAD013BB3
:102AB0008BF8B83119B0BDEC0C8BBDE8F08F9BF8EA
:102AC000D03163B1022D04F032842E4B0A932E4A8A
:102AD00003EB450332F91510B3F90A30BAE52B4B75
:102AE000234493ED000A049BD3ED01DA039B29EE06
:102AF000000A38EE6DDA022D20EE0D0A83ED000A91
:102B00007FF4D5AD224A234B10681B689847079B7A
:102B100098ED007AD3ED007A1F4BD6ED006A1A7853
:102B20001E4B83ED020A1E4B67EE277A234467EEA5
:102B3000A87A93ED006A67EE867AB0EE667AA7EE21
:102B40008D7A012AF0EE477A02D0192A7FF4C6ADB9
:102B5000B4EECBDAF1EE10FACCBF01230023C8E5C6
:102B600058C00020D84E002074410020E84E0020BC
:102B700000000000844100209C840020647C002030
:102B8000E4CE00209041002054250020CCC300203A
:102B9000FC4D0020104E00205CC200202844002084
:102BA000D8C30020DBED5E6A9BED5F7AB2F900E0EE
:102BB000B2F90270B4EEE67AF1EE10FA8EEAEE7037
:102BC00087EAE77C4CBFB7EE007AF7EE006AA0EB2D
:102BD000EE70ACEBE77C4CBF77EE665A76EEC75AE8
:102BE000604540F3FA87BEF1000FD6BFCEF100007A
:102BF00007EE10EA07EE100A274FB8EEC77A3F78C3
:102C000027EE297A002F00F0F887244F97ED005A1D
:102C1000B5EEC05AF1EE10FA41F36187204FD7EDBF
:102C2000004AF5EEC04AF1EE10FA41F3588734EE4F
:102C3000C77AB7EE006AC7EE246A75EEC65AF4EE9C
:102C4000C66A65EEAA5AF1EE10FA85EE857A88BF5B
:102C5000F0EE466AF5EEC06AF1EE10FA37EE067A4B
:102C6000B8BFF0EE6C6A66EE876AF4EEC66AF1EE03
:102C700010FA88BFF0EE466AF5EEC06AF1EE10FA7F
:102C8000B8BFF0EE6C6A074F97ED007A67EE877A6F
:102C9000A7EEA68ADBE400BF04C4002000C4002025
:102CA00008C40020FCC30020E14BE24A5C8B92ED9B
:102CB000037AE14A07EE904AE04C92ED003AE04A8E
:102CC00094ED005AD2ED006ADE4C8BED7C5AF8EEA2
:102CD000E77A8BED7B3A77EE677A87EEA66ADA4D74
:102CE000DA4AD5ED005ADA4DDFEDDA6AD5ED003A71
:102CF000D94DDFEDDA4A95ED004A92ED007AF7EE14
:102D0000007AB4EEE76A75EEA35AF1EE10FA88BFC6
:102D1000B0EE676A75EE845AB4EEE66AF1EE10FA28
:102D200065EEA45AB8BFB0EE666AF1EE476A33EEBC
:102D3000454AF4EEE65AF1EE10FA8BED7D6A8BED22
:102D40007F4A00F19F84F4EEC75AF1EE10FA88BF73
:102D5000F0EE475ABC4ADFEDC14AD2ED017ABC4AD7
:102D6000D2ED012ABC4A77EEA27AD2ED013A77EE93
:102D7000A37A67EEA47AF4EEE76AF1EE10FA08DCC3
:102D8000B4EEE77AF1EE10FA8CBFF0EE676AF0EE7F
:102D9000476AAD4ADFEDB13AD2ED027AAC4AD2EDE4
:102DA000024AAF4A77EEA47A92ED007A67EEA37AF0
:102DB000F1EE474AF4EEE47AF1EE10FA08D4F4EEBC
:102DC000C77AF1EE10FA8CBFF0EE474AF0EE674A90
:102DD000002841F04682F7EE007AA24AA24D5278CE
:102DE0009BF80002002AFFEE002AB7EE007A2A784C
:102DF00014BFB0EE472AB0EE622A002814BFF0EEEE
:102E0000623AF0EE473A002A02F01B87F4EEC77AE6
:102E1000F1EE10FA64EE824A944841F3638290ED39
:102E2000027A90ED011AD0ED031A9FED8A2A26EE60
:102E3000877A67EEA32AA1EE257AA1EEA47A27EE7F
:102E4000227AB4EEC27AF1EE10FAB4BFF0EE427A12
:102E5000F0EE477A8DED0C7A88BFB0EE427A012A07
:102E600000F0BF81D0ED063AD0ED051A90ED072AAB
:102E700066EEA33AE5EEA13AE4EE823A63EEA23AB8
:102E8000F4EEC73AF1EE10FAF4EEE73A8CBFB0EE8A
:102E9000472AB0EE632AF1EE10FA98BFB0EE427AFC
:102EA000A8BFF0EE637A022ACDED0D3A00F09981C9
:102EB000D0ED0A3AD0ED091A90ED0B2A66EEA33A4E
:102EC000E5EEA13AE4EE823A63EEA23AF4EEC73AB6
:102ED000F1EE10FAF4EEE73A8CBFB0EE472AB0EE0E
:102EE000632AF1EE10FA98BFB0EE427AA8BFF0EE76
:102EF000637A032ACDED0E3A00F07381D0ED0E3ADD
:102F0000D0ED0D1A90ED0F2A66EEA33AE5EEA13A48
:102F1000E2EE243A63EEA23AB4EEE37AF1EE10FA6E
:102F2000F4EEE37A8CBFB0EE632AB0EE472AF1EEFE
:102F300010FA58BFB0EE427AB8BFF0EE637A042AB6
:102F4000CDED0F3A00F04D81D0ED123AD0ED111ACF
:102F500090ED132A66EEA33AE1EEA53AE2EE243AAA
:102F600063EEA23AF4EEC73AF1EE10FAF4EEE37A29
:102F70008CBFB0EE472AB0EE632AF1EE10FAA8BF7C
:102F8000B0EE427AB8BFF0EE637A052ACDED103A82
:102F900000F02781D0ED163AD0ED151A90ED172AE2
:102FA00066EEA33AE1EEA53AE2EE243A63EEA23AE7
:102FB000F4EEC73AF1EE10FAF4EEE37A8CBFB0EE1D
:102FC000472AB0EE632AF1EE10FA58BFB0EE427A0B
:102FD000B8BFF0EE637A062ACDED113A00F0018118
:102FE000D0ED1A3AD0ED191A90ED1B2A66EEA33AED
:102FF000E1EEA53AE2EE243A63EEA23AF4EEC73AE5
:10300000F1EE10FAF4EEE73A8CBFB0EE472AB0EEDC
:10301000632AF1EE10FA98BFB0EE427AA8BFF0EE44
:10302000637A072ACDED123A00F0DB8020E000BF82
:1030300058C00020D0CF00207441002070410020F3
:10304000E04E00204C6500202844002034C40020BD
:103050003444002000000000404400206F12833AF6
:1030600038C4002020290020D1CE0020184E002096
:10307000D0ED1E3AD0ED1D1A90ED1F2A66EEA33A50
:10308000E1EEA53AE2EE243A63EEA23AF4EEC73A54
:10309000F1EE10FAF4EEE73A8CBFB0EE472AB0EE4C
:1030A000632AF1EE10FA98BFB0EE427AA8BFF0EEB4
:1030B000637A082ACDED133A00F09380D0ED223ADE
:1030C000D0ED211A90ED232A66EEA33AE1EEA53A5F
:1030D000E2EE243A63EEA23AB4EEE37AF1EE10FAAD
:1030E000F4EEE37A8CBFB0EE632AB0EE472AF1EE3D
:1030F00010FA58BFB0EE427AB8BFF0EE637A092AF0
:10310000CDED143A6DD0D0ED263AD0ED251A90EDE4
:10311000272A66EEA33AE1EEA53AE2EE243A63EE00
:10312000A23AF4EEC73AF1EE10FAF4EEE73A8CBFA9
:10313000B0EE472AB0EE632AF1EE10FA98BFB0EE77
:10314000427AA8BFF0EE637A0A2ACDED153A48D04C
:10315000D0ED2A3AD0ED291A90ED2B2A66EEA33A4B
:10316000E5EEA13AE2EE243A63EEA23AB4EEE37A57
:10317000F1EE10FAF4EEE37A8CBFB0EE632AB0EE13
:10318000472AF1EE10FACDED163A58BFB0EE427A6A
:10319000A8BFF0EE673A0B2A03F02281D0ED2E7A19
:1031A000D0ED2D1A90ED2F2A66EEA77AE1EEA57AE2
:1031B000E2EE247A67EEA27AF4EEC77AF1EE10FA24
:1031C000F4EEE37A8CBFF0EE476AF0EE676AF1EE58
:1031D00010FACDED177A98BFB0EE667AB8BFF0EE70
:1031E000637A77EEC77AF7EE006AF4EEE67AF1EEEC
:1031F00010FACBED707A43F3C58086EEA77A012AE8
:10320000DDED0C7A67EE877ACDED0C7A55D0DDEDE9
:103210000D7A67EE877A022ACDED0D7A4DD0DDED7D
:103220000E7A67EE877A032ACDED0E7A45D0DDED72
:103230000F7A67EE877A042ACDED0F7A3DD0DDED67
:10324000107A67EE877A052ACDED107A35D0DDED5C
:10325000117A67EE877A062ACDED117A2DD0DDED51
:10326000127A67EE877A072ACDED127A25D0DDED46
:10327000137A67EE877A082ACDED137A1DD0DDED3B
:10328000147A67EE877A092ACDED147A15D0DDED30
:10329000157A67EE877A0A2ACDED157A0DD0DDED25
:1032A000167A67EE877A0B2ACDED167A05D0DDED1A
:1032B000177A27EE877A8DED177AE048006810F0CC
:1032C000805000F08584B6EE006A8BED7D6A002A9E
:1032D00002F0D2842478DFF88483DFF884C3DFF837
:1032E0008493D74F9BF8F8E15B8B0593FDEEC37A8F
:1032F000D8ED006A99F80390BCF906803F7804F095
:10330000010301F0100C17EE904A01F48001BEF1A8
:10331000000F40F0BB81BCF1000F40F06585C9484B
:10332000DDED0C7A90ED007AC749E7EE067AB9F147
:10333000000F42F09B85BDEEC57A17EE106AB0EE25
:10334000457AA4EE277AFDEEC77A17EE90EA17EEDB
:10335000907AA645A8BF27467645C8BF374607EEF0
:10336000907AF8EEE77A012AC1ED007A00F04981FF
:1033700090ED047ADDED0D7AE7EE067AB0EE457A4F
:10338000A4EE277AFDEEC77A17EE90EA17EE907A50
:10339000A645A8BF27467645C8BF374607EE907AB0
:1033A000F8EEE77A022AC1ED017A00F02A8190ED69
:1033B000087ADDED0E7AE7EE067A2746B0EE457A1A
:1033C000A4EE277AFDEEC77A17EE90EA7445A8BFFF
:1033D00077467645C8BF374607EE907AF8EEE77A2B
:1033E000032AC1ED027A00F00C8190ED0C7ADDED3C
:1033F0000F7AE7EE067AB0EE457AA4EE277AFDEE74
:10340000C77A17EE90EA17EE907AA645A8BF27462E
:10341000B645B8BF374607EE907AF8EEE77A042A49
:10342000C1ED037A00F0ED8090ED107ADDED107AB9
:10343000E7EE067AB0EE457AA4EE277AFDEEC77A7B
:1034400017EE90EA17EE907AA645A8BF2746B64534
:10345000B8BF374607EE907AF8EEE77A052AC1ED55
:10346000047A00F0CE8090ED147ADDED117AE7EE6B
:10347000067AB0EE457AA4EE277AFDEEC77A17EE0B
:1034800090EA17EE907AA645A8BF2746B645B8BF82
:10349000374607EE907AF8EEE77A062AC1ED057A0C
:1034A00000F0AF8090ED187ADDED127AE7EE067A43
:1034B000B0EE457AA4EE277AFDEEC77A17EE90EAD1
:1034C00017EE907AA645A8BF2746B645B8BF37463F
:1034D00007EE907AF8EEE77A072AC1ED067A00F057
:1034E000908090ED1C7ADDED137AE7EE067AB0EE6F
:1034F000457AA4EE277AFDEEC77A17EE90EA17EE2A
:10350000907AA645A8BF2746B645B8BF374607EE0E
:10351000907AF8EEE77A082AC1ED077A71D090ED3B
:10352000207ADDED147AE7EE067AB0EE457AA4EE65
:10353000277AFDEEC77A17EE90EA17EE907AA64545
:10354000A8BF2746B645B8BF374607EE907AF8EED3
:10355000E77A092AC1ED087A53D090ED247ADDED9F
:10356000157AE7EE067AB0EE457AA4EE277AFDEEFC
:10357000C77A17EE90EA17EE907AA645A8BF2746BD
:10358000B645B8BF374607EE907AF8EEE77A0A2AD2
:10359000C1ED097A35D090ED287ADDED167AE7EEA7
:1035A000067AB0EE457AA4EE277AFDEEC77A17EEDA
:1035B00090EA17EE907AA645A8BF2746B645B8BF51
:1035C000374607EE907AF8EEE77A0B2AC1ED0A7AD1
:1035D00017D090ED2C7ADDED177AE7EE067AA4EE9F
:1035E000275AFDEEC57A17EE900A8442A8BF04461A
:1035F0008642D8BF264607EE906AF8EEE77AC1ED1C
:103600000B7A002B00F0B583104B1B68002B40F0A9
:10361000BD830F4B1B7843B3287858B10A4E0D4F2A
:103620000024E0B23B68B6EC010A984728780134E0
:103630008442F6DB084B1B6816E000BF4CC8002034
:10364000ACBB0020184E00205C440020C4C3002006
:1036500014C00020A0BB0020A8BB0020144E0020F6
:10366000FC2800205427002098479AF80030072BA8
:1036700001F0398201238BF8003119B0BDEC0C8BBD
:10368000BDE8F08FF0EE665AFFF764BBBCF1000FA7
:1036900040F01383E848DDED0C7A90ED007AE749BD
:1036A000E7EE067AB1EE444AB0EE437AA4EE277A0A
:1036B000F0EE477A002F41F09983B9F1000F43F003
:1036C000A481BDEEC57AFDEEE77A17EE106A17EE1B
:1036D00090EA17EE907AA645A8BF27467645C8BF60
:1036E000374607EE907AF8EEE77A012AC1ED007AC4
:1036F00087D090ED047ADDED0D7AE7EE067AB0EE34
:10370000437AA4EE277AFDEEC77A17EE90EA17EE19
:10371000907AA645A8BF2746B645B8BF374607EEFC
:10372000907AF8EEE77A022AC1ED017A3FF469AFA8
:1037300090ED087ADDED0E7AE7EE067AB0EE437A88
:10374000A4EE277AFDEEC77A17EE90EA17EE907A8C
:10375000A645A8BF2746B645B8BF374607EE907ABC
:10376000F8EEE77A032AC1ED027A3FF44AAF90ED12
:103770000C7ADDED0F7AE7EE067AB0EE437AA4EE2E
:10378000277AFDEEC77A17EE90EA17EE907AA645F3
:10379000A8BF2746B645B8BF374607EE907AF8EE81
:1037A000E77A042AC1ED037A3FF42BAF90ED107A4B
:1037B000DDED107AE7EE067AB0EE437AA4EE277AD2
:1037C000FDEEC77A17EE90EA17EE907AA645A8BFED
:1037D0002746B645B8BF374607EE907AF8EEE77A47
:1037E000052AC1ED047A3FF40CAF90ED147ADDEDBB
:1037F000117AE7EE067AB0EE437AA4EE277AFDEE70
:10380000C77A17EE90EA17EE907AA645A8BF27462A
:10381000B645B8BF374607EE907AF8EEE77A062A43
:10382000C1ED057A3FF4EDAE90ED187ADDED127A38
:10383000E7EE067AB0EE437AA4EE277AFDEEC77A79
:1038400017EE90EA17EE907AA645A8BF2746B64530
:10385000B8BF374607EE907AF8EEE77A072AC1ED4F
:10386000067A3FF4CEAE90ED1C7ADDED137AE7EEEA
:10387000067AB0EE437AA4EE277AFDEEC77A17EE09
:1038800090EA17EE907AA645A8BF2746B645B8BF7E
:10389000374607EE907AF8EEE77A082AC1ED077A04
:1038A0003FF4AFAE90ED207ADDED147AE7EE067AC4
:1038B000B0EE437AA4EE277AFDEEC77A17EE90EACF
:1038C00017EE907AA645A8BF2746B645B8BF37463B
:1038D00007EE907AF8EEE77A092AC1ED087A3FF40C
:1038E00090AE90ED247ADDED157AE7EE067AB0EE33
:1038F000437AA4EE277AFDEEC77A17EE90EA17EE28
:10390000907AA645A8BF2746B645B8BF374607EE0A
:10391000907AF8EEE77A0A2AC1ED097A3FF471AE9F
:1039200090ED287ADDED167AE7EE067AB0EE437A6E
:10393000A4EE277AFDEEC77A17EE90EA17EE907A9A
:10394000A645A8BF2746B645B8BF374607EE907ACA
:10395000F8EEE77A0B2AC1ED0A7A3FF452AE90ED09
:103960002C7ADDED177AE7EE067AA4EE273AFDEE23
:10397000C37A38E60A9BB2F90070B3F90A303049CD
:10398000F81A096880EAE073A3EBE0738B42BEF695
:103990007EAEB2F902300A9AB2F90C209A1A82EA83
:1039A000E273A3EBE27399427EF771AE0999254B5E
:1039B000D1ED017A93ED007AF0EEE77AF4EEC77A72
:1039C000F1EE10FA7EF563AED1ED027AF0EEE77A11
:1039D000B4EEE77AF1EE10FA7EF759AE1A4B1A8878
:1039E00000238BF8D031002A40F09A83174A184BF5
:1039F0001178186881F00101F5F76CFEFEF747BEFB
:103A0000144B154A234493ED007AD2ED007A134B00
:103A100067EE277AF7EE006AF4EEE67AF1EE10FA36
:103A200093ED007A88BFF0EE667A67EE877A27EE2C
:103A3000888AFEF787BE00BF184E00205C44002035
:103A400024C4002028C4002034C7002036C700202A
:103A500038C700201C2B0020F4C30020F0C3002036
:103A6000072B02F075830026CA4DCB4C2B685905F5
:103A700001F10D81C94B1B78002B40F00281C84B2E
:103A80009BF8127127B1C74A1288920742F0FE8054
:103A90009BF81881DA7FB8F1000F41F025819D7FF6
:103AA000002D00F0E185022D02F0C480032D01F00D
:103AB0007B84BD4949880232D2B2B8F1000F02F0CE
:103AC000AD80002902F0AA80B8480568B1FBF5F185
:103AD0000DB2ABF84851002A03F01E8107EE905A50
:103AE000F8EEE77AF7EE006A86EEA77AB049012A87
:103AF000DBED576AD1ED007A77EEE67A67EE877AEA
:103B0000CBED537A21D0D1ED017ADBED586A77EE17
:103B1000E67A022A67EE877ACBED547A15D0D1ED9A
:103B2000027ADBED596A77EEE67A032A67EE877A46
:103B3000CBED557A09D0D1ED037ADBED5A6A77EEF9
:103B4000E67A67EE877ACBED567A9AF80000092874
:103B500003F04A81002D40F38E8592B3DBED577A56
:103B60009BED537A77EE877A012ACBED577AC1ED38
:103B7000007A21D0DBED587A9BED547A77EE877A84
:103B8000022ACBED587AC1ED017A15D0DBED597AD6
:103B90009BED557A77EE877A032ACBED597AC1ED02
:103BA000027A09D0DBED5A7A9BED567A77EE877A66
:103BB000CBED5A7AC1ED037A013A022AB8BF02224C
:103BC000D2B2B8F1000F0CBF1046022000F054BD75
:103BD0004E023FF578ABFFF77ABB002FD6BF784295
:103BE00007EE107A07EE100A724FB8EEC77A3F78E8
:103BF00027EE297A002F7FF408A86F4F97ED006A0F
:103C0000B4EEEB6AF1EE10FA41F12580B7EE005AFE
:103C100035EE465ADFED696A694F36EEC77A25EE12
:103C20000C5AD7ED006AA5EE076A26EE267AB5EEA5
:103C3000C07AF1EE10FA40F25287CAEE876AB7EE08
:103C4000006A35EEC67AF0EE465AE7EE265AF0EEF6
:103C5000656AFFF70AB801230899CBF8D411022A44
:103C60008BF8D0317EF49CAD564A1288002A43F07E
:103C70005680554A554B11781868F5F72BFDFEF71D
:103C80008FBD534A464BB2F906105A8B91423FF70B
:103C9000F7AE504A1278012A01F08687192A01F0FE
:103CA00083870E2A3FF4ECAE082A3FF4E9AE404980
:103CB00000228A60CBF80C21E2E6002B42F07080F3
:103CC000002F41F00683FDEEC57A0DF1300E17EEA0
:103CD000907AFDEEE67A0EEB820304933E48DFF81D
:103CE0000081CDF818B04FFA89F317EE906AB1EE63
:103CF000444A89F0010C05929B46034693ED007AF5
:103D0000FEEC017AE7EE067A1030B0EE437AA4EECC
:103D1000277AFDEEC77A17EE903A17EE902AA34263
:103D2000A8BF22469E42CCBF002109F00101002914
:103D300014BF114631469F42CCBF00230CF0010353
:103D400007EE901A002B14BF13463B46B8EEE77AF5
:103D500007EE903A049BF8EEE77ABBF1000F18BF2C
:103D6000F0EE477A9E45E8EC017AC6D1059ADDF877
:103D700018B0002A3FF448AC92001849184827F0C0
:103D800011FC184B1B68002B3FF443AC1EF09AFA51
:103D90003FE400BF88C00020787C0020F0150020A0
:103DA00058C000203C270020F0280020D0460020EA
:103DB000D0CF002004C400200CC4002000003443F5
:103DC00000C4002034C7002036C7002038C70020B8
:103DD000FC28002020290020184E0020CC41002083
:103DE0005C440020C4C30020002B41F09087B9F14F
:103DF000000F42F00783CF48DDED0C7A90ED007A9A
:103E0000CD49E7EE067ABDEEC57A17EE103AB0EE70
:103E1000457AA4EE277AFDEEC77A17EE907A17EE70
:103E2000906AA742A8BF2646BB42C8BF1E4607EEFF
:103E3000906AF8EEE77A012AC1ED007A9CD090ED05
:103E4000047ADDED0D7AE7EE067AB0EE457AA4EE5F
:103E5000277AFDEEC77A17EE907A17EE906AA7429E
:103E6000A8BF26469F42B8BF1E4607EE906AF8EEEE
:103E7000E77A022AC1ED017A3FF47EAF90ED087A2D
:103E8000DDED0E7AE7EE067AB0EE457AA4EE277AFB
:103E9000FDEEC77A17EE907A17EE906AA742A8BF98
:103EA00026469F42B8BF1E4607EE906AF8EEE77AB4
:103EB000032AC1ED027A3FF45FAF90ED0C7ADDED9D
:103EC0000F7AE7EE067AB0EE457AA4EE277AFDEE99
:103ED000C77A17EE907A17EE906AA742A8BF2646D7
:103EE0009F42B8BF1E4607EE906AF8EEE77A042AB2
:103EF000C1ED037A3FF440AF90ED107ADDED107A1A
:103F0000E7EE067AB0EE457AA4EE277AFDEEC77AA0
:103F100017EE907A17EE906AA742A8BF26469F42F6
:103F2000B8BF1E4607EE906AF8EEE77A052AC1EDA3
:103F3000047A3FF421AF90ED147ADDED117AE7EECB
:103F4000067AB0EE457AA4EE277AFDEEC77A17EE30
:103F5000907A17EE906AA742A8BF26469F42B8BF44
:103F60001E4607EE906AF8EEE77A062AC1ED057A5A
:103F70003FF402AF90ED187ADDED127AE7EE067AA3
:103F8000B0EE457AA4EE277AFDEEC77A17EE907A66
:103F900017EE906AA742A8BF26469F42B8BF1E46AA
:103FA00007EE906AF8EEE77A072AC1ED067A3FF449
:103FB000E3AE90ED1C7ADDED137AE7EE067AB0EE13
:103FC000457AA4EE277AFDEEC77A17EE907A17EEBF
:103FD000906AA742A8BF26469F42B8BF1E4607EE7A
:103FE000906AF8EEE77A082AC1ED077A3FF4C4AE8A
:103FF00090ED207ADDED147AE7EE067AB0EE457AA0
:10400000A4EE277AFDEEC77A17EE907A17EE906A43
:10401000A742A8BF26469F42B8BF1E4607EE906A39
:10402000F8EEE77A092AC1ED087A3FF4A5AE90EDE3
:10403000247ADDED157AE7EE067AB0EE457AA4EE45
:10404000277AFDEEC77A17EE907A17EE906AA742AC
:10405000A8BF26469F42B8BF1E4607EE906AF8EEFC
:10406000E77A0A2AC1ED097A3FF486AE90ED287A04
:10407000DDED167AE7EE067AB0EE457AA4EE277A01
:10408000FDEEC77A17EE907A17EE906AA742A8BFA6
:1040900026469F42B8BF1E4607EE906AF8EEE77AC2
:1040A0000B2AC1ED0A7A3FF467AE90ED2C7ADDED74
:1040B000177AE7EE067AA4EE275AFDEEC57A17EED8
:1040C000900A8442A8BF04468342D8BF234607EE25
:1040D000903AF8EEE77AC1ED0B7A4AE607EE902ABD
:1040E000F8EEE77A154FDFF860E097ED005A9EEDA5
:1040F000003A134F8BED7B3A77EE677A06EE905AD3
:10410000BCEEC77AF8EEE66A17EE102A77EEE67A8A
:104110008BED7C5AABF8E821D7ED006AFEF7DDBDE8
:1041200008494A69002A3EF4B2AA0A6813604B742F
:10413000FEF7ADBA184E00205C440020D84E002097
:10414000E84E00203CC700207441002007EE103AE2
:104150009AF800305B4FCBF8A061B8EEC77AF7EE63
:10416000006A132B86EE879AB7F90400BBF8A461A6
:1041700094ED080A01F01F84534B544A93ED001A42
:1041800093ED093A93ED162A93ED1F6AD3ED0B1ABE
:1041900093ED144AD3ED015AD3ED0A3A93ED0C7A1C
:1041A00093ED155AD3ED172AD3ED206AD3ED044AC7
:1041B000D3ED030A69EE277A69EE288A29EE088A88
:1041C000A7EE813A02EB860E0021A2EE286ACBF818
:1041D0009411CBF89811A8EE214AE7EEA53AA8EE83
:1041E000075A93ED1A7AD3ED0F5A93ED021AD3EDD5
:1041F0000E1A8EED003AE2EEA86A64EEC34A27EE8C
:10420000467A93ED0D2AD3ED192A8EED204AE3EE7E
:10421000603A65EEC45A93ED183AC3ED093AE7EEF9
:10422000814AF0EE477AA4EE615AE8EE025AE2EED5
:10423000C66AE3EE287AC3ED0A4A83ED145AC3ED49
:10424000155A8EED406AC3ED1F6AC3ED207ACBF894
:104250009C11731C03F01F03ABF8A431B880FEF768
:1042600014B91B4A107900283EF4B5AD19480078FE
:1042700000283EF4B0AD12789FED172A07EE102A01
:10428000164A07EE900A1288F8EEE77A03EE902AB3
:10429000B8EE477AF8EE633A27EE277AF7EE002A6F
:1042A000C7EE237AF4EEC27AF1EE10FA88BFF0EE90
:1042B000427AF4EEE27AF1EE10FAB8BFF0EE627AEA
:1042C000FEF78BBDE4CE002074870020D884002048
:1042D0005C250020CFCF0020713DAA3F88CF002071
:1042E0000000000090ED027A90ED012AD0ED037AF3
:1042F0005FED052A26EE877AA5EE827AA7EEA47AEC
:1043000027EE237AB4EEE27AF1EE10FAB4BFF0EEC3
:10431000627AF0EE477A8DED0C7A88BFB0EE627A61
:10432000012A3EF45EAFD0ED062AD0ED051A90EDDD
:10433000072A66EEA22AE5EEA12AE2EE242A62EE20
:10434000A32AF4EEC72AF1EE10FAF4EEE72A8CBFA6
:10435000B0EE472AB0EE622AF1EE10FA98BFB0EE46
:10436000427AA8BFF0EE627A022ACDED0D2A3EF421
:1043700038AFD0ED0A2AD0ED091A90ED0B2A66EE7F
:10438000A22AE5EEA12AE2EE242A62EEA32AF4EEA6
:10439000C72AF1EE10FAF4EEE72A8CBFB0EE472AF6
:1043A000B0EE622AF1EE10FA98BFB0EE427AA8BFE2
:1043B000F0EE627A032ACDED0E2A3EF412AFD0ED74
:1043C0000E2AD0ED0D1A90ED0F2A66EEA22AE5EE28
:1043D000A12AE2EE242A62EEA32AF4EEC72AF1EE25
:1043E00010FAF4EEE72A8CBFB0EE472AB0EE622A4C
:1043F000F1EE10FA98BFB0EE427AA8BFF0EE627A02
:10440000042ACDED0F2A3EF4ECAED0ED122AD0ED09
:10441000111A90ED132A66EEA22AE1EEA52AE2EE29
:10442000242A62EEA32AF4EEC72AF1EE10FAF4EE83
:10443000E72A8CBFB0EE472AB0EE622AF1EE10FAFE
:1044400098BFB0EE427AA8BFF0EE627A052ACDEDB1
:10445000102A3EF4C6AED0ED162AD0ED151A90ED16
:10446000172A66EEA22AE1EEA52AE2EE242A62EEDF
:10447000A32AF4EEC72AF1EE10FAF4EEE72A8CBF75
:10448000B0EE472AB0EE622AF1EE10FA98BFB0EE15
:10449000427AA8BFF0EE627A062ACDED112A3EF4E8
:1044A000A0AED0ED1A2AD0ED191A90ED1B2A66EEB7
:1044B000A22AE1EEA52AE2EE242A62EEA32AF4EE75
:1044C000C72AF1EE10FAF4EEE72A8CBFB0EE472AC5
:1044D000B0EE622AF1EE10FA98BFB0EE427AA8BFB1
:1044E000F0EE627A072ACDED122A3EF47AAED0EDD4
:1044F0001E2AD0ED1D1A90ED1F2A66EEA22AE1EECB
:10450000A52AE2EE242A62EEA32AF4EEC72AF1EEEF
:1045100010FAF4EEE72A8CBFB0EE472AB0EE622A1A
:10452000F1EE10FA98BFB0EE427AA8BFF0EE627AD0
:10453000082ACDED132A3EF454AED0ED222AD0ED58
:10454000211A90ED232A66EEA22AE1EEA52AE2EED8
:10455000242A62EEA32AF4EEC72AF1EE10FAF4EE52
:10456000E72A8CBFB0EE472AB0EE622AF1EE10FACD
:1045700098BFB0EE427AA8BFF0EE627A092ACDED7C
:10458000142A3EF42EAE90ED262AD0ED251AD0ED59
:10459000272A26EE822AA1EEA52AA2EEA42A22EE3E
:1045A000232AB4EEC72AF1EE10FAB4EEE72A8CBF44
:1045B000F0EE472AF0EE422AF1EE10FA8DED152AC0
:1045C00098BFB0EE627AB8BFB0EE672A0A2A01F04F
:1045D000CA87D0ED2A7AD0ED291AD0ED2B2A66EEC3
:1045E000A77AE1EEA57AE2EEA47A67EEA37AF4EE7A
:1045F000C77AF1EE10FAF4EEC27A8CBFF0EE472AD9
:10460000F0EE672AF1EE10FA98BFB0EE627AA8BF1A
:10461000B0EE672A0B2ACDED167A01F0A487D0ED13
:104620002E7AD0ED2D1AD0ED2F2A66EEA77AE5EE80
:10463000A17AE4EEA27A67EEA37AB4EEE77AF1EE1D
:1046400010FAB4EEE72A8CBFF0EE676AF0EE476A24
:10465000F1EE10FACDED177A58BFB0EE667AA8BF2A
:10466000F0EE427AFEF7BDBDABF84851B8F1000F4D
:1046700000F07881D2490220D24ADFEDD36AD2F825
:1046800000E09AF800C09EF800209EF8028007EE35
:10469000902AF8EEE77AB0EE007A67EEA67AF4EEAA
:1046A000C77AF1EE10FA40F3D38237EEC77ADFED26
:1046B000C76AB0EE676AA7EE266AB0EE467A9FED4B
:1046C000C46AD1ED006A66EE866AB0EEE66ACBEDAA
:1046D0005B6A8BED5E6AB8F1000F13D005EE908A2D
:1046E000B8EEE55ADFEDB85A66EEA64A25EE255A31
:1046F000F7EE005A75EEC55A64EE864AE5EE245A86
:1047000066EEA56ADFEDB35A9EF8052027EE257AFE
:1047100027EE267ACAB1DFEDAC6ADFEDAF5A26EE9E
:10472000266A06EE902AF8EEE66A66EE866AF4EEEF
:10473000E56AF1EE10FA00F3BA85F7EE005A75EE6D
:10474000E66A85EEA66A27EE067ABCF10C0F9FEDAD
:10475000A38ADFEDA36A00F07E85B4EEC87AF1EE9D
:1047600010FA98BFB0EE478AB4EEE68AF1EE10FA7E
:10477000B8BFB0EE668A8BED418A002800F0E68073
:10478000B0EE007AF4EEC77AF1EE10FA05DD37EEFE
:10479000C77ADFED8E6AE7EE267A91ED017ADFEDDA
:1047A0008C6A27EE267AB0EEC76A8BED5C7A8BEDC9
:1047B0005F6AB8F1000F13D006EE908ADFED825ADF
:1047C000F8EEE66A27EE075A66EEA56AF7EE005A9B
:1047D00075EEE65A25EE065AE6EE855A27EE257A5C
:1047E000DFED7C6A9EF8062067EEA67A67EE877A90
:1047F000AAB107EE102AB8EEC77ADFED735ADFEDE3
:10480000766A27EE067A27EE257AB4EEE67AF1EE9E
:1048100010FA40F35085DFED736A67EEA67ABCF1BB
:104820000C0F00F0F984DFED6D6A9FED6D7AF4EE08
:10483000E67AF1EE10FA88BFF0EE667AF4EEC77A07
:10484000F1EE10FAB8BFF0EE477A0128CBED427ACC
:104850007CDD9EF80120DFED5C6A07EE902AF8EE21
:10486000E77AB0EE007A67EEA67A9EF80920F4EEB9
:10487000C77AF1EE10FA05DD37EEC77ADFED536A3D
:10488000E7EE267A91ED027ADFED516A27EE267A7D
:10489000B0EEC76A8BED5D7A8BED606A9AB106EE79
:1048A000902ADFED495AF8EEE66A27EE075A66EEDF
:1048B000A56AF7EE005A75EEE65A25EE065AE6EEC0
:1048C000855A27EE257ADFED436A9EF8072067EECA
:1048D000A67A67EE877A0AB307EE102AB8EEC77A8F
:1048E000DFED395ADFED3C6A27EE067A27EE257AAE
:1048F000B4EEE67AF1EE10FA0CDCB5EEC07AF1EE29
:1049000010FA01F15C81B7EE006A36EE477AC6EE26
:10491000076A01E0DFED336A67EEA67ABCF10C0F9F
:1049200000F0B484DFED2D6A9FED2D7AF4EEE67A87
:10493000F1EE10FA88BFF0EE667AF4EEC77AF1EE87
:1049400010FAB8BFF0EE477ACBED437ABCF1090F0D
:1049500000F0598493F82150002D40F00C8400237E
:104960008BF81831204B1B68990609D51F4B1B8803
:1049700003F0300323B11E4B1B78DA0701F1F785F2
:1049800012F09EFD002840F03D811A4B1B7823B9A0
:10499000194B9B78002B41F07481089804F0CEFEEF
:1049A0009AF80030072B00F079840022072B8BF84F
:1049B00000217DF419ADFDF775FB0390FDF716BDE1
:1049C000D0CF0020442700200AD7233CD7A368413A
:1049D0006F12033B00004843A4707D3F00C0F944C0
:1049E00000C0F9C40000C842B08400203C27002069
:1049F0006A2500207C6A002018C80020A94A099274
:104A00002A460026CDF810B0A74FDFF8A882DDF8BF
:104A100024B035469146B7EC018AD4ED087AB8EE59
:104A2000C88A28EE278A002D02F0D3836BBB9AF840
:104A30000030082B39D006F5D260B0EE480A204489
:104A4000D4F88C36984706F5E360D4F81437204440
:104A500098479AF80030032BB0EE408A20D0D4F863
:104A6000AC30D7F84406B0EE480A98470BEB850304
:104A70000135032D06F12C0683ED010A3DF428AD26
:104A8000D9F8003003F00053C5E706F5F460B0EE46
:104A9000480A2044D4F89C379847B0EE408AC6E7CD
:104AA00026F08AFF28F81500D9E7B0EE480A26F06C
:104AB00083FF28F81500BEE77C4BDFF824B21A68A4
:104AC0007B4B7C4F9BF80001D2691B883A807B802E
:104AD00000287EF4C8AF0390774CFDF787BCDFED6C
:104AE000776AFEF7D0B8FDF7DDFA039A714B801AAA
:104AF000D880FEF7BFBDDFF8EC91DBED017A9BEDCE
:104B0000006AB9F80000D9F8143077EEA77AF0EE11
:104B1000006AB0EE677AA6EE267A01380BEBC00287
:104B2000D6EE267A083A1033F6EE003A27EE237ACC
:104B300067EEA37A8BED207ACBED217ADFF8A0B176
:104B40005F460BF1800192ED027A92ED036AD7ED98
:104B5000036AD7ED027A53ED014A13ED025A37EE9C
:104B6000674A76EEC65A77EE277AE4EE845A013821
:104B7000A2F10802E5EE047A07F1080703F1080341
:104B800036EE267A01F10801E4EE877AE5EE475A1F
:104B900067EEA37A25EEA37AC1ED007A81ED017A62
:104BA000D1D1B8F1140F07D1FDF77CFA049B414F26
:104BB000C01A7880DBF8A8613A4B0993404A2B6809
:104BC000013682FB06129119F217C2EBA102C2EB69
:104BD000C202B61ACBF8A86103F0005310E7FDF744
:104BE00061FA9AF800300B9A324F801A012B7880C4
:104BF00000F0D780072B7DF4FFADFDF753FA03904B
:104C0000FDF7FCBD2F4D12F017FB6B78022B01F066
:104C1000A482032B7FF4B9AE41F2B813EB5C002BF6
:104C200042F04A8041F2A403EB5C002B42F03F804B
:104C300041F2E803EB5C002B42F0348041F22C138C
:104C4000EB5C002B3FF4A1AE1F4822F04BFA9CE630
:104C5000B0EE677A33E51D4F97ED007AFEF7E7BFB8
:104C60001B4D1C4F1C4A95ED005A97ED003A1B4D09
:104C700012788BED7B3A8BED7C5AD5ED006A12B140
:104C800001228BF8F821DBED7D7AFEF726B8A368C8
:104C9000002B3EF4EFAE04F1440120469847FEF7A6
:104CA000E9BE00BF9C840020B07C002024C9002005
:104CB0000A410020E4CE0020787C002000000000A3
:104CC000932449927CA30020A8B4002000C40020B3
:104CD00070410020DC4E0020ACBB0020E44E0020E0
:104CE000A4290020C084002038493948D1F8EC10AC
:104CF000076844F620608142A8BF0146B1F57A7F7B
:104D0000B8BF4FF47A7188B2FF06ABF81A01296870
:104D100041F14883C90440F151832E49D1F800C0C4
:104D2000BCF836707F082C492C4DD1ED037ADBF8A6
:104D30001C11A5FB00508509642090FBF5F0142898
:104D4000BDEEE77A0BEB410EA8BF14200131814282
:104D5000CBF81C1117EE109AA4BF0021CBF81C1140
:104D60000BEB4101AEF82091B1F9201107EE101ABA
:104D7000B8EEC77A77EEC77AFDEEE77ACDED037A23
:104D8000BDF90C0080EAE071A1EBE071B94201F3DA
:104D9000B487134908464FF07E510160FEF77FBE8D
:104DA000104FFDF77FF9104ADBF8E43112680390E9
:104DB000C31A9A1ACBF8E401BB80FA80FDF71EBD36
:104DC000FDF770F90B90FDF79FBB00BFDC160020CC
:104DD0004CC8002040270020D0CF0020D34D6210C7
:104DE00098000020E4CE0020D0460020B9F1000F4A
:104DF0003EF467ACF4EEC57AF1EE10FAB8BFF0EE0F
:104E0000667AFDEEE77ABDEEE67A17EE907A17EE57
:104E100090EAA74217EE106AA8BFA646BE42C8BFD6
:104E2000B64607EE90EAF8EEE77A012AC1ED007A7D
:104E30003EF4E7AB90ED047ADDED0D7AE7EE067A0D
:104E4000B0EE437AA4EE277AB4EEC57AF1EE10FA0A
:104E5000F0EE477AB8BFF0EE667AFDEEE77A17EE2D
:104E6000907A17EE90EAA742A8BFA646B742B8BF0D
:104E7000B64607EE90EAF8EEE77A022AC1ED017A2B
:104E80003EF4BFAB90ED087ADDED0E7AE7EE067AE0
:104E9000B0EE437AA4EE277AB4EEC57AF1EE10FABA
:104EA000F0EE477AB8BFF0EE667AFDEEE77A17EEDD
:104EB000907A17EE90EAA742A8BFA646B742B8BFBD
:104EC000B64607EE90EAF8EEE77A032AC1ED027AD9
:104ED0003EF497AB90ED0C7ADDED0F7AE7EE067AB3
:104EE000B0EE437AA4EE277AB4EEC57AF1EE10FA6A
:104EF000F0EE477AB8BFF0EE667AFDEEE77A17EE8D
:104F0000907A17EE90EAA742A8BFA646B742B8BF6C
:104F1000B64607EE90EAF8EEE77A042AC1ED037A86
:104F20003EF46FAB90ED107ADDED107AE7EE067A85
:104F3000B0EE437AA4EE277AB4EEC57AF1EE10FA19
:104F4000F0EE477AB8BFF0EE667AFDEEE77A17EE3C
:104F5000907A17EE90EAA742A8BFA646B742B8BF1C
:104F6000B64607EE90EAF8EEE77A052AC1ED047A34
:104F70003EF447AB90ED147ADDED117AE7EE067A58
:104F8000B0EE437AA4EE277AB4EEC57AF1EE10FAC9
:104F9000F0EE477AB8BFF0EE667AFDEEE77A17EEEC
:104FA000907A17EE90EAA742A8BFA646B742B8BFCC
:104FB000B64607EE90EAF8EEE77A062AC1ED057AE2
:104FC0003EF41FAB90ED187ADDED127AE7EE067A2B
:104FD000B0EE437AA4EE277AB4EEC57AF1EE10FA79
:104FE000F0EE477AB8BFF0EE667AFDEEE77A17EE9C
:104FF000907A17EE90EAA742A8BFA646B742B8BF7C
:10500000B64607EE90EAF8EEE77A072AC1ED067A8F
:105010003EF4F7AA90ED1C7ADDED137AE7EE067AFE
:10502000B0EE437AA4EE277AB4EEC57AF1EE10FA28
:10503000F0EE477AB8BFF0EE667AFDEEE77A17EE4B
:10504000907A17EE90EAA742A8BFA646B742B8BF2B
:10505000B64607EE90EAF8EEE77A082AC1ED077A3D
:105060003EF4CFAA90ED207ADDED147AE7EE067AD1
:10507000B0EE437AA4EE277AB4EEC57AF1EE10FAD8
:10508000F0EE477AB8BFF0EE667AFDEEE77A17EEFB
:10509000907A17EE90EAA742A8BFA646B742B8BFDB
:1050A000B64607EE90EAF8EEE77A092AC1ED087AEB
:1050B0003EF4A7AA90ED247ADDED157AE7EE067AA4
:1050C000B0EE437AA4EE277AB4EEC57AF1EE10FA88
:1050D000F0EE477AB8BFF0EE667AFDEEE77A17EEAB
:1050E000907A17EE90EAA742A8BFA646B742B8BF8B
:1050F000B64607EE90EAF8EEE77A0A2AC1ED097A99
:105100003EF47FAA90ED287ADDED167AE7EE067A76
:10511000B0EE437AA4EE277AB4EEC57AF1EE10FA37
:10512000F0EE477AB8BFF0EE667AFDEEE77A17EE5A
:10513000907A17EE90EAA742A8BFA646B742B8BF3A
:10514000B64607EE90EAF8EEE77A0B2AC1ED0A7A46
:105150003EF457AA90ED2C7ADDED177AE7EE067A49
:10516000A4EE273AB4EEC35AF1EE10FAC8BFB0EE7F
:10517000663AFEF7FCBB1E219E48F5F715FC002899
:105180003FF4EDAB9C4B1B8858063FF5E8AB9BF812
:105190008431AB4241F04A86984BDBED627A93ED65
:1051A000017A9BED435ADFED965A9FED966A67EEC2
:1051B000C56A67EE887AE7EE086AE5EE077AF4EEEC
:1051C000E56AF1EE10FA8CBFB0EE657AB0EE667A61
:1051D000B4EEC67AF1EE10FAF4EEE57AB8BFB0EEAE
:1051E000467AF1EE10FA88BFF0EE657AF4EEC67AF0
:1051F000F1EE10FAB8BFF0EE467A8BED417ACBEDC6
:10520000437AFFF7ACBBFDEEC87A7F4F17EE902ACA
:10521000BD80FA80FFF79EBB9FED797ADFED796A5A
:10522000794FF4EEC77AF1EE10FA98BFB0EE677AD4
:10523000FDEEE77AB4EEE67AF1EE10FA17EE902A78
:10524000B8BFB0EE667A01288BED427A7A803FF7DC
:1052500000ABFFF77FBBB4EEC87AF1EE10FA98BF4F
:10526000B0EE478ABDEEC77AB4EEE68A664FF1EE3D
:1052700010FA17EE102AB8BFB0EE668A8BED418A9D
:105280003A8000287FF47CAAFFF764BBBDEEE77A82
:105290005D4F17EE102ABA80FFF744BBFCF702FF00
:1052A000594F9AF80030801BB880FFF77EBB9FED06
:1052B000576AFFF748BAB5EEC07AF1EE10FA00F17E
:1052C0007A84B7EE006A36EE477AC6EE076AFFF7D1
:1052D000A4BAFDEEC57A0CA817EE907AFDEEE67A38
:1052E00000EB82030493DFF83081DFF830E1CDF882
:1052F00018B04FFA89F317EE906AB1EE444A89F07C
:10530000010C05929B46434693ED007AF0EC017A3E
:10531000E7EE067A09F0010308F11008B0EE437ACF
:10532000A4EE277AB4EEC75AF1EE10FAD8BF0023E4
:10533000002BF0EE477A18BFB0EE667ABDEEC77A62
:10534000FDEEE77A17EE102A17EE901AA24217EE3A
:10535000103AA8BF23469642CCBF002209F00102B2
:10536000002A08BF3346A14217EE902A07EE103AF2
:10537000A8BF22468F42CCBF00230CF00103002BB4
:1053800008BF3A4607EE902AB8EEC77AF8EEE77AF9
:10539000049BBBF1000F18BFF0EE477A9842EEEC89
:1053A000017AB0D1FEF7E2BC93F82010C1EB4110B6
:1053B00001EB8001C90089B2FEF77DBB1449D1F829
:1053C00000C0BCF93670AEE4DFF854901148D9F84B
:1053D0000820B9F80C1025F0ABFA9AF80080B8F163
:1053E000140F01F0AC85DBF8A8610136CBF8A86199
:1053F000FFF783BB4CC800203C270020980000200A
:1054000000C0F94400C0F9C4E4CE00200000C84246
:1054100040270020A4290020184E00205C440020D2
:10542000C0840020DFF86493B9F80070D9F804E074
:105430004FEA570C4FEA8C020BEB8708FF080BEB87
:10544000020300F09F8010320137C54803EB0717B5
:10545000424410330EF1100608F1100151ED032AF9
:1054600051ED043A10ED043A10ED032A51ED026AB1
:1054700011ED016A10ED020A10ED018A12ED044AE5
:1054800012ED035A53ED044A53ED035A13ED027A19
:1054900053ED017A52ED020A12ED011A73EE238ADE
:1054A00072EE221A40ED048A40ED031A70EE268A4D
:1054B00078EE061A40ED028A40ED011A74EE848AF5
:1054C00075EE851A43ED048A43ED031A77EE208AC0
:1054D00077EE811A43ED028A43ED011A73EE633AC7
:1054E00075EE655A16ED035A32EE623A74EE644A6E
:1054F00065EE631A16ED044A23EE052A64EE652A6A
:10550000E3EE041A1033BB4224EE843AA3EE842A5D
:1055100000F1100006F11006A5EE853A01F1100128
:1055200002F11002E4EE852A41ED071A01ED082A86
:1055300002ED073A42ED082A56ED055A16ED065AD5
:1055400070EE666A38EE466A30EEC77A71EE677AB8
:1055500026EE253A65EEE63A25EE674A67EE054AFD
:10556000E6EE053AA6EE853AA7EE254AE7EEA54A0D
:1055700001ED063A41ED053A02ED064A42ED054AD3
:105580007FF46CAF1FFA8CF672463146754818F0FE
:1055900005FC3146D9F80420404618F0FFFB9AF884
:1055A0000030142B7FF406ABFFF7FEBA6E4BDBF82E
:1055B000ACC10993BBF8A491C9F12003D8B26B4BDD
:1055C00009EB4C1703EB8707830801F0D7830133FE
:1055D0001B016749624A059307EB030E07F11003AD
:1055E00013ED024A13ED035A13ED016A13ED047A29
:1055F00051ED024A51ED035A51ED016A51ED047A21
:1056000064EE244A65EE255A66EE266A67EE277A2E
:105610001033734542ED024A42ED035A42ED016AEE
:1056200042ED047A01F1100102F11002D8D1059B7C
:105630005049A3F11002174401EB020E5A4410F036
:10564000030309D0B7EC017AFEEC017A67EE277A02
:10565000013BE2EC017AF5D1B9F1000F41F0FC8198
:10566000B8F1140F7FF4AAAAFCF71CFD049B424F6B
:10567000DBF8A861C01A7880FFF7A0BADBF8AC911C
:10568000394A3E4B099203EBC903126805929DED1E
:10569000057A9B88DFED3A7A3A4AF8EE478A09EEB6
:1056A000103A643BC82BA8BFC82368EEA78AF8EE5F
:1056B000497A782BB8BF782368EEA78A07EE903A2C
:1056C0002C27B0EE680A07FB0927B8EEE78A26F018
:1056D000BFF9B8EEC99AF0EE409AB0EE680A26F02B
:1056E00019F938EE097A79EE487A28EE098A67EED8
:1056F000877AB7EE006A88EE277AB8F1140FF8EED1
:10570000007A77EE076A60EE277A89EEA67A77EE5E
:10571000065A36EE477AC6EE256A67EEA67A27EE77
:10572000267AC7ED006A87ED047AC7ED026AC7EDF5
:10573000017AC7ED037A01F0F683134B9AF80080E3
:1057400009F1010983FB093CACEBE97C0CEB4C0C47
:105750000136A9EB0C0CCBF8A861CBF8ACC129E75A
:10576000B4290020A42900209C840020D884002093
:105770006886002058860020E4CE0020D8860020CD
:1057800027D4D2361884002056555555C0840020A1
:10579000DFF8409499F800205FEA920C01F027842A
:1057A000DFF86CE40CF1010040010EEB00070EF194
:1057B0002003AEF1700113ED076A53ED056A13ED96
:1057C000037A53ED017A53ED025A13ED084A53ED73
:1057D000064A13ED045A26EE066A66EEA66A27EE1E
:1057E000077A67EEA77AA4EE046A2033BB42E4EEA0
:1057F000A46A01F11001A5EE057AE5EEA57AF1EEB5
:10580000C65AB1EEE66AF1EEC76AB1EEE77A41ED4B
:10581000085A01ED076A41ED066A01ED057ACAD121
:10582000203886440BEB0C1112F0030318BF0EF165
:10583000080E0FD05EED017A1EED027A67EEA77AB0
:10584000013BE7EE077A0EF1080EB1EEE77AA1EC24
:10585000017AEFD1B8F1140F01F057830136CBF87C
:10586000A86101E0DB4B1A78DBF8ACE1DA489FED88
:10587000DB7A4FEACE07C31983ED007A002A7BD08A
:10588000D749B0EE476AF0EE476A0023F1EC017A9F
:10589000013367EEA77A05EE903AB4EEE77AF1EEBF
:1058A00010FAF8EEE55AB8BFB0EE677A934276EE9A
:1058B000A76AA7EEA56AE9D1F5EEC06AC319F1EEB1
:1058C00010FA83ED007A57DDC6EE265AC54BC64A5C
:1058D0001288F7EE007A75EEE75AD3ED007A65EE9E
:1058E000A77AFDEEE77A17EE903A812B41F3948088
:1058F0009342A8BF134607EE903AF8EEE77ABB4B07
:105900002C2101FB0E3393ED097AD3ED003A93ED90
:105910000A6A93ED014AD3ED046AD3ED034A93ED8D
:10592000025AA3EEA77AA4EE276A66EEC76AA7EE2C
:10593000646ABDEEC77AE5EE276A17EE101A812970
:1059400083ED096AC3ED0A6A41F363808A42A8BF06
:105950000A4607EE902AF8EEE77AFCEEE77ACDEDFC
:10596000057ABDF81430C2199380BEF1000F03D13F
:10597000B8F1130F01F0EA81B8F1150F7FF411A906
:1059800038449B4F838827F81E309A4BDBF8A86178
:105990000993FFF713B9FCF785FB9AF80080049090
:1059A000B8F1140F05BF924FDBF8A861DBF8A861CE
:1059B0003E80FCF774BDDFF85C82DFF85C9298ED06
:1059C000004A98ED097AD8ED014A98ED0A6AD8EDB7
:1059D000046A98ED035AD8ED025A69EE277A09EB6A
:1059E0008603A7EE847AA7EEA46A66EEC76AA7EEDE
:1059F000456AE7EEA56A20EE070A88ED096AC8ED58
:105A00000A6A29EE088A69EE288A83ED007A25F071
:105A1000D3FFD8ED145AD8ED1F6A98ED0B1AD8EDC4
:105A2000161A98ED155A98ED207A98ED0C2AD8EDB3
:105A3000172A98ED0F6AD8ED1A7A98ED0E3AD8ED3C
:105A40000D3A98ED194AD8ED184AE8EE015A0021AE
:105A500009EB8602E8EEA16A00B2CBF89411A8EE39
:105A6000025ACBF89811CBF89C11A8EEA27A26EE38
:105A7000656A67EEE67AA5EEC35AA8EE236AA6EE3B
:105A8000C47AE8EEA47A88ED145AC2ED205A88ED63
:105A9000156AC2ED406A88ED1F7AC8ED207AFEF7DC
:105AA000D8BBB4F92430E26207EE903A0122F8EE56
:105AB000E77A2366E2670023012EC4ED1C7AC4ED69
:105AC0001B7A636701F03E81AE427CF474AFB4F997
:105AD0002630636607EE903A00220123F8EEE77A5B
:105AE0002263C4F890300023012EC4ED217AC4ED66
:105AF000207AC4F8883001F02181AE427CF48BAF6B
:105B0000B4F92830A36607EE903A00220123F8EE9C
:105B1000E77A6263C4F8A4300023012EC4ED267A2C
:105B2000C4ED257AC4F89C307CF4A5AF9FED2B8A98
:105B3000B8F1030F47D0B9F1000F09D007EE909AE2
:105B4000F8EEE77AF4EEC87AF1EE10FA01F160822D
:105B5000294AA36E12689BF8B011F88003EB550335
:105B600093FBF5F50023656393621363D36221B160
:105B7000224B1B88002B7CF47FAF214B1B6813F456
:105B8000003304D01F4B1B79002B41F026821E48A6
:105B90001A46C15C012903F10C0300F04187013270
:105BA000152AF6D1FCF768BF184A927B002A3EF40A
:105BB0007EA8FDF765BFF7EE006AFEF72EBEF7EE92
:105BC000006AFEF7A9BEB0EE480A25F0F5FE00B265
:105BD000B1E700BFBA840020D88600200000000092
:105BE000A4290020BC840020B8840020F086002076
:105BF000E4CE00209C84002024C900203A27002005
:105C0000144800205C250020C8EA0308B0BA002030
:105C1000242A002074870020D8840020BBF8485133
:105C2000013D2DB2002DABF848517EF71FAD8649DE
:105C3000FDF793BFBBF81A1101F57A7189B2FDF730
:105C40003ABF8248DFED827A0068CBED707A10F0BF
:105C5000805000F0C983B7EE007A77EE677AF4EEF1
:105C6000C67AF1EE10FA88BFF0EE467AB0EE676AB7
:105C7000CBED7D7AFDF72BBB237803F00103FDF715
:105C8000C0BC089806F09EFFFEF787BE714ADFEDA4
:105C9000727A92ED080AB4EEE70AF1EE10FA40F2D9
:105CA000D786039325F01EFFDBED457A20EE270A09
:105CB00025F082FEB0F5617F039B00F3238707EE9A
:105CC000900AF8EEE76ADFED657A66EEA76A07EEFE
:105CD000907AB8EEE77AFDEEE67A17EE902A203257
:105CE000402A41F236819FED5E0A039325F064FE5F
:105CF00000B207EE900A039BB8EEE77A5249D1ED65
:105D0000037A77EE877AC1ED037AFDF7C1BE049B73
:105D1000002B00F01187FDEEE67A0CA901EB820260
:105D200017EE90CAFDEEC57A13464E484E4E4A46CF
:105D300017EE90EA994614E0FDEEC77A17EE908AC6
:105D4000C64503DCA0454346A8BF234607EE903A6C
:105D5000F8EEE77A4945E6EC017A00F110003DF4EF
:105D600053AC90ED007AF1EC017AE7EE067A7346D7
:105D7000B0EE457AA7EE847AF0EE477A002ADBD0BF
:105D800037B1B4EE475AF1EE10FAC8BFF0EE667ABA
:105D9000FDEEE77A634617EE908AC445D2DDD5E77B
:105DA000049B002B00F02087FDEEC57A0CA901EBC7
:105DB000820217EE90EAFDEEE67A134629482A4E53
:105DC0004A4617EE90CAB1EE444A994614E0FDEEF9
:105DD000C77A17EE903A734503DBA342A8BF234668
:105DE000984607EE908AF8EEE77A4945E6EC017AA4
:105DF00000F110003DF408AC90ED007AF1EC017A6E
:105E0000E7EE067AF046B0EE437AA4EE277AF0EE9B
:105E1000477A002ADBD0634637B1B4EE457AF1EE1B
:105E200010FA48BFF0EE667AFDEEE77A17EE908A38
:105E3000E04504DBA04517EE903AA8BF234607EEE5
:105E4000903AF8EEE77AD0E7D0CF00204CC8002097
:105E500000000080A44700208FC2753CD06D393A05
:105E600000000000184E00205C440020BDEEE67AE1
:105E700017EE106AB0EE457AA4EE277AF0EE477A74
:105E8000002F40F0FF83FDEEC77A17EE90EA17EE81
:105E9000907AA645A8BF27467645C8BF374607EE85
:105EA000907AF8EEE77A012AC1ED007A3DF4A9ABC9
:105EB00090ED047ADDED0D7AE7EE067AB0EE457AE4
:105EC000A4EE277AFDEEC77A17EE90EA17EE907AE5
:105ED000A645A8BF2746B645B8BF374607EE907A15
:105EE000F8EEE77A022AC1ED017A3DF48AAB90ED33
:105EF000087ADDED0E7AE7EE067AB0EE457AA4EE8A
:105F0000277AFDEEC77A17EE90EA17EE907AA6454B
:105F1000A8BF2746B645B8BF374607EE907AF8EED9
:105F2000E77A032AC1ED027A3DF46BAB90ED0C7A6F
:105F3000DDED0F7AE7EE067AB0EE457AA4EE277A29
:105F4000FDEEC77A17EE90EA17EE907AA645A8BF45
:105F50002746B645B8BF374607EE907AF8EEE77A9F
:105F6000042AC1ED037A3DF44CAB90ED107ADDEDDF
:105F7000107AE7EE067AB0EE457AA4EE277AFDEEC7
:105F8000C77A17EE90EA17EE907AA645A8BF274683
:105F9000B645B8BF374607EE907AF8EEE77A052A9D
:105FA000C1ED047A3DF42DAB90ED147ADDED117A5C
:105FB000E7EE067AB0EE457AA4EE277AFDEEC77AD0
:105FC00017EE90EA17EE907AA645A8BF2746B64589
:105FD000B8BF374607EE907AF8EEE77A062AC1EDA9
:105FE000057A3DF40EAB90ED187ADDED127AE7EE0E
:105FF000067AB0EE457AA4EE277AFDEEC77A17EE60
:1060000090EA17EE907AA645A8BF2746B645B8BFD6
:10601000374607EE907AF8EEE77A072AC1ED067A5E
:106020003DF4EFAA90ED1C7ADDED137AE7EE067AE7
:10603000B0EE457AA4EE277AFDEEC77A17EE90EA25
:1060400017EE907AA645A8BF2746B645B8BF374693
:1060500007EE907AF8EEE77A082AC1ED077A3DF468
:10606000D0AA90ED207ADDED147AE7EE067AB0EE54
:10607000457AA4EE277AFDEEC77A17EE90EA17EE7E
:10608000907AA645A8BF2746B645B8BF374607EE63
:10609000907AF8EEE77A092AC1ED087A3DF4B1AAC0
:1060A00090ED247ADDED157AE7EE067AB0EE457ACA
:1060B000A4EE277AFDEEC77A17EE90EA17EE907AF3
:1060C000A645A8BF2746B645B8BF374607EE907A23
:1060D000F8EEE77A0A2AC1ED097A3DF492AA90ED2A
:1060E000287ADDED167AE7EE067AB0EE457AA4EE70
:1060F000277AFDEEC77A17EE90EA17EE907AA6455A
:10610000A8BF2746B645B8BF374607EE907AF8EEE7
:10611000E77A0B2AC1ED0A7A3DF473AA90ED2C7A46
:10612000DDED177AE7EE067AA4EE275AFDEEC57A82
:1061300017EE900A8442A8BF0446B042A8BF264684
:1061400007EE906AF8EEE77AC1ED0B7AFDF759BADF
:10615000FBF7A8FF0646FDF787BCAB784FF00109B7
:10616000B046072B01F2D480DFE803F0A3BD5E52F6
:106170006B3C4604032346466B70FEF706BC2B6956
:106180000622652B4446AA70DDF80C8034D92A78A3
:10619000032A14BF6FF0FF026FF07F02A3F16503C3
:1061A00003EA020303F1010314BF4FF4807280225B
:1061B0009A422B6120D23A68EE6802329F199742C8
:1061C00002D31FF015FF2B69C34A6E60D16FAF6019
:1061D000490203FB01F30521166042F81C3C42F81A
:1061E000183CA970AA68BD49012020F0A5FC01282F
:1061F00041F06F800623AB700021B94820F010F801
:10620000012841F06680AB780133DBB2AB70A8E7C0
:1062100041F270134646EB5C002B3EF4B6ABB0483F
:1062200020F060FFFEF7B1BBAE4B00930320A870D7
:1062300030230522AC49AA48464620F0EBFBFEF786
:10624000A4BB2A782B7DA94FCDF80C80032A14BF5C
:106250004FF480768026A046002B79D0012BFBD10D
:10626000A34BD5F804E0D3F800C03A684FF0FF33F1
:1062700000244FEA4C2CB3FBFCFC1CEB0E0044F159
:1062800000010024A14202F1020208BF904238BF7F
:106290000EEB0C029749022010F0EAFE032800F2F0
:1062A000A386DFE800F0023F023F039E4446FEF76C
:1062B0006CBB002346460DF13008414618460922C2
:1062C00010F096FD01287EF460AB0C9B93F8FE2144
:1062D000552A00F0A28641F2B41202210123A954EA
:1062E0006B70FEF752BB46460DF1300841F2FC17C9
:1062F0004146E8590023092210F07AFD01287EF476
:1063000044AB00230C992B70B1F80B30B3F5007F30
:1063100000F07C8741F2B41203210123A9546B7071
:10632000FEF733BB6C68AB682A69191B914284BFC6
:10633000EC60296103283FF422AF0133B3FBF6F28E
:1063400006FB12320AB133449B1A00226B602A7595
:106350003A6862490232002010F08AFE032800F2F7
:10636000438601A353F820F0AB620108796301086A
:10637000AB6201087F6101086B6885F814900133F6
:10638000AB606DE75C48006810F080502CD0B6EE32
:10639000007A67EE877AF4EEC67AF1EE10FA3FF7EC
:1063A00065AC58E4CD003EF5B5ACFDF778BB534D78
:1063B000534F544A95ED005A97ED003A524D1278DA
:1063C000CBED7D7A8BED7B3A8BED7C5AD5ED006A77
:1063D000002A3CF482AC01228BF8F821FCF77DBC4A
:1063E000F0EE637AFCF7FDBE11F4800001D00020CE
:1063F000CDE7B6EE007AB4EEC76AF1EE10FAC6DC6D
:10640000FCF765BFFDEEE67A0CAB4049DFF800E132
:1064100017EE906A03EB820CD1ED007AB3EC017AAF
:10642000A7EE867A1031F0EE455AE4EE075A07EEF1
:10643000906AB0EE657A37B1B4EE655AF1EE10FAB3
:10644000C8BFB0EE667ABDEEC77A17EE100A864274
:1064500004DCA042A8BF204607EE900AF8EEE77AD7
:106460009C45EEEC017AD7D1FDF783BC012A7FF77A
:106470005DAB07EE101AB8EEC77AC7EE876AB1EEC9
:10648000E68AFFF755BB012A40F3588407EE101A3D
:10649000B8EEC77AC7EE876AB1EEE68AB8F1030FA5
:1064A00014D0B9F1000F09D007EE909AF8EEE77A10
:1064B000B4EEE78AF1EE10FA00F3AA85636E03EBFF
:1064C000550393FBF5F32363FFF717BBB0EE480AC0
:1064D00025F072FA00B2E4E710B5002080A3002096
:1064E000ECB400205D5F0308100D040884B50020A3
:1064F0008CB5002084A300204CC8002070410020EF
:10650000DC4E0020ACBB0020E44E0020184E0020E2
:106510005C440020012A40F3158407EE101AB8EEFF
:10652000C77AC7EE876AB1EEE68AB8F1030F14D0D6
:10653000B9F1000F09D007EE909AF8EEE77AB4EEC1
:10654000E78AF1EE10FA00F36385236E03EB55033F
:1065500093FBF5F3E362FFF7B7BAB0EE480A25F014
:106560002BFA00B2E4E7F0EE427AFCF73ABE3D4B7C
:106570003D4AB3F90430DFED3D7A82FB0312DB17AD
:10658000C3EBA2031BB208EE103AB8EEC88A28EE9D
:10659000278AB0EE480AF4F72FF9F0EE408AB0EE01
:1065A000480AF4F7AFF8324BD878002800F0898316
:1065B000304ABBF98E11B2F9023044F250655B1AD1
:1065C000AB4200F3D1832C4DAB42BCBF03F50C436F
:1065D000A03345429D4200F3CF838342A8BF0346C8
:1065E000B2F90020BBF98C711944D31B44F25062FC
:1065F00009B29342ABF88E1100F3BA831E4A93425C
:10660000BCBF03F50C43A0339D4203DC9842A8BFF6
:10661000184605467B191BB207EE903A07EE101A92
:10662000F8EEE77AF8EEC76A27EEE87A60EE277AA6
:10663000A0EE267AABF88C31E8EEA67ADFED0F6A91
:1066400027EE267A67EEA67ABDEEC77AFDEEE77AE8
:1066500017EE102A17EE903AABF89021ABF8923172
:10666000FEF78EB9542500206766666635FA8E3CC3
:10667000106800206C680020B0B9FFFFCDCCCC3D85
:1066800000000243B4EEC57AF1EE10FAB8BFF0EEA6
:10669000667AFDEEE77A17EE907A17EE90EAA74257
:1066A000A8BFA646BE42C8BFB64607EE90EAF8EEBF
:1066B000E77A012AC1ED007A3CF4A3AF90ED047AA9
:1066C000DDED0D7AE7EE067AB0EE457AA4EE277A94
:1066D000B4EEC57AF1EE10FAF0EE477AB8BFF0EEFC
:1066E000667AFDEEE77A17EE907A17EE90EAA74207
:1066F000A8BFA646B742B8BFB64607EE90EAF8EE86
:10670000E77A022AC1ED017A3CF47BAF90ED087A7A
:10671000DDED0E7AE7EE067AB0EE457AA4EE277A42
:10672000B4EEC57AF1EE10FAF0EE477AB8BFF0EEAB
:10673000667AFDEEE77A17EE907A17EE90EAA742B6
:10674000A8BFA646B742B8BFB64607EE90EAF8EE35
:10675000E77A032AC1ED027A3CF453AF90ED0C7A4C
:10676000DDED0F7AE7EE067AB0EE457AA4EE277AF1
:10677000B4EEC57AF1EE10FAF0EE477AB8BFF0EE5B
:10678000667AFDEEE77A17EE907A17EE90EAA74266
:10679000A8BFA646B742B8BFB64607EE90EAF8EEE5
:1067A000E77A042AC1ED037A3CF42BAF90ED107A1E
:1067B000DDED107AE7EE067AB0EE457AA4EE277AA0
:1067C000B4EEC57AF1EE10FAF0EE477AB8BFF0EE0B
:1067D000667AFDEEE77A17EE907A17EE90EAA74216
:1067E000A8BFA646B742B8BFB64607EE90EAF8EE95
:1067F000E77A052AC1ED047A3CF403AF90ED147AF0
:10680000DDED117AE7EE067AB0EE457AA4EE277A4E
:10681000B4EEC57AF1EE10FAF0EE477AB8BFF0EEBA
:10682000667AFDEEE77A17EE907A17EE90EAA742C5
:10683000A8BFA646B742B8BFB64607EE90EAF8EE44
:10684000E77A062AC1ED057A3CF4DBAE90ED187AC2
:10685000DDED127AE7EE067AB0EE457AA4EE277AFD
:10686000B4EEC57AF1EE10FAF0EE477AB8BFF0EE6A
:10687000667AFDEEE77A17EE907A17EE90EAA74275
:10688000A8BFA646B742B8BFB64607EE90EAF8EEF4
:10689000E77A072AC1ED067A3CF4B3AE90ED1C7A94
:1068A000DDED137AE7EE067AB0EE457AA4EE277AAC
:1068B000B4EEC57AF1EE10FAF0EE477AB8BFF0EE1A
:1068C000667AFDEEE77A17EE907A17EE90EAA74225
:1068D000A8BFA646B742B8BFB64607EE90EAF8EEA4
:1068E000E77A082AC1ED077A3CF48BAE90ED207A66
:1068F000DDED147AE7EE067AB0EE457AA4EE277A5B
:10690000B4EEC57AF1EE10FAF0EE477AB8BFF0EEC9
:10691000667AFDEEE77A17EE907A17EE90EAA742D4
:10692000A8BFA646B742B8BFB64607EE90EAF8EE53
:10693000E77A092AC1ED087A3CF463AE90ED247A37
:10694000DDED157AE7EE067AB0EE457AA4EE277A09
:10695000B4EEC57AF1EE10FAF0EE477AB8BFF0EE79
:10696000667AFDEEE77A17EE907A17EE90EAA74284
:10697000A8BFA646B742B8BFB64607EE90EAF8EE03
:10698000E77A0A2AC1ED097A3CF43BAE90ED287A09
:10699000DDED167AE7EE067AB0EE457AA4EE277AB8
:1069A000B4EEC57AF1EE10FAF0EE477AB8BFF0EE29
:1069B000667AFDEEE77A17EE907A17EE90EAA74234
:1069C000A8BFA646B742B8BFB64607EE90EAF8EEB3
:1069D000E77A0B2AC1ED0A7A3CF413AE90ED2C7ADB
:1069E000DDED177AE7EE067AB0EE457AA4EE277A67
:1069F000B4EEC75AF0EE477AF1EE10FAC8BFF0EEE7
:106A0000667AFDEEE77AFCF7EEBDBDEEE67AFCF7BE
:106A10005ABE8223FEF7A7BF5FEDE77AFEF76FBF8E
:106A2000DBF8B45151003DB18B1800EB83036D7856
:106A30005B78AB42BCF420A80A4400EB8200002241
:106A4000CBF8B401ABF80222CBF80422FCF714B85F
:106A50009FEDCD7AFFF752B9830001EB030E0BEBEC
:106A60000307CA4B03EBCC1C5FEA990300F01C83BD
:106A700001331B0105930CEB03000EF110010CF127
:106A8000100307F1100213ED024A13ED035A13ED40
:106A9000016A13ED047A51ED024A51ED035A51EDAA
:106AA000016A51ED047A64EE244A65EE255A66EED9
:106AB000266A67EE277A1033834242ED024A42ED9E
:106AC000035A42ED016A42ED047A01F1100102F12C
:106AD0001002D8D1059B103B0CEB03010EEB030217
:106AE0003B4419F003093EF4BBADB1EC017AF2EC82
:106AF000017A67EE277AB9F10109E3EC017AF4D162
:106B0000FEF7AEBD07EE907ADFEDA16AB8EEE77A48
:106B100066EEA65A9FED9F5A9FED9F6ADFED9F7A22
:106B2000A5EE856A26EEA55AE5EE867AE5EE276A99
:106B300026EE870AFFF7D9B8FDEEC57A0CAB03EB5A
:106B4000820217EE90EAFDEEE67A07911146CDF843
:106B500020B04A46924EDFF88CC2CDED047ACDF8D3
:106B6000188017EE90BA894605E09945ECEC017A59
:106B700006F1100678D096ED007AF3EC017AE7EE94
:106B8000067AB0EE457AA4EE277AF0EE477ADAB9C3
:106B9000FDEEC77A714617EE908AC64503DCA04524
:106BA0004146A8BF214607EE901AF8EEE77A002882
:106BB000DBD107990029D8D10699884605998845DF
:106BC000B8BFF0EE667AD0E737B1B4EE475AF1EECF
:106BD00010FAC8BFF0EE667AFDEEE77A594617EE76
:106BE000908AC345DFDCDAE7FDEEE67A0CABCDED4B
:106BF000047AFDEEC57A03EB82020791CDF820B04E
:106C00001146674EDFF8DCC1DDF810B0CDF8188012
:106C100017EE90EA4A46B1EE444A894696ED007A6C
:106C2000F3EC017AE7EE067AB0EE437AA4EE277A27
:106C3000F0EE477AE2B9FDEEC77A714617EE908A18
:106C4000C64504DCA04517EE901AA8BF214607EE02
:106C5000901AF8EEE77A002800F0CE814B45ECEC74
:106C6000017A06F11006D9D1DDF820B0FCF7CCBCD2
:106C700037B1B4EE475AF1EE10FAC8BFF0EE667ABB
:106C8000BDEEE77A07EE90BA17EE101A8B4506DCD8
:106C900017EE101AA142A8BF214607EE901AF8EE8F
:106CA000E77AD8E73F4820F01DFAFDF7C7BF3E4816
:106CB00020F018FAFDF7BCBF3C4820F013FAFDF7AE
:106CC000B1BF3B4B9FED3B6AB3F90020B3F90230F3
:106CD00007EE902A06EE903AF8EEE77AF8EEE66ACA
:106CE00027EEE87A60EE277AA0EE267AE8EEA67A1A
:106CF00027EE067A67EE867AA6E4BCF838109FED98
:106D00002E7A07EE901AF8EEE77A2C4967EE877A2A
:106D1000C1ED007AFCF7C3BE2949FCF716BF294F25
:106D20007A69002A3BF43CAD27493A68088827492C
:106D300091FBF0F111607B74FBF732BD9FED128A7D
:106D4000FFF7ACBB9FED108AFFF7EFBB9FED200A6A
:106D5000204B099325EE800A24F02EFE1E4FDBF80F
:106D6000A861F880FDF72ABFA3F50C43A03B30E4EF
:106D7000A3F50C43A03B47E42B4631E41749184ADE
:106D80008E46FEF75CBC00BF00000000D8840020E7
:106D900084F9223F92E741B99730083C15A82ABEF2
:106DA000184E002064B4002020B4002034B5002028
:106DB0006C680020CDCCCC3D6F12833A9800002047
:106DC000D0CF00203CC7002054C7002020A10700DE
:106DD0000000C8429C840020E4CE00205886002099
:106DE000A42900205C44002091ED000A0593049240
:106DF000039124F0E1FDDFF8A4E3DA4FDEF8ECE0E4
:106E0000DFF89CC338808CFB0E3C4FEAEE70C0EB81
:106E1000AC1007EE900AF8EEE77A03A9FDEEE77AE8
:106E20000EC917EE900A7880FCF794BE07EE905AD0
:106E3000B8EEE76ADFEDCC7A9FEDCC7A8BF884511F
:106E400026EE276A76EE077AFDEEE76A16EE903AAE
:106E50002033402B40F23B819FEDC57AC54BFDEEC0
:106E6000C67A83ED017A17EE903A2033402B00F278
:106E70002B81DFEDC17AB4EEE76AF1EE10FA40F350
:106E80004D82DFEDBE5ADFEDBE7A01E0B0EE666AFC
:106E9000B4EEE76AF1EE10FA76EE656AF6DCDFED45
:106EA000C27AF4EEE76AF1EE10FA40F13482DFEDD7
:106EB000B35A9FEDB46A01E0F0EE676AF4EEC66A79
:106EC000F1EE10FA76EEA57AF6D4DFEDA86AF4EECC
:106ED000E67AF1EE10FA40F3EB80DFEDA76A76EE8A
:106EE000E77A67EEA75A9FEDA85A9FEDA86ADFEDF3
:106EF000A86AA5EE856A27EEA55AE5EE866AE5EE54
:106F0000267ACBED627AFEF74CB9FBF7CBF8049BFF
:106F1000944F99F80020DBF8A8619AF80080C01A15
:106F2000B880FEF79BBCFBF7BDF8049B8D4FDBF8E8
:106F3000AC91DBF8A861C01A7880FEF7FEBBFBF7C6
:106F4000B1F8049B874F9AF80080C01A7880FEF74A
:106F50004ABADFED897AF4EEE76AF1EE10FA40F30F
:106F6000E381DFED865A9FED866A01E0F0EE676A05
:106F7000F4EEC66AF1EE10FA76EEE57AF6DCDFEDB5
:106F80008A6AF4EEE67AF1EE10FA40F1CA81DFED9A
:106F90007B5A9FED7C6A01E0F0EE667AF4EEC67AE9
:106FA000F1EE10FA77EEA56AF6D4DFED707AF4EE22
:106FB000E76AF1EE10FA04DDDFED6F7A77EEE66A4C
:106FC000A6E5DFED787AF4EEE76AF1EE10FA44BF59
:106FD000DFED757A77EEE66A9AE56E4B1B78002B4B
:106FE0005ED00023FEF7D3BD2B7DFFF735B96A498C
:106FF00001F1800EFEF718BC079900297FF42EAE30
:107000000699884605998845B8BFF0EE667A25E668
:10701000F880A4F8A850FBF736BD93F8FF21AA2A00
:107020007FF459A9D3F8C6214AB193F8C211A1F14E
:107030000B0001282DD901F0F701062929D0D3F83A
:10704000D6214AB193F8D211A1F10B00012820D921
:1070500001F0F70106291CD0D3F8E6214AB193F8D4
:10706000E211A1F10B00012813D901F0F701062963
:107070000FD0D3F8F621002A3FF42DA993F8F2316E
:10708000A3F10B01012904D903F0F703062B7FF4C8
:1070900022A941F2FC1101236A50AB70FFF726B917
:1070A0001EF014FDFBF7E8BC3B467246614618E54E
:1070B000DFED3C6AF4EEE67AF1EE10FA44BFDFED64
:1070C0003A6A76EEE77A0CE7DFED297A19E7B4EE53
:1070D000C76AF1EE10FA0FDDB0EE677ADFED275ADE
:1070E000DFED276A01E0B0EE677AB4EEE67AF1EE02
:1070F00010FA77EEE57AF6DC9FED2B7AF4EEC77A9C
:10710000F1EE10FA0FD5B0EE677ADFED1C5ADFED25
:107110001D6A01E0B0EE677AB4EEE67AF1EE10FA9D
:1071200077EEA57AF6D49FED117AF4EEC77AF1EEF8
:1071300010FA42DD9FED107A77EE677A67EEA75A74
:107140009FED115ADFED116A9FED117AE5EE856A28
:1071500027EEA55AA5EEA67AE5EE077AB0EE677A95
:107160007CE600BFE4CE002035FA8E3CDB0FC93F41
:107170000000000098000020DB0F4940DB0FC940F1
:10718000E4CB1641E4CB16C192E741B99730083CF5
:1071900015A82ABECFCF0020A4290020DC1600208D
:1071A000D34D6210DB0FC9BFDB0F49C09BF8E03144
:1071B000002B7BF419ABFBF700BB1FED067AF4EE56
:1071C000C77AF1EE10FA44BF1FED097A77EE677ABD
:1071D000B4E79AF80010132900F091804BB106F53E
